
/home/bartosz/Desktop/III_sem_master/master_thesis/rpi_pico_vga_pio/build/vga_interface_pio.elf:     file format elf32-littlearm

Sections:
Idx Name          Size      VMA       LMA       File off  Algn
  0 .boot2        00000100  10000000  10000000  00001000  2**0
                  CONTENTS, ALLOC, LOAD, READONLY, CODE
  1 .text         00004d00  10000100  10000100  00001100  2**3
                  CONTENTS, ALLOC, LOAD, READONLY, CODE
  2 .rodata       0000113c  10004e00  10004e00  00005e00  2**3
                  CONTENTS, ALLOC, LOAD, READONLY, DATA
  3 .binary_info  00000024  10005f3c  10005f3c  00006f3c  2**2
                  CONTENTS, ALLOC, LOAD, READONLY, DATA
  4 .ram_vector_table 000000c0  20000000  20000000  00008000  2**2
                  ALLOC
  5 .data         00000244  200000c0  10005f60  000070c0  2**4
                  CONTENTS, ALLOC, LOAD, READONLY, CODE
  6 .uninitialized_data 00000000  20000304  20000304  00007304  2**0
                  CONTENTS
  7 .scratch_x    00000000  20040000  20040000  00007304  2**0
                  CONTENTS
  8 .scratch_y    00000000  20041000  20041000  00007304  2**0
                  CONTENTS
  9 .bss          00025be0  20000308  20000308  00008000  2**3
                  ALLOC
 10 .heap         00000800  20025ee8  20025ee8  00007304  2**2
                  CONTENTS, READONLY
 11 .stack_dummy  00000800  20041000  20041000  00007b20  2**5
                  CONTENTS, READONLY
 12 .ARM.attributes 00000028  00000000  00000000  00008320  2**0
                  CONTENTS, READONLY
 13 .comment      00000049  00000000  00000000  00008348  2**0
                  CONTENTS, READONLY
 14 .debug_info   0001aabe  00000000  00000000  00008391  2**0
                  CONTENTS, READONLY, DEBUGGING, OCTETS
 15 .debug_abbrev 00004b91  00000000  00000000  00022e4f  2**0
                  CONTENTS, READONLY, DEBUGGING, OCTETS
 16 .debug_loc    00011ece  00000000  00000000  000279e0  2**0
                  CONTENTS, READONLY, DEBUGGING, OCTETS
 17 .debug_aranges 00000f88  00000000  00000000  000398b0  2**3
                  CONTENTS, READONLY, DEBUGGING, OCTETS
 18 .debug_ranges 00003cf8  00000000  00000000  0003a838  2**3
                  CONTENTS, READONLY, DEBUGGING, OCTETS
 19 .debug_line   00011a2d  00000000  00000000  0003e530  2**0
                  CONTENTS, READONLY, DEBUGGING, OCTETS
 20 .debug_str    000048cf  00000000  00000000  0004ff5d  2**0
                  CONTENTS, READONLY, DEBUGGING, OCTETS
 21 .debug_frame  00001c44  00000000  00000000  0005482c  2**2
                  CONTENTS, READONLY, DEBUGGING, OCTETS

/home/bartosz/Desktop/III_sem_master/master_thesis/rpi_pico_vga_pio/build/vga_interface_pio.elf:     file format elf32-littlearm


Disassembly of section .boot2:

10000000 <__boot2_start__>:
10000000:	4b32b500 	.word	0x4b32b500
10000004:	60582021 	.word	0x60582021
10000008:	21026898 	.word	0x21026898
1000000c:	60984388 	.word	0x60984388
10000010:	611860d8 	.word	0x611860d8
10000014:	4b2e6158 	.word	0x4b2e6158
10000018:	60992100 	.word	0x60992100
1000001c:	61592102 	.word	0x61592102
10000020:	22f02101 	.word	0x22f02101
10000024:	492b5099 	.word	0x492b5099
10000028:	21016019 	.word	0x21016019
1000002c:	20356099 	.word	0x20356099
10000030:	f844f000 	.word	0xf844f000
10000034:	42902202 	.word	0x42902202
10000038:	2106d014 	.word	0x2106d014
1000003c:	f0006619 	.word	0xf0006619
10000040:	6e19f834 	.word	0x6e19f834
10000044:	66192101 	.word	0x66192101
10000048:	66182000 	.word	0x66182000
1000004c:	f000661a 	.word	0xf000661a
10000050:	6e19f82c 	.word	0x6e19f82c
10000054:	6e196e19 	.word	0x6e196e19
10000058:	f0002005 	.word	0xf0002005
1000005c:	2101f82f 	.word	0x2101f82f
10000060:	d1f94208 	.word	0xd1f94208
10000064:	60992100 	.word	0x60992100
10000068:	6019491b 	.word	0x6019491b
1000006c:	60592100 	.word	0x60592100
10000070:	481b491a 	.word	0x481b491a
10000074:	21016001 	.word	0x21016001
10000078:	21eb6099 	.word	0x21eb6099
1000007c:	21a06619 	.word	0x21a06619
10000080:	f0006619 	.word	0xf0006619
10000084:	2100f812 	.word	0x2100f812
10000088:	49166099 	.word	0x49166099
1000008c:	60014814 	.word	0x60014814
10000090:	60992101 	.word	0x60992101
10000094:	2800bc01 	.word	0x2800bc01
10000098:	4700d000 	.word	0x4700d000
1000009c:	49134812 	.word	0x49134812
100000a0:	c8036008 	.word	0xc8036008
100000a4:	8808f380 	.word	0x8808f380
100000a8:	b5034708 	.word	0xb5034708
100000ac:	20046a99 	.word	0x20046a99
100000b0:	d0fb4201 	.word	0xd0fb4201
100000b4:	42012001 	.word	0x42012001
100000b8:	bd03d1f8 	.word	0xbd03d1f8
100000bc:	6618b502 	.word	0x6618b502
100000c0:	f7ff6618 	.word	0xf7ff6618
100000c4:	6e18fff2 	.word	0x6e18fff2
100000c8:	bd026e18 	.word	0xbd026e18
100000cc:	40020000 	.word	0x40020000
100000d0:	18000000 	.word	0x18000000
100000d4:	00070000 	.word	0x00070000
100000d8:	005f0300 	.word	0x005f0300
100000dc:	00002221 	.word	0x00002221
100000e0:	180000f4 	.word	0x180000f4
100000e4:	a0002022 	.word	0xa0002022
100000e8:	10000100 	.word	0x10000100
100000ec:	e000ed08 	.word	0xe000ed08
	...
100000fc:	7a4eb274 	.word	0x7a4eb274

Disassembly of section .text:

10000100 <__VECTOR_TABLE>:
10000100:	20042000 	.word	0x20042000
10000104:	100001f7 	.word	0x100001f7
10000108:	100001c3 	.word	0x100001c3
1000010c:	100001c5 	.word	0x100001c5
10000110:	100001c1 	.word	0x100001c1
10000114:	100001c1 	.word	0x100001c1
10000118:	100001c1 	.word	0x100001c1
1000011c:	100001c1 	.word	0x100001c1
10000120:	100001c1 	.word	0x100001c1
10000124:	100001c1 	.word	0x100001c1
10000128:	100001c1 	.word	0x100001c1
1000012c:	100001c7 	.word	0x100001c7
10000130:	100001c1 	.word	0x100001c1
10000134:	100001c1 	.word	0x100001c1
10000138:	100001c9 	.word	0x100001c9
1000013c:	100001cb 	.word	0x100001cb
10000140:	100001cd 	.word	0x100001cd
10000144:	100001cd 	.word	0x100001cd
10000148:	100001cd 	.word	0x100001cd
1000014c:	100001cd 	.word	0x100001cd
10000150:	100001cd 	.word	0x100001cd
10000154:	100001cd 	.word	0x100001cd
10000158:	100001cd 	.word	0x100001cd
1000015c:	100001cd 	.word	0x100001cd
10000160:	100001cd 	.word	0x100001cd
10000164:	100001cd 	.word	0x100001cd
10000168:	100001cd 	.word	0x100001cd
1000016c:	100001cd 	.word	0x100001cd
10000170:	100001cd 	.word	0x100001cd
10000174:	100001cd 	.word	0x100001cd
10000178:	100001cd 	.word	0x100001cd
1000017c:	100001cd 	.word	0x100001cd
10000180:	100001cd 	.word	0x100001cd
10000184:	100001cd 	.word	0x100001cd
10000188:	100001cd 	.word	0x100001cd
1000018c:	100001cd 	.word	0x100001cd
10000190:	100001cd 	.word	0x100001cd
10000194:	100001cd 	.word	0x100001cd
10000198:	100001cd 	.word	0x100001cd
1000019c:	100001cd 	.word	0x100001cd
100001a0:	100001cd 	.word	0x100001cd
100001a4:	100001cd 	.word	0x100001cd
100001a8:	100001cd 	.word	0x100001cd
100001ac:	100001cd 	.word	0x100001cd
100001b0:	100001cd 	.word	0x100001cd
100001b4:	100001cd 	.word	0x100001cd
100001b8:	100001cd 	.word	0x100001cd
100001bc:	100001cd 	.word	0x100001cd

100001c0 <isr_invalid>:
100001c0:	be00      	bkpt	0x0000

100001c2 <isr_nmi>:
100001c2:	be00      	bkpt	0x0000

100001c4 <isr_hardfault>:
100001c4:	be00      	bkpt	0x0000

100001c6 <isr_svcall>:
100001c6:	be00      	bkpt	0x0000

100001c8 <isr_pendsv>:
100001c8:	be00      	bkpt	0x0000

100001ca <isr_systick>:
100001ca:	be00      	bkpt	0x0000

100001cc <__unhandled_user_irq>:
100001cc:	f3ef 8005 	mrs	r0, IPSR
100001d0:	3810      	subs	r0, #16

100001d2 <unhandled_user_irq_num_in_r0>:
100001d2:	be00      	bkpt	0x0000

100001d4 <binary_info_header>:
100001d4:	7188ebf2 	.word	0x7188ebf2
100001d8:	10005f3c 	.word	0x10005f3c
100001dc:	10005f60 	.word	0x10005f60
100001e0:	10000234 	.word	0x10000234
100001e4:	e71aa390 	.word	0xe71aa390

100001e8 <_entry_point>:
100001e8:	2000      	movs	r0, #0
100001ea:	491f      	ldr	r1, [pc, #124]	; (10000268 <hold_non_core0_in_bootrom+0xa>)
100001ec:	6008      	str	r0, [r1, #0]
100001ee:	c806      	ldmia	r0!, {r1, r2}
100001f0:	f381 8808 	msr	MSP, r1
100001f4:	4710      	bx	r2

100001f6 <_reset_handler>:
100001f6:	481d      	ldr	r0, [pc, #116]	; (1000026c <hold_non_core0_in_bootrom+0xe>)
100001f8:	6800      	ldr	r0, [r0, #0]
100001fa:	2800      	cmp	r0, #0
100001fc:	d12f      	bne.n	1000025e <hold_non_core0_in_bootrom>
100001fe:	a40d      	add	r4, pc, #52	; (adr r4, 10000234 <data_cpy_table>)
10000200:	cc0e      	ldmia	r4!, {r1, r2, r3}
10000202:	2900      	cmp	r1, #0
10000204:	d002      	beq.n	1000020c <_reset_handler+0x16>
10000206:	f000 f812 	bl	1000022e <data_cpy>
1000020a:	e7f9      	b.n	10000200 <_reset_handler+0xa>
1000020c:	4918      	ldr	r1, [pc, #96]	; (10000270 <hold_non_core0_in_bootrom+0x12>)
1000020e:	4a19      	ldr	r2, [pc, #100]	; (10000274 <hold_non_core0_in_bootrom+0x16>)
10000210:	2000      	movs	r0, #0
10000212:	e000      	b.n	10000216 <bss_fill_test>

10000214 <bss_fill_loop>:
10000214:	c101      	stmia	r1!, {r0}

10000216 <bss_fill_test>:
10000216:	4291      	cmp	r1, r2
10000218:	d1fc      	bne.n	10000214 <bss_fill_loop>

1000021a <platform_entry>:
1000021a:	4917      	ldr	r1, [pc, #92]	; (10000278 <hold_non_core0_in_bootrom+0x1a>)
1000021c:	4788      	blx	r1
1000021e:	4917      	ldr	r1, [pc, #92]	; (1000027c <hold_non_core0_in_bootrom+0x1e>)
10000220:	4788      	blx	r1
10000222:	4917      	ldr	r1, [pc, #92]	; (10000280 <hold_non_core0_in_bootrom+0x22>)
10000224:	4788      	blx	r1
10000226:	be00      	bkpt	0x0000
10000228:	e7fd      	b.n	10000226 <platform_entry+0xc>

1000022a <data_cpy_loop>:
1000022a:	c901      	ldmia	r1!, {r0}
1000022c:	c201      	stmia	r2!, {r0}

1000022e <data_cpy>:
1000022e:	429a      	cmp	r2, r3
10000230:	d3fb      	bcc.n	1000022a <data_cpy_loop>
10000232:	4770      	bx	lr

10000234 <data_cpy_table>:
10000234:	10005f60 	.word	0x10005f60
10000238:	200000c0 	.word	0x200000c0
1000023c:	20000304 	.word	0x20000304
10000240:	100061a4 	.word	0x100061a4
10000244:	20040000 	.word	0x20040000
10000248:	20040000 	.word	0x20040000
1000024c:	100061a4 	.word	0x100061a4
10000250:	20041000 	.word	0x20041000
10000254:	20041000 	.word	0x20041000
10000258:	00000000 	.word	0x00000000
1000025c:	4770      	bx	lr

1000025e <hold_non_core0_in_bootrom>:
1000025e:	4809      	ldr	r0, [pc, #36]	; (10000284 <hold_non_core0_in_bootrom+0x26>)
10000260:	f003 fa40 	bl	100036e4 <rom_func_lookup>
10000264:	4700      	bx	r0
10000266:	0000      	.short	0x0000
10000268:	e000ed08 	.word	0xe000ed08
1000026c:	d0000000 	.word	0xd0000000
10000270:	20000308 	.word	0x20000308
10000274:	20025ee8 	.word	0x20025ee8
10000278:	1000246d 	.word	0x1000246d
1000027c:	100003bd 	.word	0x100003bd
10000280:	10002429 	.word	0x10002429
10000284:	00005657 	.word	0x00005657

10000288 <__bi_50>:
10000288:	50520006 5360b3ab 10005de8              ..RP..`S.]..

10000294 <__bi_38>:
10000294:	50520006 02031c86 10005df8              ..RP.....]..

100002a0 <__bi_30>:
100002a0:	50520006 9da22254 10005e0c              ..RPT"...^..

100002ac <__bi_22>:
100002ac:	50520005 68f465de 100061a4              ..RP.e.h.a..

100002b8 <_init>:
100002b8:	b5f8      	push	{r3, r4, r5, r6, r7, lr}
100002ba:	46c0      	nop			; (mov r8, r8)

100002bc <__do_global_dtors_aux>:
100002bc:	b510      	push	{r4, lr}
100002be:	4c06      	ldr	r4, [pc, #24]	; (100002d8 <__do_global_dtors_aux+0x1c>)
100002c0:	7823      	ldrb	r3, [r4, #0]
100002c2:	2b00      	cmp	r3, #0
100002c4:	d107      	bne.n	100002d6 <__do_global_dtors_aux+0x1a>
100002c6:	4b05      	ldr	r3, [pc, #20]	; (100002dc <__do_global_dtors_aux+0x20>)
100002c8:	2b00      	cmp	r3, #0
100002ca:	d002      	beq.n	100002d2 <__do_global_dtors_aux+0x16>
100002cc:	4804      	ldr	r0, [pc, #16]	; (100002e0 <__do_global_dtors_aux+0x24>)
100002ce:	e000      	b.n	100002d2 <__do_global_dtors_aux+0x16>
100002d0:	bf00      	nop
100002d2:	2301      	movs	r3, #1
100002d4:	7023      	strb	r3, [r4, #0]
100002d6:	bd10      	pop	{r4, pc}
100002d8:	20000408 	.word	0x20000408
100002dc:	00000000 	.word	0x00000000
100002e0:	10004e00 	.word	0x10004e00

100002e4 <frame_dummy>:
100002e4:	4b04      	ldr	r3, [pc, #16]	; (100002f8 <frame_dummy+0x14>)
100002e6:	b510      	push	{r4, lr}
100002e8:	2b00      	cmp	r3, #0
100002ea:	d003      	beq.n	100002f4 <frame_dummy+0x10>
100002ec:	4903      	ldr	r1, [pc, #12]	; (100002fc <frame_dummy+0x18>)
100002ee:	4804      	ldr	r0, [pc, #16]	; (10000300 <frame_dummy+0x1c>)
100002f0:	e000      	b.n	100002f4 <frame_dummy+0x10>
100002f2:	bf00      	nop
100002f4:	bd10      	pop	{r4, pc}
100002f6:	46c0      	nop			; (mov r8, r8)
100002f8:	00000000 	.word	0x00000000
100002fc:	2000040c 	.word	0x2000040c
10000300:	10004e00 	.word	0x10004e00

10000304 <pio_get_default_sm_config>:
10000304:	b510      	push	{r4, lr}
10000306:	0004      	movs	r4, r0
10000308:	2210      	movs	r2, #16
1000030a:	2100      	movs	r1, #0
1000030c:	f004 f934 	bl	10004578 <__wrap_memset>
10000310:	2380      	movs	r3, #128	; 0x80
10000312:	025b      	lsls	r3, r3, #9
10000314:	6023      	str	r3, [r4, #0]
10000316:	23f8      	movs	r3, #248	; 0xf8
10000318:	025b      	lsls	r3, r3, #9
1000031a:	6063      	str	r3, [r4, #4]
1000031c:	2380      	movs	r3, #128	; 0x80
1000031e:	02db      	lsls	r3, r3, #11
10000320:	60a3      	str	r3, [r4, #8]
10000322:	23c0      	movs	r3, #192	; 0xc0
10000324:	031b      	lsls	r3, r3, #12
10000326:	60a3      	str	r3, [r4, #8]
10000328:	0020      	movs	r0, r4
1000032a:	bd10      	pop	{r4, pc}

1000032c <dma_channel_get_default_config>:
1000032c:	b510      	push	{r4, lr}
1000032e:	0003      	movs	r3, r0
10000330:	480e      	ldr	r0, [pc, #56]	; (1000036c <dma_channel_get_default_config+0x40>)
10000332:	2b0c      	cmp	r3, #12
10000334:	d814      	bhi.n	10000360 <dma_channel_get_default_config+0x34>
10000336:	4a0e      	ldr	r2, [pc, #56]	; (10000370 <dma_channel_get_default_config+0x44>)
10000338:	4010      	ands	r0, r2
1000033a:	02db      	lsls	r3, r3, #11
1000033c:	4318      	orrs	r0, r3
1000033e:	230c      	movs	r3, #12
10000340:	4398      	bics	r0, r3
10000342:	3b04      	subs	r3, #4
10000344:	4318      	orrs	r0, r3
10000346:	4b0b      	ldr	r3, [pc, #44]	; (10000374 <dma_channel_get_default_config+0x48>)
10000348:	4018      	ands	r0, r3
1000034a:	4b0b      	ldr	r3, [pc, #44]	; (10000378 <dma_channel_get_default_config+0x4c>)
1000034c:	4018      	ands	r0, r3
1000034e:	4b0b      	ldr	r3, [pc, #44]	; (1000037c <dma_channel_get_default_config+0x50>)
10000350:	4018      	ands	r0, r3
10000352:	2301      	movs	r3, #1
10000354:	4318      	orrs	r0, r3
10000356:	4b0a      	ldr	r3, [pc, #40]	; (10000380 <dma_channel_get_default_config+0x54>)
10000358:	4018      	ands	r0, r3
1000035a:	2302      	movs	r3, #2
1000035c:	4398      	bics	r0, r3
1000035e:	bd10      	pop	{r4, pc}
10000360:	4b08      	ldr	r3, [pc, #32]	; (10000384 <dma_channel_get_default_config+0x58>)
10000362:	4a09      	ldr	r2, [pc, #36]	; (10000388 <dma_channel_get_default_config+0x5c>)
10000364:	21c3      	movs	r1, #195	; 0xc3
10000366:	4809      	ldr	r0, [pc, #36]	; (1000038c <dma_channel_get_default_config+0x60>)
10000368:	f002 f862 	bl	10002430 <__assert_func>
1000036c:	001f8010 	.word	0x001f8010
10000370:	ffff87ff 	.word	0xffff87ff
10000374:	fffff83f 	.word	0xfffff83f
10000378:	ffbfffff 	.word	0xffbfffff
1000037c:	ffdfffff 	.word	0xffdfffff
10000380:	ff7fffff 	.word	0xff7fffff
10000384:	10004e00 	.word	0x10004e00
10000388:	10004ea4 	.word	0x10004ea4
1000038c:	10004e20 	.word	0x10004e20

10000390 <draw_one_pixel>:
10000390:	000b      	movs	r3, r1
10000392:	0089      	lsls	r1, r1, #2
10000394:	18c9      	adds	r1, r1, r3
10000396:	01c9      	lsls	r1, r1, #7
10000398:	1809      	adds	r1, r1, r0
1000039a:	07c3      	lsls	r3, r0, #31
1000039c:	d506      	bpl.n	100003ac <draw_one_pixel+0x1c>
1000039e:	0849      	lsrs	r1, r1, #1
100003a0:	00d2      	lsls	r2, r2, #3
100003a2:	4805      	ldr	r0, [pc, #20]	; (100003b8 <draw_one_pixel+0x28>)
100003a4:	5c43      	ldrb	r3, [r0, r1]
100003a6:	431a      	orrs	r2, r3
100003a8:	5442      	strb	r2, [r0, r1]
100003aa:	4770      	bx	lr
100003ac:	0849      	lsrs	r1, r1, #1
100003ae:	4b02      	ldr	r3, [pc, #8]	; (100003b8 <draw_one_pixel+0x28>)
100003b0:	5c58      	ldrb	r0, [r3, r1]
100003b2:	4302      	orrs	r2, r0
100003b4:	545a      	strb	r2, [r3, r1]
100003b6:	e7f8      	b.n	100003aa <draw_one_pixel+0x1a>
100003b8:	200006e4 	.word	0x200006e4

100003bc <main>:
100003bc:	b5f0      	push	{r4, r5, r6, r7, lr}
100003be:	46de      	mov	lr, fp
100003c0:	4657      	mov	r7, sl
100003c2:	464e      	mov	r6, r9
100003c4:	4645      	mov	r5, r8
100003c6:	b5e0      	push	{r5, r6, r7, lr}
100003c8:	b08f      	sub	sp, #60	; 0x3c
100003ca:	4cc7      	ldr	r4, [pc, #796]	; (100006e8 <main+0x32c>)
100003cc:	49c7      	ldr	r1, [pc, #796]	; (100006ec <main+0x330>)
100003ce:	0020      	movs	r0, r4
100003d0:	f004 fbe4 	bl	10004b9c <pio_add_program>
100003d4:	4682      	mov	sl, r0
100003d6:	49c6      	ldr	r1, [pc, #792]	; (100006f0 <main+0x334>)
100003d8:	0020      	movs	r0, r4
100003da:	f004 fbdf 	bl	10004b9c <pio_add_program>
100003de:	9003      	str	r0, [sp, #12]
100003e0:	49c4      	ldr	r1, [pc, #784]	; (100006f4 <main+0x338>)
100003e2:	0020      	movs	r0, r4
100003e4:	f004 fbda 	bl	10004b9c <pio_add_program>
100003e8:	9004      	str	r0, [sp, #16]
100003ea:	2000      	movs	r0, #0
100003ec:	f7ff ff9e 	bl	1000032c <dma_channel_get_default_config>
100003f0:	0004      	movs	r4, r0
100003f2:	2001      	movs	r0, #1
100003f4:	f7ff ff9a 	bl	1000032c <dma_channel_get_default_config>
100003f8:	0005      	movs	r5, r0
100003fa:	f004 fa27 	bl	1000484c <stdio_init_all>
100003fe:	f000 f99b 	bl	10000738 <setup_default_uart>
10000402:	2019      	movs	r0, #25
10000404:	f000 f9b4 	bl	10000770 <gpio_init>
10000408:	23d0      	movs	r3, #208	; 0xd0
1000040a:	061b      	lsls	r3, r3, #24
1000040c:	2280      	movs	r2, #128	; 0x80
1000040e:	0492      	lsls	r2, r2, #18
10000410:	625a      	str	r2, [r3, #36]	; 0x24
10000412:	2700      	movs	r7, #0
10000414:	46d0      	mov	r8, sl
10000416:	e034      	b.n	10000482 <main+0xc6>
10000418:	23a0      	movs	r3, #160	; 0xa0
1000041a:	005b      	lsls	r3, r3, #1
1000041c:	429f      	cmp	r7, r3
1000041e:	db17      	blt.n	10000450 <main+0x94>
10000420:	2eef      	cmp	r6, #239	; 0xef
10000422:	dc15      	bgt.n	10000450 <main+0x94>
10000424:	2204      	movs	r2, #4
10000426:	0031      	movs	r1, r6
10000428:	0038      	movs	r0, r7
1000042a:	f7ff ffb1 	bl	10000390 <draw_one_pixel>
1000042e:	3601      	adds	r6, #1
10000430:	23f0      	movs	r3, #240	; 0xf0
10000432:	005b      	lsls	r3, r3, #1
10000434:	429e      	cmp	r6, r3
10000436:	da23      	bge.n	10000480 <main+0xc4>
10000438:	23a0      	movs	r3, #160	; 0xa0
1000043a:	005b      	lsls	r3, r3, #1
1000043c:	429f      	cmp	r7, r3
1000043e:	daeb      	bge.n	10000418 <main+0x5c>
10000440:	2eef      	cmp	r6, #239	; 0xef
10000442:	dce9      	bgt.n	10000418 <main+0x5c>
10000444:	2201      	movs	r2, #1
10000446:	0031      	movs	r1, r6
10000448:	0038      	movs	r0, r7
1000044a:	f7ff ffa1 	bl	10000390 <draw_one_pixel>
1000044e:	e7ee      	b.n	1000042e <main+0x72>
10000450:	23a0      	movs	r3, #160	; 0xa0
10000452:	005b      	lsls	r3, r3, #1
10000454:	429f      	cmp	r7, r3
10000456:	da07      	bge.n	10000468 <main+0xac>
10000458:	2eef      	cmp	r6, #239	; 0xef
1000045a:	dd05      	ble.n	10000468 <main+0xac>
1000045c:	2203      	movs	r2, #3
1000045e:	0031      	movs	r1, r6
10000460:	0038      	movs	r0, r7
10000462:	f7ff ff95 	bl	10000390 <draw_one_pixel>
10000466:	e7e2      	b.n	1000042e <main+0x72>
10000468:	23a0      	movs	r3, #160	; 0xa0
1000046a:	005b      	lsls	r3, r3, #1
1000046c:	429f      	cmp	r7, r3
1000046e:	dbde      	blt.n	1000042e <main+0x72>
10000470:	2eef      	cmp	r6, #239	; 0xef
10000472:	dddc      	ble.n	1000042e <main+0x72>
10000474:	2202      	movs	r2, #2
10000476:	0031      	movs	r1, r6
10000478:	0038      	movs	r0, r7
1000047a:	f7ff ff89 	bl	10000390 <draw_one_pixel>
1000047e:	e7d6      	b.n	1000042e <main+0x72>
10000480:	3701      	adds	r7, #1
10000482:	23a0      	movs	r3, #160	; 0xa0
10000484:	009b      	lsls	r3, r3, #2
10000486:	429f      	cmp	r7, r3
10000488:	da01      	bge.n	1000048e <main+0xd2>
1000048a:	2600      	movs	r6, #0
1000048c:	e7d0      	b.n	10000430 <main+0x74>
1000048e:	46c2      	mov	sl, r8
10000490:	a80a      	add	r0, sp, #40	; 0x28
10000492:	f7ff ff37 	bl	10000304 <pio_get_default_sm_config>
10000496:	4643      	mov	r3, r8
10000498:	1c59      	adds	r1, r3, #1
1000049a:	4642      	mov	r2, r8
1000049c:	3208      	adds	r2, #8
1000049e:	9b0b      	ldr	r3, [sp, #44]	; 0x2c
100004a0:	9305      	str	r3, [sp, #20]
100004a2:	4b95      	ldr	r3, [pc, #596]	; (100006f8 <main+0x33c>)
100004a4:	469b      	mov	fp, r3
100004a6:	9b05      	ldr	r3, [sp, #20]
100004a8:	4658      	mov	r0, fp
100004aa:	4003      	ands	r3, r0
100004ac:	01c9      	lsls	r1, r1, #7
100004ae:	430b      	orrs	r3, r1
100004b0:	0312      	lsls	r2, r2, #12
100004b2:	4313      	orrs	r3, r2
100004b4:	930b      	str	r3, [sp, #44]	; 0x2c
100004b6:	2710      	movs	r7, #16
100004b8:	2210      	movs	r2, #16
100004ba:	a90a      	add	r1, sp, #40	; 0x28
100004bc:	a806      	add	r0, sp, #24
100004be:	f004 f861 	bl	10004584 <__wrap___aeabi_memcpy>
100004c2:	9b09      	ldr	r3, [sp, #36]	; 0x24
100004c4:	9305      	str	r3, [sp, #20]
100004c6:	4b8d      	ldr	r3, [pc, #564]	; (100006fc <main+0x340>)
100004c8:	4698      	mov	r8, r3
100004ca:	9a05      	ldr	r2, [sp, #20]
100004cc:	401a      	ands	r2, r3
100004ce:	23b0      	movs	r3, #176	; 0xb0
100004d0:	005b      	lsls	r3, r3, #1
100004d2:	4313      	orrs	r3, r2
100004d4:	2280      	movs	r2, #128	; 0x80
100004d6:	04d2      	lsls	r2, r2, #19
100004d8:	4313      	orrs	r3, r2
100004da:	9309      	str	r3, [sp, #36]	; 0x24
100004dc:	23a0      	movs	r3, #160	; 0xa0
100004de:	02db      	lsls	r3, r3, #11
100004e0:	9306      	str	r3, [sp, #24]
100004e2:	2106      	movs	r1, #6
100004e4:	200b      	movs	r0, #11
100004e6:	f000 f92b 	bl	10000740 <gpio_set_function>
100004ea:	4e7f      	ldr	r6, [pc, #508]	; (100006e8 <main+0x32c>)
100004ec:	2001      	movs	r0, #1
100004ee:	4681      	mov	r9, r0
100004f0:	9000      	str	r0, [sp, #0]
100004f2:	2301      	movs	r3, #1
100004f4:	220b      	movs	r2, #11
100004f6:	2100      	movs	r1, #0
100004f8:	0030      	movs	r0, r6
100004fa:	f004 fb6b 	bl	10004bd4 <pio_sm_set_consecutive_pindirs>
100004fe:	ab06      	add	r3, sp, #24
10000500:	4652      	mov	r2, sl
10000502:	2100      	movs	r1, #0
10000504:	0030      	movs	r0, r6
10000506:	f004 fbb7 	bl	10004c78 <pio_sm_init>
1000050a:	a80a      	add	r0, sp, #40	; 0x28
1000050c:	f7ff fefa 	bl	10000304 <pio_get_default_sm_config>
10000510:	9b03      	ldr	r3, [sp, #12]
10000512:	1c59      	adds	r1, r3, #1
10000514:	330d      	adds	r3, #13
10000516:	001a      	movs	r2, r3
10000518:	980b      	ldr	r0, [sp, #44]	; 0x2c
1000051a:	9005      	str	r0, [sp, #20]
1000051c:	465b      	mov	r3, fp
1000051e:	4018      	ands	r0, r3
10000520:	0003      	movs	r3, r0
10000522:	01c9      	lsls	r1, r1, #7
10000524:	430b      	orrs	r3, r1
10000526:	0312      	lsls	r2, r2, #12
10000528:	4313      	orrs	r3, r2
1000052a:	930b      	str	r3, [sp, #44]	; 0x2c
1000052c:	980d      	ldr	r0, [sp, #52]	; 0x34
1000052e:	9005      	str	r0, [sp, #20]
10000530:	00c2      	lsls	r2, r0, #3
10000532:	08d2      	lsrs	r2, r2, #3
10000534:	2180      	movs	r1, #128	; 0x80
10000536:	05c9      	lsls	r1, r1, #23
10000538:	430a      	orrs	r2, r1
1000053a:	920d      	str	r2, [sp, #52]	; 0x34
1000053c:	4a70      	ldr	r2, [pc, #448]	; (10000700 <main+0x344>)
1000053e:	4013      	ands	r3, r2
10000540:	4319      	orrs	r1, r3
10000542:	910b      	str	r1, [sp, #44]	; 0x2c
10000544:	2210      	movs	r2, #16
10000546:	a90a      	add	r1, sp, #40	; 0x28
10000548:	a806      	add	r0, sp, #24
1000054a:	f004 f81b 	bl	10004584 <__wrap___aeabi_memcpy>
1000054e:	9809      	ldr	r0, [sp, #36]	; 0x24
10000550:	9005      	str	r0, [sp, #20]
10000552:	4641      	mov	r1, r8
10000554:	4008      	ands	r0, r1
10000556:	23a0      	movs	r3, #160	; 0xa0
10000558:	005b      	lsls	r3, r3, #1
1000055a:	4303      	orrs	r3, r0
1000055c:	2280      	movs	r2, #128	; 0x80
1000055e:	04d2      	lsls	r2, r2, #19
10000560:	4313      	orrs	r3, r2
10000562:	9309      	str	r3, [sp, #36]	; 0x24
10000564:	4a67      	ldr	r2, [pc, #412]	; (10000704 <main+0x348>)
10000566:	4013      	ands	r3, r2
10000568:	22a0      	movs	r2, #160	; 0xa0
1000056a:	0192      	lsls	r2, r2, #6
1000056c:	4313      	orrs	r3, r2
1000056e:	9309      	str	r3, [sp, #36]	; 0x24
10000570:	21a0      	movs	r1, #160	; 0xa0
10000572:	02c9      	lsls	r1, r1, #11
10000574:	9106      	str	r1, [sp, #24]
10000576:	2106      	movs	r1, #6
10000578:	200a      	movs	r0, #10
1000057a:	f000 f8e1 	bl	10000740 <gpio_set_function>
1000057e:	4649      	mov	r1, r9
10000580:	9100      	str	r1, [sp, #0]
10000582:	2301      	movs	r3, #1
10000584:	220a      	movs	r2, #10
10000586:	0030      	movs	r0, r6
10000588:	f004 fb24 	bl	10004bd4 <pio_sm_set_consecutive_pindirs>
1000058c:	a906      	add	r1, sp, #24
1000058e:	000b      	movs	r3, r1
10000590:	9a03      	ldr	r2, [sp, #12]
10000592:	2101      	movs	r1, #1
10000594:	0030      	movs	r0, r6
10000596:	f004 fb6f 	bl	10004c78 <pio_sm_init>
1000059a:	a80a      	add	r0, sp, #40	; 0x28
1000059c:	f7ff feb2 	bl	10000304 <pio_get_default_sm_config>
100005a0:	9b04      	ldr	r3, [sp, #16]
100005a2:	1c99      	adds	r1, r3, #2
100005a4:	3308      	adds	r3, #8
100005a6:	001a      	movs	r2, r3
100005a8:	980b      	ldr	r0, [sp, #44]	; 0x2c
100005aa:	9003      	str	r0, [sp, #12]
100005ac:	4658      	mov	r0, fp
100005ae:	9b03      	ldr	r3, [sp, #12]
100005b0:	4018      	ands	r0, r3
100005b2:	0003      	movs	r3, r0
100005b4:	01c9      	lsls	r1, r1, #7
100005b6:	430b      	orrs	r3, r1
100005b8:	0312      	lsls	r2, r2, #12
100005ba:	4313      	orrs	r3, r2
100005bc:	930b      	str	r3, [sp, #44]	; 0x2c
100005be:	2210      	movs	r2, #16
100005c0:	a90a      	add	r1, sp, #40	; 0x28
100005c2:	a806      	add	r0, sp, #24
100005c4:	f003 ffde 	bl	10004584 <__wrap___aeabi_memcpy>
100005c8:	9909      	ldr	r1, [sp, #36]	; 0x24
100005ca:	9103      	str	r1, [sp, #12]
100005cc:	4642      	mov	r2, r8
100005ce:	400a      	ands	r2, r1
100005d0:	23c0      	movs	r3, #192	; 0xc0
100005d2:	005b      	lsls	r3, r3, #1
100005d4:	431a      	orrs	r2, r3
100005d6:	23c0      	movs	r3, #192	; 0xc0
100005d8:	051b      	lsls	r3, r3, #20
100005da:	4313      	orrs	r3, r2
100005dc:	9309      	str	r3, [sp, #36]	; 0x24
100005de:	4a4a      	ldr	r2, [pc, #296]	; (10000708 <main+0x34c>)
100005e0:	4013      	ands	r3, r2
100005e2:	210c      	movs	r1, #12
100005e4:	4688      	mov	r8, r1
100005e6:	430b      	orrs	r3, r1
100005e8:	22c0      	movs	r2, #192	; 0xc0
100005ea:	0392      	lsls	r2, r2, #14
100005ec:	4313      	orrs	r3, r2
100005ee:	9309      	str	r3, [sp, #36]	; 0x24
100005f0:	3906      	subs	r1, #6
100005f2:	200c      	movs	r0, #12
100005f4:	f000 f8a4 	bl	10000740 <gpio_set_function>
100005f8:	2106      	movs	r1, #6
100005fa:	200d      	movs	r0, #13
100005fc:	f000 f8a0 	bl	10000740 <gpio_set_function>
10000600:	2106      	movs	r1, #6
10000602:	200e      	movs	r0, #14
10000604:	f000 f89c 	bl	10000740 <gpio_set_function>
10000608:	4649      	mov	r1, r9
1000060a:	9100      	str	r1, [sp, #0]
1000060c:	2303      	movs	r3, #3
1000060e:	220c      	movs	r2, #12
10000610:	3101      	adds	r1, #1
10000612:	0030      	movs	r0, r6
10000614:	f004 fade 	bl	10004bd4 <pio_sm_set_consecutive_pindirs>
10000618:	a906      	add	r1, sp, #24
1000061a:	000b      	movs	r3, r1
1000061c:	9a04      	ldr	r2, [sp, #16]
1000061e:	2102      	movs	r1, #2
10000620:	0030      	movs	r0, r6
10000622:	f004 fb29 	bl	10004c78 <pio_sm_init>
10000626:	433c      	orrs	r4, r7
10000628:	43bd      	bics	r5, r7
1000062a:	4b38      	ldr	r3, [pc, #224]	; (1000070c <main+0x350>)
1000062c:	401c      	ands	r4, r3
1000062e:	2080      	movs	r0, #128	; 0x80
10000630:	0100      	lsls	r0, r0, #4
10000632:	4304      	orrs	r4, r0
10000634:	401d      	ands	r5, r3
10000636:	4643      	mov	r3, r8
10000638:	439c      	bics	r4, r3
1000063a:	439d      	bics	r5, r3
1000063c:	3b04      	subs	r3, #4
1000063e:	431d      	orrs	r5, r3
10000640:	3318      	adds	r3, #24
10000642:	439c      	bics	r4, r3
10000644:	439d      	bics	r5, r3
10000646:	4b32      	ldr	r3, [pc, #200]	; (10000710 <main+0x354>)
10000648:	401c      	ands	r4, r3
1000064a:	2080      	movs	r0, #128	; 0x80
1000064c:	0240      	lsls	r0, r0, #9
1000064e:	4304      	orrs	r4, r0
10000650:	23a0      	movs	r3, #160	; 0xa0
10000652:	05db      	lsls	r3, r3, #23
10000654:	4a2f      	ldr	r2, [pc, #188]	; (10000714 <main+0x358>)
10000656:	601a      	str	r2, [r3, #0]
10000658:	4a2f      	ldr	r2, [pc, #188]	; (10000718 <main+0x35c>)
1000065a:	605a      	str	r2, [r3, #4]
1000065c:	2296      	movs	r2, #150	; 0x96
1000065e:	0292      	lsls	r2, r2, #10
10000660:	609a      	str	r2, [r3, #8]
10000662:	611c      	str	r4, [r3, #16]
10000664:	4a2d      	ldr	r2, [pc, #180]	; (1000071c <main+0x360>)
10000666:	492e      	ldr	r1, [pc, #184]	; (10000720 <main+0x364>)
10000668:	6011      	str	r1, [r2, #0]
1000066a:	6053      	str	r3, [r2, #4]
1000066c:	464b      	mov	r3, r9
1000066e:	6093      	str	r3, [r2, #8]
10000670:	6115      	str	r5, [r2, #16]
10000672:	4b1d      	ldr	r3, [pc, #116]	; (100006e8 <main+0x32c>)
10000674:	685b      	ldr	r3, [r3, #4]
10000676:	03db      	lsls	r3, r3, #15
10000678:	d4fb      	bmi.n	10000672 <main+0x2b6>
1000067a:	4b1b      	ldr	r3, [pc, #108]	; (100006e8 <main+0x32c>)
1000067c:	4a29      	ldr	r2, [pc, #164]	; (10000724 <main+0x368>)
1000067e:	611a      	str	r2, [r3, #16]
10000680:	4b19      	ldr	r3, [pc, #100]	; (100006e8 <main+0x32c>)
10000682:	685b      	ldr	r3, [r3, #4]
10000684:	039b      	lsls	r3, r3, #14
10000686:	d4fb      	bmi.n	10000680 <main+0x2c4>
10000688:	4b17      	ldr	r3, [pc, #92]	; (100006e8 <main+0x32c>)
1000068a:	22e0      	movs	r2, #224	; 0xe0
1000068c:	32ff      	adds	r2, #255	; 0xff
1000068e:	615a      	str	r2, [r3, #20]
10000690:	4b15      	ldr	r3, [pc, #84]	; (100006e8 <main+0x32c>)
10000692:	685b      	ldr	r3, [r3, #4]
10000694:	035b      	lsls	r3, r3, #13
10000696:	d4fb      	bmi.n	10000690 <main+0x2d4>
10000698:	4a13      	ldr	r2, [pc, #76]	; (100006e8 <main+0x32c>)
1000069a:	2340      	movs	r3, #64	; 0x40
1000069c:	33ff      	adds	r3, #255	; 0xff
1000069e:	6193      	str	r3, [r2, #24]
100006a0:	2380      	movs	r3, #128	; 0x80
100006a2:	019b      	lsls	r3, r3, #6
100006a4:	4313      	orrs	r3, r2
100006a6:	4a20      	ldr	r2, [pc, #128]	; (10000728 <main+0x36c>)
100006a8:	601a      	str	r2, [r3, #0]
100006aa:	22a0      	movs	r2, #160	; 0xa0
100006ac:	05d2      	lsls	r2, r2, #23
100006ae:	2386      	movs	r3, #134	; 0x86
100006b0:	00db      	lsls	r3, r3, #3
100006b2:	2101      	movs	r1, #1
100006b4:	50d1      	str	r1, [r2, r3]
100006b6:	4b1d      	ldr	r3, [pc, #116]	; (1000072c <main+0x370>)
100006b8:	6a98      	ldr	r0, [r3, #40]	; 0x28
100006ba:	491d      	ldr	r1, [pc, #116]	; (10000730 <main+0x374>)
100006bc:	f003 f866 	bl	1000378c <__wrap___aeabi_uidiv>
100006c0:	0001      	movs	r1, r0
100006c2:	481c      	ldr	r0, [pc, #112]	; (10000734 <main+0x378>)
100006c4:	f004 f8b6 	bl	10004834 <__wrap_printf>
100006c8:	25d0      	movs	r5, #208	; 0xd0
100006ca:	062d      	lsls	r5, r5, #24
100006cc:	2680      	movs	r6, #128	; 0x80
100006ce:	04b6      	lsls	r6, r6, #18
100006d0:	616e      	str	r6, [r5, #20]
100006d2:	24fa      	movs	r4, #250	; 0xfa
100006d4:	0064      	lsls	r4, r4, #1
100006d6:	0020      	movs	r0, r4
100006d8:	f001 f82c 	bl	10001734 <sleep_ms>
100006dc:	61ae      	str	r6, [r5, #24]
100006de:	0020      	movs	r0, r4
100006e0:	f001 f828 	bl	10001734 <sleep_ms>
100006e4:	e7e7      	b.n	100006b6 <main+0x2fa>
100006e6:	46c0      	nop			; (mov r8, r8)
100006e8:	50200000 	.word	0x50200000
100006ec:	10004edc 	.word	0x10004edc
100006f0:	10004ef8 	.word	0x10004ef8
100006f4:	10004ec0 	.word	0x10004ec0
100006f8:	fffe007f 	.word	0xfffe007f
100006fc:	e3fffc1f 	.word	0xe3fffc1f
10000700:	9fffffff 	.word	0x9fffffff
10000704:	ffff83ff 	.word	0xffff83ff
10000708:	fc0fffe0 	.word	0xfc0fffe0
1000070c:	ffff87ff 	.word	0xffff87ff
10000710:	ffe07fff 	.word	0xffe07fff
10000714:	200006e4 	.word	0x200006e4
10000718:	50200018 	.word	0x50200018
1000071c:	50000040 	.word	0x50000040
10000720:	20000238 	.word	0x20000238
10000724:	0000028f 	.word	0x0000028f
10000728:	00000707 	.word	0x00000707
1000072c:	40054000 	.word	0x40054000
10000730:	000f4240 	.word	0x000f4240
10000734:	10004e74 	.word	0x10004e74

10000738 <setup_default_uart>:
10000738:	b510      	push	{r4, lr}
1000073a:	f004 f983 	bl	10004a44 <stdio_uart_init>
1000073e:	bd10      	pop	{r4, pc}

10000740 <gpio_set_function>:
10000740:	b510      	push	{r4, lr}
10000742:	0083      	lsls	r3, r0, #2
10000744:	4a08      	ldr	r2, [pc, #32]	; (10000768 <gpio_set_function+0x28>)
10000746:	4694      	mov	ip, r2
10000748:	4463      	add	r3, ip
1000074a:	681c      	ldr	r4, [r3, #0]
1000074c:	2240      	movs	r2, #64	; 0x40
1000074e:	4062      	eors	r2, r4
10000750:	24c0      	movs	r4, #192	; 0xc0
10000752:	4014      	ands	r4, r2
10000754:	2280      	movs	r2, #128	; 0x80
10000756:	0152      	lsls	r2, r2, #5
10000758:	4313      	orrs	r3, r2
1000075a:	601c      	str	r4, [r3, #0]
1000075c:	00c0      	lsls	r0, r0, #3
1000075e:	4b03      	ldr	r3, [pc, #12]	; (1000076c <gpio_set_function+0x2c>)
10000760:	469c      	mov	ip, r3
10000762:	4460      	add	r0, ip
10000764:	6041      	str	r1, [r0, #4]
10000766:	bd10      	pop	{r4, pc}
10000768:	4001c004 	.word	0x4001c004
1000076c:	40014000 	.word	0x40014000

10000770 <gpio_init>:
10000770:	b510      	push	{r4, lr}
10000772:	2301      	movs	r3, #1
10000774:	4083      	lsls	r3, r0
10000776:	22d0      	movs	r2, #208	; 0xd0
10000778:	0612      	lsls	r2, r2, #24
1000077a:	6293      	str	r3, [r2, #40]	; 0x28
1000077c:	6193      	str	r3, [r2, #24]
1000077e:	2105      	movs	r1, #5
10000780:	f7ff ffde 	bl	10000740 <gpio_set_function>
10000784:	bd10      	pop	{r4, pc}
	...

10000788 <running_on_fpga>:
10000788:	4b03      	ldr	r3, [pc, #12]	; (10000798 <running_on_fpga+0x10>)
1000078a:	681b      	ldr	r3, [r3, #0]
1000078c:	2002      	movs	r0, #2
1000078e:	4018      	ands	r0, r3
10000790:	1e43      	subs	r3, r0, #1
10000792:	4198      	sbcs	r0, r3
10000794:	b2c0      	uxtb	r0, r0
10000796:	4770      	bx	lr
10000798:	4006c000 	.word	0x4006c000

1000079c <hw_claim_lock>:
1000079c:	f3ef 8010 	mrs	r0, PRIMASK
100007a0:	b672      	cpsid	i
100007a2:	4b03      	ldr	r3, [pc, #12]	; (100007b0 <hw_claim_lock+0x14>)
100007a4:	681b      	ldr	r3, [r3, #0]
100007a6:	2b00      	cmp	r3, #0
100007a8:	d0fb      	beq.n	100007a2 <hw_claim_lock+0x6>
100007aa:	f3bf 8f5f 	dmb	sy
100007ae:	4770      	bx	lr
100007b0:	d000012c 	.word	0xd000012c

100007b4 <hw_claim_unlock>:
100007b4:	f3bf 8f5f 	dmb	sy
100007b8:	4b02      	ldr	r3, [pc, #8]	; (100007c4 <hw_claim_unlock+0x10>)
100007ba:	2200      	movs	r2, #0
100007bc:	601a      	str	r2, [r3, #0]
100007be:	f380 8810 	msr	PRIMASK, r0
100007c2:	4770      	bx	lr
100007c4:	d000012c 	.word	0xd000012c

100007c8 <hw_claim_or_assert>:
100007c8:	b5f8      	push	{r3, r4, r5, r6, r7, lr}
100007ca:	0006      	movs	r6, r0
100007cc:	000c      	movs	r4, r1
100007ce:	0015      	movs	r5, r2
100007d0:	f7ff ffe4 	bl	1000079c <hw_claim_lock>
100007d4:	08e3      	lsrs	r3, r4, #3
100007d6:	18f7      	adds	r7, r6, r3
100007d8:	5cf1      	ldrb	r1, [r6, r3]
100007da:	2207      	movs	r2, #7
100007dc:	4022      	ands	r2, r4
100007de:	2301      	movs	r3, #1
100007e0:	4093      	lsls	r3, r2
100007e2:	420b      	tst	r3, r1
100007e4:	d105      	bne.n	100007f2 <hw_claim_or_assert+0x2a>
100007e6:	b2db      	uxtb	r3, r3
100007e8:	430b      	orrs	r3, r1
100007ea:	703b      	strb	r3, [r7, #0]
100007ec:	f7ff ffe2 	bl	100007b4 <hw_claim_unlock>
100007f0:	bdf8      	pop	{r3, r4, r5, r6, r7, pc}
100007f2:	0021      	movs	r1, r4
100007f4:	0028      	movs	r0, r5
100007f6:	f001 feb5 	bl	10002564 <panic>
	...

100007fc <spin_locks_reset>:
100007fc:	2300      	movs	r3, #0
100007fe:	e007      	b.n	10000810 <spin_locks_reset+0x14>
10000800:	4a05      	ldr	r2, [pc, #20]	; (10000818 <spin_locks_reset+0x1c>)
10000802:	189a      	adds	r2, r3, r2
10000804:	0092      	lsls	r2, r2, #2
10000806:	f3bf 8f5f 	dmb	sy
1000080a:	2100      	movs	r1, #0
1000080c:	6011      	str	r1, [r2, #0]
1000080e:	3301      	adds	r3, #1
10000810:	2b1f      	cmp	r3, #31
10000812:	d9f5      	bls.n	10000800 <spin_locks_reset+0x4>
10000814:	4770      	bx	lr
10000816:	46c0      	nop			; (mov r8, r8)
10000818:	34000040 	.word	0x34000040

1000081c <next_striped_spin_lock_num>:
1000081c:	4a05      	ldr	r2, [pc, #20]	; (10000834 <next_striped_spin_lock_num+0x18>)
1000081e:	7810      	ldrb	r0, [r2, #0]
10000820:	1c43      	adds	r3, r0, #1
10000822:	b2db      	uxtb	r3, r3
10000824:	7013      	strb	r3, [r2, #0]
10000826:	2b17      	cmp	r3, #23
10000828:	d902      	bls.n	10000830 <next_striped_spin_lock_num+0x14>
1000082a:	0013      	movs	r3, r2
1000082c:	2210      	movs	r2, #16
1000082e:	701a      	strb	r2, [r3, #0]
10000830:	4770      	bx	lr
10000832:	46c0      	nop			; (mov r8, r8)
10000834:	2000023c 	.word	0x2000023c

10000838 <set_raw_irq_handler_and_unlock>:
10000838:	4b07      	ldr	r3, [pc, #28]	; (10000858 <set_raw_irq_handler_and_unlock+0x20>)
1000083a:	689b      	ldr	r3, [r3, #8]
1000083c:	3010      	adds	r0, #16
1000083e:	0080      	lsls	r0, r0, #2
10000840:	5019      	str	r1, [r3, r0]
10000842:	f3bf 8f5f 	dmb	sy
10000846:	f3bf 8f5f 	dmb	sy
1000084a:	4b04      	ldr	r3, [pc, #16]	; (1000085c <set_raw_irq_handler_and_unlock+0x24>)
1000084c:	2100      	movs	r1, #0
1000084e:	6019      	str	r1, [r3, #0]
10000850:	f382 8810 	msr	PRIMASK, r2
10000854:	4770      	bx	lr
10000856:	46c0      	nop			; (mov r8, r8)
10000858:	e000ed00 	.word	0xe000ed00
1000085c:	d0000124 	.word	0xd0000124

10000860 <make_branch>:
10000860:	b510      	push	{r4, lr}
10000862:	1a09      	subs	r1, r1, r0
10000864:	1f08      	subs	r0, r1, #4
10000866:	4b0a      	ldr	r3, [pc, #40]	; (10000890 <make_branch+0x30>)
10000868:	469c      	mov	ip, r3
1000086a:	4461      	add	r1, ip
1000086c:	4a09      	ldr	r2, [pc, #36]	; (10000894 <make_branch+0x34>)
1000086e:	4291      	cmp	r1, r2
10000870:	d808      	bhi.n	10000884 <make_branch+0x24>
10000872:	07c3      	lsls	r3, r0, #31
10000874:	d406      	bmi.n	10000884 <make_branch+0x24>
10000876:	1040      	asrs	r0, r0, #1
10000878:	0540      	lsls	r0, r0, #21
1000087a:	0d40      	lsrs	r0, r0, #21
1000087c:	4b06      	ldr	r3, [pc, #24]	; (10000898 <make_branch+0x38>)
1000087e:	4318      	orrs	r0, r3
10000880:	b280      	uxth	r0, r0
10000882:	bd10      	pop	{r4, pc}
10000884:	4b05      	ldr	r3, [pc, #20]	; (1000089c <make_branch+0x3c>)
10000886:	4a06      	ldr	r2, [pc, #24]	; (100008a0 <make_branch+0x40>)
10000888:	21a3      	movs	r1, #163	; 0xa3
1000088a:	4806      	ldr	r0, [pc, #24]	; (100008a4 <make_branch+0x44>)
1000088c:	f001 fdd0 	bl	10002430 <__assert_func>
10000890:	000007fc 	.word	0x000007fc
10000894:	00000ffe 	.word	0x00000ffe
10000898:	ffffe000 	.word	0xffffe000
1000089c:	10004f1c 	.word	0x10004f1c
100008a0:	10005174 	.word	0x10005174
100008a4:	10004f4c 	.word	0x10004f4c

100008a8 <insert_branch_and_link>:
100008a8:	b510      	push	{r4, lr}
100008aa:	1a09      	subs	r1, r1, r0
100008ac:	3904      	subs	r1, #4
100008ae:	084c      	lsrs	r4, r1, #1
100008b0:	0b09      	lsrs	r1, r1, #12
100008b2:	d108      	bne.n	100008c6 <insert_branch_and_link+0x1e>
100008b4:	0549      	lsls	r1, r1, #21
100008b6:	0d49      	lsrs	r1, r1, #21
100008b8:	4a06      	ldr	r2, [pc, #24]	; (100008d4 <insert_branch_and_link+0x2c>)
100008ba:	4311      	orrs	r1, r2
100008bc:	8001      	strh	r1, [r0, #0]
100008be:	4b06      	ldr	r3, [pc, #24]	; (100008d8 <insert_branch_and_link+0x30>)
100008c0:	4323      	orrs	r3, r4
100008c2:	8043      	strh	r3, [r0, #2]
100008c4:	bd10      	pop	{r4, pc}
100008c6:	4b05      	ldr	r3, [pc, #20]	; (100008dc <insert_branch_and_link+0x34>)
100008c8:	4a05      	ldr	r2, [pc, #20]	; (100008e0 <insert_branch_and_link+0x38>)
100008ca:	21ab      	movs	r1, #171	; 0xab
100008cc:	4805      	ldr	r0, [pc, #20]	; (100008e4 <insert_branch_and_link+0x3c>)
100008ce:	f001 fdaf 	bl	10002430 <__assert_func>
100008d2:	46c0      	nop			; (mov r8, r8)
100008d4:	fffff000 	.word	0xfffff000
100008d8:	fffff800 	.word	0xfffff800
100008dc:	10004f90 	.word	0x10004f90
100008e0:	10005148 	.word	0x10005148
100008e4:	10004f4c 	.word	0x10004f4c

100008e8 <irq_is_enabled>:
100008e8:	2301      	movs	r3, #1
100008ea:	4083      	lsls	r3, r0
100008ec:	4a03      	ldr	r2, [pc, #12]	; (100008fc <irq_is_enabled+0x14>)
100008ee:	6810      	ldr	r0, [r2, #0]
100008f0:	4018      	ands	r0, r3
100008f2:	1e43      	subs	r3, r0, #1
100008f4:	4198      	sbcs	r0, r3
100008f6:	b2c0      	uxtb	r0, r0
100008f8:	4770      	bx	lr
100008fa:	46c0      	nop			; (mov r8, r8)
100008fc:	e000e100 	.word	0xe000e100

10000900 <irq_set_mask_enabled>:
10000900:	2900      	cmp	r1, #0
10000902:	d004      	beq.n	1000090e <irq_set_mask_enabled+0xe>
10000904:	4b03      	ldr	r3, [pc, #12]	; (10000914 <irq_set_mask_enabled+0x14>)
10000906:	6018      	str	r0, [r3, #0]
10000908:	4b03      	ldr	r3, [pc, #12]	; (10000918 <irq_set_mask_enabled+0x18>)
1000090a:	6018      	str	r0, [r3, #0]
1000090c:	4770      	bx	lr
1000090e:	4b03      	ldr	r3, [pc, #12]	; (1000091c <irq_set_mask_enabled+0x1c>)
10000910:	6018      	str	r0, [r3, #0]
10000912:	e7fb      	b.n	1000090c <irq_set_mask_enabled+0xc>
10000914:	e000e280 	.word	0xe000e280
10000918:	e000e100 	.word	0xe000e100
1000091c:	e000e180 	.word	0xe000e180

10000920 <irq_set_enabled>:
10000920:	b510      	push	{r4, lr}
10000922:	2301      	movs	r3, #1
10000924:	4083      	lsls	r3, r0
10000926:	0018      	movs	r0, r3
10000928:	f7ff ffea 	bl	10000900 <irq_set_mask_enabled>
1000092c:	bd10      	pop	{r4, pc}
	...

10000930 <irq_get_vtable_handler>:
10000930:	4b02      	ldr	r3, [pc, #8]	; (1000093c <irq_get_vtable_handler+0xc>)
10000932:	689b      	ldr	r3, [r3, #8]
10000934:	3010      	adds	r0, #16
10000936:	0080      	lsls	r0, r0, #2
10000938:	58c0      	ldr	r0, [r0, r3]
1000093a:	4770      	bx	lr
1000093c:	e000ed00 	.word	0xe000ed00

10000940 <irq_set_exclusive_handler>:
10000940:	b570      	push	{r4, r5, r6, lr}
10000942:	0004      	movs	r4, r0
10000944:	000d      	movs	r5, r1
10000946:	f3ef 8610 	mrs	r6, PRIMASK
1000094a:	b672      	cpsid	i
1000094c:	4b0c      	ldr	r3, [pc, #48]	; (10000980 <irq_set_exclusive_handler+0x40>)
1000094e:	681b      	ldr	r3, [r3, #0]
10000950:	2b00      	cmp	r3, #0
10000952:	d0fb      	beq.n	1000094c <irq_set_exclusive_handler+0xc>
10000954:	f3bf 8f5f 	dmb	sy
10000958:	0020      	movs	r0, r4
1000095a:	f7ff ffe9 	bl	10000930 <irq_get_vtable_handler>
1000095e:	4b09      	ldr	r3, [pc, #36]	; (10000984 <irq_set_exclusive_handler+0x44>)
10000960:	4298      	cmp	r0, r3
10000962:	d001      	beq.n	10000968 <irq_set_exclusive_handler+0x28>
10000964:	42a8      	cmp	r0, r5
10000966:	d105      	bne.n	10000974 <irq_set_exclusive_handler+0x34>
10000968:	0032      	movs	r2, r6
1000096a:	0029      	movs	r1, r5
1000096c:	0020      	movs	r0, r4
1000096e:	f7ff ff63 	bl	10000838 <set_raw_irq_handler_and_unlock>
10000972:	bd70      	pop	{r4, r5, r6, pc}
10000974:	4b04      	ldr	r3, [pc, #16]	; (10000988 <irq_set_exclusive_handler+0x48>)
10000976:	4a05      	ldr	r2, [pc, #20]	; (1000098c <irq_set_exclusive_handler+0x4c>)
10000978:	2186      	movs	r1, #134	; 0x86
1000097a:	4805      	ldr	r0, [pc, #20]	; (10000990 <irq_set_exclusive_handler+0x50>)
1000097c:	f001 fd58 	bl	10002430 <__assert_func>
10000980:	d0000124 	.word	0xd0000124
10000984:	100001cd 	.word	0x100001cd
10000988:	10004fa0 	.word	0x10004fa0
1000098c:	10005190 	.word	0x10005190
10000990:	10004f4c 	.word	0x10004f4c

10000994 <irq_remove_handler>:
10000994:	b5f0      	push	{r4, r5, r6, r7, lr}
10000996:	46ce      	mov	lr, r9
10000998:	4647      	mov	r7, r8
1000099a:	b580      	push	{r7, lr}
1000099c:	b083      	sub	sp, #12
1000099e:	0006      	movs	r6, r0
100009a0:	000d      	movs	r5, r1
100009a2:	f3ef 8810 	mrs	r8, PRIMASK
100009a6:	b672      	cpsid	i
100009a8:	4b56      	ldr	r3, [pc, #344]	; (10000b04 <irq_remove_handler+0x170>)
100009aa:	681b      	ldr	r3, [r3, #0]
100009ac:	2b00      	cmp	r3, #0
100009ae:	d0fb      	beq.n	100009a8 <irq_remove_handler+0x14>
100009b0:	f3bf 8f5f 	dmb	sy
100009b4:	4b54      	ldr	r3, [pc, #336]	; (10000b08 <irq_remove_handler+0x174>)
100009b6:	689a      	ldr	r2, [r3, #8]
100009b8:	0034      	movs	r4, r6
100009ba:	3410      	adds	r4, #16
100009bc:	00a3      	lsls	r3, r4, #2
100009be:	58d7      	ldr	r7, [r2, r3]
100009c0:	4b52      	ldr	r3, [pc, #328]	; (10000b0c <irq_remove_handler+0x178>)
100009c2:	429f      	cmp	r7, r3
100009c4:	d007      	beq.n	100009d6 <irq_remove_handler+0x42>
100009c6:	42af      	cmp	r7, r5
100009c8:	d100      	bne.n	100009cc <irq_remove_handler+0x38>
100009ca:	e098      	b.n	10000afe <irq_remove_handler+0x16a>
100009cc:	9701      	str	r7, [sp, #4]
100009ce:	4b50      	ldr	r3, [pc, #320]	; (10000b10 <irq_remove_handler+0x17c>)
100009d0:	1afb      	subs	r3, r7, r3
100009d2:	2b2f      	cmp	r3, #47	; 0x2f
100009d4:	d909      	bls.n	100009ea <irq_remove_handler+0x56>
100009d6:	4642      	mov	r2, r8
100009d8:	0039      	movs	r1, r7
100009da:	0030      	movs	r0, r6
100009dc:	f7ff ff2c 	bl	10000838 <set_raw_irq_handler_and_unlock>
100009e0:	b003      	add	sp, #12
100009e2:	bcc0      	pop	{r6, r7}
100009e4:	46b9      	mov	r9, r7
100009e6:	46b0      	mov	r8, r6
100009e8:	bdf0      	pop	{r4, r5, r6, r7, pc}
100009ea:	0030      	movs	r0, r6
100009ec:	f7ff ff7c 	bl	100008e8 <irq_is_enabled>
100009f0:	4681      	mov	r9, r0
100009f2:	2100      	movs	r1, #0
100009f4:	0030      	movs	r0, r6
100009f6:	f7ff ff93 	bl	10000920 <irq_set_enabled>
100009fa:	f3bf 8f5f 	dmb	sy
100009fe:	f3ef 8105 	mrs	r1, IPSR
10000a02:	2900      	cmp	r1, #0
10000a04:	d001      	beq.n	10000a0a <irq_remove_handler+0x76>
10000a06:	428c      	cmp	r4, r1
10000a08:	d111      	bne.n	10000a2e <irq_remove_handler+0x9a>
10000a0a:	2301      	movs	r3, #1
10000a0c:	9c01      	ldr	r4, [sp, #4]
10000a0e:	439c      	bics	r4, r3
10000a10:	2200      	movs	r2, #0
10000a12:	68a3      	ldr	r3, [r4, #8]
10000a14:	42ab      	cmp	r3, r5
10000a16:	d012      	beq.n	10000a3e <irq_remove_handler+0xaa>
10000a18:	2206      	movs	r2, #6
10000a1a:	56a2      	ldrsb	r2, [r4, r2]
10000a1c:	2a00      	cmp	r2, #0
10000a1e:	db0d      	blt.n	10000a3c <irq_remove_handler+0xa8>
10000a20:	0053      	lsls	r3, r2, #1
10000a22:	189b      	adds	r3, r3, r2
10000a24:	009b      	lsls	r3, r3, #2
10000a26:	0022      	movs	r2, r4
10000a28:	4c39      	ldr	r4, [pc, #228]	; (10000b10 <irq_remove_handler+0x17c>)
10000a2a:	18e4      	adds	r4, r4, r3
10000a2c:	e7f1      	b.n	10000a12 <irq_remove_handler+0x7e>
10000a2e:	2136      	movs	r1, #54	; 0x36
10000a30:	4b38      	ldr	r3, [pc, #224]	; (10000b14 <irq_remove_handler+0x180>)
10000a32:	4a39      	ldr	r2, [pc, #228]	; (10000b18 <irq_remove_handler+0x184>)
10000a34:	31ff      	adds	r1, #255	; 0xff
10000a36:	4839      	ldr	r0, [pc, #228]	; (10000b1c <irq_remove_handler+0x188>)
10000a38:	f001 fcfa 	bl	10002430 <__assert_func>
10000a3c:	0022      	movs	r2, r4
10000a3e:	42ab      	cmp	r3, r5
10000a40:	d156      	bne.n	10000af0 <irq_remove_handler+0x15c>
10000a42:	2506      	movs	r5, #6
10000a44:	5765      	ldrsb	r5, [r4, r5]
10000a46:	2d00      	cmp	r5, #0
10000a48:	db38      	blt.n	10000abc <irq_remove_handler+0x128>
10000a4a:	006b      	lsls	r3, r5, #1
10000a4c:	195b      	adds	r3, r3, r5
10000a4e:	009a      	lsls	r2, r3, #2
10000a50:	4b2f      	ldr	r3, [pc, #188]	; (10000b10 <irq_remove_handler+0x17c>)
10000a52:	189b      	adds	r3, r3, r2
10000a54:	689a      	ldr	r2, [r3, #8]
10000a56:	60a2      	str	r2, [r4, #8]
10000a58:	79da      	ldrb	r2, [r3, #7]
10000a5a:	71e2      	strb	r2, [r4, #7]
10000a5c:	2206      	movs	r2, #6
10000a5e:	569a      	ldrsb	r2, [r3, r2]
10000a60:	71a2      	strb	r2, [r4, #6]
10000a62:	799b      	ldrb	r3, [r3, #6]
10000a64:	b25b      	sxtb	r3, r3
10000a66:	2b00      	cmp	r3, #0
10000a68:	da0f      	bge.n	10000a8a <irq_remove_handler+0xf6>
10000a6a:	482d      	ldr	r0, [pc, #180]	; (10000b20 <irq_remove_handler+0x18c>)
10000a6c:	80a0      	strh	r0, [r4, #4]
10000a6e:	006b      	lsls	r3, r5, #1
10000a70:	195b      	adds	r3, r3, r5
10000a72:	009b      	lsls	r3, r3, #2
10000a74:	4a26      	ldr	r2, [pc, #152]	; (10000b10 <irq_remove_handler+0x17c>)
10000a76:	18d3      	adds	r3, r2, r3
10000a78:	4a2a      	ldr	r2, [pc, #168]	; (10000b24 <irq_remove_handler+0x190>)
10000a7a:	7811      	ldrb	r1, [r2, #0]
10000a7c:	7199      	strb	r1, [r3, #6]
10000a7e:	7015      	strb	r5, [r2, #0]
10000a80:	4649      	mov	r1, r9
10000a82:	0030      	movs	r0, r6
10000a84:	f7ff ff4c 	bl	10000920 <irq_set_enabled>
10000a88:	e7a5      	b.n	100009d6 <irq_remove_handler+0x42>
10000a8a:	1d20      	adds	r0, r4, #4
10000a8c:	006b      	lsls	r3, r5, #1
10000a8e:	195b      	adds	r3, r3, r5
10000a90:	009b      	lsls	r3, r3, #2
10000a92:	4a1f      	ldr	r2, [pc, #124]	; (10000b10 <irq_remove_handler+0x17c>)
10000a94:	189b      	adds	r3, r3, r2
10000a96:	1d1a      	adds	r2, r3, #4
10000a98:	889b      	ldrh	r3, [r3, #4]
10000a9a:	0ad9      	lsrs	r1, r3, #11
10000a9c:	291c      	cmp	r1, #28
10000a9e:	d107      	bne.n	10000ab0 <irq_remove_handler+0x11c>
10000aa0:	055b      	lsls	r3, r3, #21
10000aa2:	155b      	asrs	r3, r3, #21
10000aa4:	3302      	adds	r3, #2
10000aa6:	0059      	lsls	r1, r3, #1
10000aa8:	1851      	adds	r1, r2, r1
10000aaa:	f7ff fed9 	bl	10000860 <make_branch>
10000aae:	e7dd      	b.n	10000a6c <irq_remove_handler+0xd8>
10000ab0:	4b1d      	ldr	r3, [pc, #116]	; (10000b28 <irq_remove_handler+0x194>)
10000ab2:	4a1e      	ldr	r2, [pc, #120]	; (10000b2c <irq_remove_handler+0x198>)
10000ab4:	21b1      	movs	r1, #177	; 0xb1
10000ab6:	4819      	ldr	r0, [pc, #100]	; (10000b1c <irq_remove_handler+0x188>)
10000ab8:	f001 fcba 	bl	10002430 <__assert_func>
10000abc:	2900      	cmp	r1, #0
10000abe:	d112      	bne.n	10000ae6 <irq_remove_handler+0x152>
10000ac0:	2a00      	cmp	r2, #0
10000ac2:	d00e      	beq.n	10000ae2 <irq_remove_handler+0x14e>
10000ac4:	23ff      	movs	r3, #255	; 0xff
10000ac6:	7193      	strb	r3, [r2, #6]
10000ac8:	4b19      	ldr	r3, [pc, #100]	; (10000b30 <irq_remove_handler+0x19c>)
10000aca:	8093      	strh	r3, [r2, #4]
10000acc:	4a15      	ldr	r2, [pc, #84]	; (10000b24 <irq_remove_handler+0x190>)
10000ace:	7813      	ldrb	r3, [r2, #0]
10000ad0:	71a3      	strb	r3, [r4, #6]
10000ad2:	4b18      	ldr	r3, [pc, #96]	; (10000b34 <irq_remove_handler+0x1a0>)
10000ad4:	490e      	ldr	r1, [pc, #56]	; (10000b10 <irq_remove_handler+0x17c>)
10000ad6:	1a64      	subs	r4, r4, r1
10000ad8:	4164      	adcs	r4, r4
10000ada:	4363      	muls	r3, r4
10000adc:	0d1b      	lsrs	r3, r3, #20
10000ade:	7013      	strb	r3, [r2, #0]
10000ae0:	e7ce      	b.n	10000a80 <irq_remove_handler+0xec>
10000ae2:	4f0a      	ldr	r7, [pc, #40]	; (10000b0c <irq_remove_handler+0x178>)
10000ae4:	e7f2      	b.n	10000acc <irq_remove_handler+0x138>
10000ae6:	1d20      	adds	r0, r4, #4
10000ae8:	4913      	ldr	r1, [pc, #76]	; (10000b38 <irq_remove_handler+0x1a4>)
10000aea:	f7ff fedd 	bl	100008a8 <insert_branch_and_link>
10000aee:	e7c7      	b.n	10000a80 <irq_remove_handler+0xec>
10000af0:	216a      	movs	r1, #106	; 0x6a
10000af2:	4b12      	ldr	r3, [pc, #72]	; (10000b3c <irq_remove_handler+0x1a8>)
10000af4:	4a08      	ldr	r2, [pc, #32]	; (10000b18 <irq_remove_handler+0x184>)
10000af6:	31ff      	adds	r1, #255	; 0xff
10000af8:	4808      	ldr	r0, [pc, #32]	; (10000b1c <irq_remove_handler+0x188>)
10000afa:	f001 fc99 	bl	10002430 <__assert_func>
10000afe:	4f03      	ldr	r7, [pc, #12]	; (10000b0c <irq_remove_handler+0x178>)
10000b00:	e769      	b.n	100009d6 <irq_remove_handler+0x42>
10000b02:	46c0      	nop			; (mov r8, r8)
10000b04:	d0000124 	.word	0xd0000124
10000b08:	e000ed00 	.word	0xe000ed00
10000b0c:	100001cd 	.word	0x100001cd
10000b10:	20000240 	.word	0x20000240
10000b14:	100050b4 	.word	0x100050b4
10000b18:	10005160 	.word	0x10005160
10000b1c:	10004f4c 	.word	0x10004f4c
10000b20:	0000bd01 	.word	0x0000bd01
10000b24:	20025ee5 	.word	0x20025ee5
10000b28:	1000509c 	.word	0x1000509c
10000b2c:	10005180 	.word	0x10005180
10000b30:	ffffbd01 	.word	0xffffbd01
10000b34:	0000aaaa 	.word	0x0000aaaa
10000b38:	2000027a 	.word	0x2000027a
10000b3c:	100050e8 	.word	0x100050e8

10000b40 <irq_add_tail_to_free_list>:
10000b40:	b570      	push	{r4, r5, r6, lr}
10000b42:	2101      	movs	r1, #1
10000b44:	4301      	orrs	r1, r0
10000b46:	4b2e      	ldr	r3, [pc, #184]	; (10000c00 <irq_add_tail_to_free_list+0xc0>)
10000b48:	1acb      	subs	r3, r1, r3
10000b4a:	2b2f      	cmp	r3, #47	; 0x2f
10000b4c:	d828      	bhi.n	10000ba0 <irq_add_tail_to_free_list+0x60>
10000b4e:	f3ef 8305 	mrs	r3, IPSR
10000b52:	2b00      	cmp	r3, #0
10000b54:	d02b      	beq.n	10000bae <irq_add_tail_to_free_list+0x6e>
10000b56:	f3ef 8c10 	mrs	ip, PRIMASK
10000b5a:	b672      	cpsid	i
10000b5c:	4a29      	ldr	r2, [pc, #164]	; (10000c04 <irq_add_tail_to_free_list+0xc4>)
10000b5e:	6812      	ldr	r2, [r2, #0]
10000b60:	2a00      	cmp	r2, #0
10000b62:	d0fb      	beq.n	10000b5c <irq_add_tail_to_free_list+0x1c>
10000b64:	f3bf 8f5f 	dmb	sy
10000b68:	4a27      	ldr	r2, [pc, #156]	; (10000c08 <irq_add_tail_to_free_list+0xc8>)
10000b6a:	0004      	movs	r4, r0
10000b6c:	4d24      	ldr	r5, [pc, #144]	; (10000c00 <irq_add_tail_to_free_list+0xc0>)
10000b6e:	1b64      	subs	r4, r4, r5
10000b70:	4164      	adcs	r4, r4
10000b72:	4362      	muls	r2, r4
10000b74:	0d12      	lsrs	r2, r2, #20
10000b76:	b254      	sxtb	r4, r2
10000b78:	4a24      	ldr	r2, [pc, #144]	; (10000c0c <irq_add_tail_to_free_list+0xcc>)
10000b7a:	6892      	ldr	r2, [r2, #8]
10000b7c:	009b      	lsls	r3, r3, #2
10000b7e:	58d2      	ldr	r2, [r2, r3]
10000b80:	428a      	cmp	r2, r1
10000b82:	d01b      	beq.n	10000bbc <irq_add_tail_to_free_list+0x7c>
10000b84:	2200      	movs	r2, #0
10000b86:	2a03      	cmp	r2, #3
10000b88:	d832      	bhi.n	10000bf0 <irq_add_tail_to_free_list+0xb0>
10000b8a:	0053      	lsls	r3, r2, #1
10000b8c:	189b      	adds	r3, r3, r2
10000b8e:	009b      	lsls	r3, r3, #2
10000b90:	491b      	ldr	r1, [pc, #108]	; (10000c00 <irq_add_tail_to_free_list+0xc0>)
10000b92:	18cb      	adds	r3, r1, r3
10000b94:	799b      	ldrb	r3, [r3, #6]
10000b96:	b25b      	sxtb	r3, r3
10000b98:	42a3      	cmp	r3, r4
10000b9a:	d01f      	beq.n	10000bdc <irq_add_tail_to_free_list+0x9c>
10000b9c:	3201      	adds	r2, #1
10000b9e:	e7f2      	b.n	10000b86 <irq_add_tail_to_free_list+0x46>
10000ba0:	21c7      	movs	r1, #199	; 0xc7
10000ba2:	4b1b      	ldr	r3, [pc, #108]	; (10000c10 <irq_add_tail_to_free_list+0xd0>)
10000ba4:	4a1b      	ldr	r2, [pc, #108]	; (10000c14 <irq_add_tail_to_free_list+0xd4>)
10000ba6:	0049      	lsls	r1, r1, #1
10000ba8:	481b      	ldr	r0, [pc, #108]	; (10000c18 <irq_add_tail_to_free_list+0xd8>)
10000baa:	f001 fc41 	bl	10002430 <__assert_func>
10000bae:	2192      	movs	r1, #146	; 0x92
10000bb0:	4b1a      	ldr	r3, [pc, #104]	; (10000c1c <irq_add_tail_to_free_list+0xdc>)
10000bb2:	4a18      	ldr	r2, [pc, #96]	; (10000c14 <irq_add_tail_to_free_list+0xd4>)
10000bb4:	31ff      	adds	r1, #255	; 0xff
10000bb6:	4818      	ldr	r0, [pc, #96]	; (10000c18 <irq_add_tail_to_free_list+0xd8>)
10000bb8:	f001 fc3a 	bl	10002430 <__assert_func>
10000bbc:	4a13      	ldr	r2, [pc, #76]	; (10000c0c <irq_add_tail_to_free_list+0xcc>)
10000bbe:	6892      	ldr	r2, [r2, #8]
10000bc0:	4917      	ldr	r1, [pc, #92]	; (10000c20 <irq_add_tail_to_free_list+0xe0>)
10000bc2:	50d1      	str	r1, [r2, r3]
10000bc4:	4b17      	ldr	r3, [pc, #92]	; (10000c24 <irq_add_tail_to_free_list+0xe4>)
10000bc6:	781a      	ldrb	r2, [r3, #0]
10000bc8:	7182      	strb	r2, [r0, #6]
10000bca:	701c      	strb	r4, [r3, #0]
10000bcc:	f3bf 8f5f 	dmb	sy
10000bd0:	4b0c      	ldr	r3, [pc, #48]	; (10000c04 <irq_add_tail_to_free_list+0xc4>)
10000bd2:	2200      	movs	r2, #0
10000bd4:	601a      	str	r2, [r3, #0]
10000bd6:	f38c 8810 	msr	PRIMASK, ip
10000bda:	bd70      	pop	{r4, r5, r6, pc}
10000bdc:	000d      	movs	r5, r1
10000bde:	0053      	lsls	r3, r2, #1
10000be0:	1899      	adds	r1, r3, r2
10000be2:	0089      	lsls	r1, r1, #2
10000be4:	1869      	adds	r1, r5, r1
10000be6:	26ff      	movs	r6, #255	; 0xff
10000be8:	718e      	strb	r6, [r1, #6]
10000bea:	4a0f      	ldr	r2, [pc, #60]	; (10000c28 <irq_add_tail_to_free_list+0xe8>)
10000bec:	808a      	strh	r2, [r1, #4]
10000bee:	e7e9      	b.n	10000bc4 <irq_add_tail_to_free_list+0x84>
10000bf0:	21d1      	movs	r1, #209	; 0xd1
10000bf2:	4b0e      	ldr	r3, [pc, #56]	; (10000c2c <irq_add_tail_to_free_list+0xec>)
10000bf4:	4a07      	ldr	r2, [pc, #28]	; (10000c14 <irq_add_tail_to_free_list+0xd4>)
10000bf6:	0049      	lsls	r1, r1, #1
10000bf8:	4807      	ldr	r0, [pc, #28]	; (10000c18 <irq_add_tail_to_free_list+0xd8>)
10000bfa:	f001 fc19 	bl	10002430 <__assert_func>
10000bfe:	46c0      	nop			; (mov r8, r8)
10000c00:	20000240 	.word	0x20000240
10000c04:	d0000124 	.word	0xd0000124
10000c08:	0000aaaa 	.word	0x0000aaaa
10000c0c:	e000ed00 	.word	0xe000ed00
10000c10:	100050f0 	.word	0x100050f0
10000c14:	1000512c 	.word	0x1000512c
10000c18:	10004f4c 	.word	0x10004f4c
10000c1c:	10005118 	.word	0x10005118
10000c20:	100001cd 	.word	0x100001cd
10000c24:	20025ee5 	.word	0x20025ee5
10000c28:	ffffbd01 	.word	0xffffbd01
10000c2c:	10005124 	.word	0x10005124

10000c30 <irq_init_priorities>:
10000c30:	2200      	movs	r2, #0
10000c32:	4b04      	ldr	r3, [pc, #16]	; (10000c44 <irq_init_priorities+0x14>)
10000c34:	e002      	b.n	10000c3c <irq_init_priorities+0xc>
10000c36:	4904      	ldr	r1, [pc, #16]	; (10000c48 <irq_init_priorities+0x18>)
10000c38:	c302      	stmia	r3!, {r1}
10000c3a:	3201      	adds	r2, #1
10000c3c:	2a07      	cmp	r2, #7
10000c3e:	d9fa      	bls.n	10000c36 <irq_init_priorities+0x6>
10000c40:	4770      	bx	lr
10000c42:	46c0      	nop			; (mov r8, r8)
10000c44:	e000e400 	.word	0xe000e400
10000c48:	80808080 	.word	0x80808080

10000c4c <lock_init>:
10000c4c:	4b02      	ldr	r3, [pc, #8]	; (10000c58 <lock_init+0xc>)
10000c4e:	469c      	mov	ip, r3
10000c50:	4461      	add	r1, ip
10000c52:	0089      	lsls	r1, r1, #2
10000c54:	6001      	str	r1, [r0, #0]
10000c56:	4770      	bx	lr
10000c58:	34000040 	.word	0x34000040

10000c5c <mutex_init>:
10000c5c:	b510      	push	{r4, lr}
10000c5e:	0004      	movs	r4, r0
10000c60:	f7ff fddc 	bl	1000081c <next_striped_spin_lock_num>
10000c64:	0001      	movs	r1, r0
10000c66:	0020      	movs	r0, r4
10000c68:	f7ff fff0 	bl	10000c4c <lock_init>
10000c6c:	23ff      	movs	r3, #255	; 0xff
10000c6e:	7123      	strb	r3, [r4, #4]
10000c70:	f3bf 8f5f 	dmb	sy
10000c74:	bd10      	pop	{r4, pc}

10000c76 <recursive_mutex_init>:
10000c76:	b510      	push	{r4, lr}
10000c78:	0004      	movs	r4, r0
10000c7a:	f7ff fdcf 	bl	1000081c <next_striped_spin_lock_num>
10000c7e:	0001      	movs	r1, r0
10000c80:	0020      	movs	r0, r4
10000c82:	f7ff ffe3 	bl	10000c4c <lock_init>
10000c86:	23ff      	movs	r3, #255	; 0xff
10000c88:	7123      	strb	r3, [r4, #4]
10000c8a:	2300      	movs	r3, #0
10000c8c:	7163      	strb	r3, [r4, #5]
10000c8e:	f3bf 8f5f 	dmb	sy
10000c92:	bd10      	pop	{r4, pc}

10000c94 <alarm_pool_post_alloc_init>:
10000c94:	b570      	push	{r4, r5, r6, lr}
10000c96:	0005      	movs	r5, r0
10000c98:	000c      	movs	r4, r1
10000c9a:	0008      	movs	r0, r1
10000c9c:	f000 fefe 	bl	10001a9c <hardware_alarm_cancel>
10000ca0:	4909      	ldr	r1, [pc, #36]	; (10000cc8 <alarm_pool_post_alloc_init+0x34>)
10000ca2:	0020      	movs	r0, r4
10000ca4:	f000 fe3e 	bl	10001924 <hardware_alarm_set_callback>
10000ca8:	f7ff fdb8 	bl	1000081c <next_striped_spin_lock_num>
10000cac:	4b07      	ldr	r3, [pc, #28]	; (10000ccc <alarm_pool_post_alloc_init+0x38>)
10000cae:	469c      	mov	ip, r3
10000cb0:	4460      	add	r0, ip
10000cb2:	0080      	lsls	r0, r0, #2
10000cb4:	6068      	str	r0, [r5, #4]
10000cb6:	752c      	strb	r4, [r5, #20]
10000cb8:	23d0      	movs	r3, #208	; 0xd0
10000cba:	061b      	lsls	r3, r3, #24
10000cbc:	781b      	ldrb	r3, [r3, #0]
10000cbe:	756b      	strb	r3, [r5, #21]
10000cc0:	00a4      	lsls	r4, r4, #2
10000cc2:	4b03      	ldr	r3, [pc, #12]	; (10000cd0 <alarm_pool_post_alloc_init+0x3c>)
10000cc4:	50e5      	str	r5, [r4, r3]
10000cc6:	bd70      	pop	{r4, r5, r6, pc}
10000cc8:	10000fd9 	.word	0x10000fd9
10000ccc:	34000040 	.word	0x34000040
10000cd0:	200004b4 	.word	0x200004b4

10000cd4 <sleep_until_callback>:
10000cd4:	4b0a      	ldr	r3, [pc, #40]	; (10000d00 <sleep_until_callback+0x2c>)
10000cd6:	681a      	ldr	r2, [r3, #0]
10000cd8:	f3ef 8110 	mrs	r1, PRIMASK
10000cdc:	b672      	cpsid	i
10000cde:	6813      	ldr	r3, [r2, #0]
10000ce0:	2b00      	cmp	r3, #0
10000ce2:	d0fc      	beq.n	10000cde <sleep_until_callback+0xa>
10000ce4:	f3bf 8f5f 	dmb	sy
10000ce8:	4b05      	ldr	r3, [pc, #20]	; (10000d00 <sleep_until_callback+0x2c>)
10000cea:	681b      	ldr	r3, [r3, #0]
10000cec:	f3bf 8f5f 	dmb	sy
10000cf0:	2200      	movs	r2, #0
10000cf2:	601a      	str	r2, [r3, #0]
10000cf4:	f381 8810 	msr	PRIMASK, r1
10000cf8:	bf40      	sev
10000cfa:	2000      	movs	r0, #0
10000cfc:	2100      	movs	r1, #0
10000cfe:	4770      	bx	lr
10000d00:	200006c8 	.word	0x200006c8

10000d04 <timer_pool_entry_comparator>:
10000d04:	b510      	push	{r4, lr}
10000d06:	2900      	cmp	r1, #0
10000d08:	d022      	beq.n	10000d50 <timer_pool_entry_comparator+0x4c>
10000d0a:	6803      	ldr	r3, [r0, #0]
10000d0c:	7b1b      	ldrb	r3, [r3, #12]
10000d0e:	4299      	cmp	r1, r3
10000d10:	d81e      	bhi.n	10000d50 <timer_pool_entry_comparator+0x4c>
10000d12:	4b17      	ldr	r3, [pc, #92]	; (10000d70 <timer_pool_entry_comparator+0x6c>)
10000d14:	469c      	mov	ip, r3
10000d16:	4461      	add	r1, ip
10000d18:	0109      	lsls	r1, r1, #4
10000d1a:	6883      	ldr	r3, [r0, #8]
10000d1c:	469c      	mov	ip, r3
10000d1e:	4461      	add	r1, ip
10000d20:	680c      	ldr	r4, [r1, #0]
10000d22:	6849      	ldr	r1, [r1, #4]
10000d24:	2a00      	cmp	r2, #0
10000d26:	d019      	beq.n	10000d5c <timer_pool_entry_comparator+0x58>
10000d28:	6803      	ldr	r3, [r0, #0]
10000d2a:	7b1b      	ldrb	r3, [r3, #12]
10000d2c:	429a      	cmp	r2, r3
10000d2e:	d815      	bhi.n	10000d5c <timer_pool_entry_comparator+0x58>
10000d30:	6883      	ldr	r3, [r0, #8]
10000d32:	480f      	ldr	r0, [pc, #60]	; (10000d70 <timer_pool_entry_comparator+0x6c>)
10000d34:	4684      	mov	ip, r0
10000d36:	4462      	add	r2, ip
10000d38:	0112      	lsls	r2, r2, #4
10000d3a:	189a      	adds	r2, r3, r2
10000d3c:	6810      	ldr	r0, [r2, #0]
10000d3e:	6853      	ldr	r3, [r2, #4]
10000d40:	0002      	movs	r2, r0
10000d42:	2001      	movs	r0, #1
10000d44:	428b      	cmp	r3, r1
10000d46:	d801      	bhi.n	10000d4c <timer_pool_entry_comparator+0x48>
10000d48:	d00e      	beq.n	10000d68 <timer_pool_entry_comparator+0x64>
10000d4a:	2000      	movs	r0, #0
10000d4c:	b2c0      	uxtb	r0, r0
10000d4e:	bd10      	pop	{r4, pc}
10000d50:	4b08      	ldr	r3, [pc, #32]	; (10000d74 <timer_pool_entry_comparator+0x70>)
10000d52:	4a09      	ldr	r2, [pc, #36]	; (10000d78 <timer_pool_entry_comparator+0x74>)
10000d54:	213c      	movs	r1, #60	; 0x3c
10000d56:	4809      	ldr	r0, [pc, #36]	; (10000d7c <timer_pool_entry_comparator+0x78>)
10000d58:	f001 fb6a 	bl	10002430 <__assert_func>
10000d5c:	4b05      	ldr	r3, [pc, #20]	; (10000d74 <timer_pool_entry_comparator+0x70>)
10000d5e:	4a06      	ldr	r2, [pc, #24]	; (10000d78 <timer_pool_entry_comparator+0x74>)
10000d60:	213c      	movs	r1, #60	; 0x3c
10000d62:	4806      	ldr	r0, [pc, #24]	; (10000d7c <timer_pool_entry_comparator+0x78>)
10000d64:	f001 fb64 	bl	10002430 <__assert_func>
10000d68:	42a2      	cmp	r2, r4
10000d6a:	d8ef      	bhi.n	10000d4c <timer_pool_entry_comparator+0x48>
10000d6c:	e7ed      	b.n	10000d4a <timer_pool_entry_comparator+0x46>
10000d6e:	46c0      	nop			; (mov r8, r8)
10000d70:	0fffffff 	.word	0x0fffffff
10000d74:	10005318 	.word	0x10005318
10000d78:	10005580 	.word	0x10005580
10000d7c:	100052dc 	.word	0x100052dc

10000d80 <ph_add_child_node>:
10000d80:	b510      	push	{r4, lr}
10000d82:	2900      	cmp	r1, #0
10000d84:	d01e      	beq.n	10000dc4 <ph_add_child_node+0x44>
10000d86:	7b03      	ldrb	r3, [r0, #12]
10000d88:	4299      	cmp	r1, r3
10000d8a:	d81b      	bhi.n	10000dc4 <ph_add_child_node+0x44>
10000d8c:	004b      	lsls	r3, r1, #1
10000d8e:	185b      	adds	r3, r3, r1
10000d90:	3b03      	subs	r3, #3
10000d92:	6804      	ldr	r4, [r0, #0]
10000d94:	46a4      	mov	ip, r4
10000d96:	4463      	add	r3, ip
10000d98:	2900      	cmp	r1, #0
10000d9a:	d019      	beq.n	10000dd0 <ph_add_child_node+0x50>
10000d9c:	2a00      	cmp	r2, #0
10000d9e:	d01d      	beq.n	10000ddc <ph_add_child_node+0x5c>
10000da0:	4291      	cmp	r1, r2
10000da2:	d021      	beq.n	10000de8 <ph_add_child_node+0x68>
10000da4:	2a00      	cmp	r2, #0
10000da6:	d025      	beq.n	10000df4 <ph_add_child_node+0x74>
10000da8:	7b04      	ldrb	r4, [r0, #12]
10000daa:	42a2      	cmp	r2, r4
10000dac:	d822      	bhi.n	10000df4 <ph_add_child_node+0x74>
10000dae:	6804      	ldr	r4, [r0, #0]
10000db0:	0050      	lsls	r0, r2, #1
10000db2:	1880      	adds	r0, r0, r2
10000db4:	3803      	subs	r0, #3
10000db6:	1820      	adds	r0, r4, r0
10000db8:	7081      	strb	r1, [r0, #2]
10000dba:	7819      	ldrb	r1, [r3, #0]
10000dbc:	2900      	cmp	r1, #0
10000dbe:	d11f      	bne.n	10000e00 <ph_add_child_node+0x80>
10000dc0:	701a      	strb	r2, [r3, #0]
10000dc2:	bd10      	pop	{r4, pc}
10000dc4:	4b10      	ldr	r3, [pc, #64]	; (10000e08 <ph_add_child_node+0x88>)
10000dc6:	4a11      	ldr	r2, [pc, #68]	; (10000e0c <ph_add_child_node+0x8c>)
10000dc8:	2168      	movs	r1, #104	; 0x68
10000dca:	4811      	ldr	r0, [pc, #68]	; (10000e10 <ph_add_child_node+0x90>)
10000dcc:	f001 fb30 	bl	10002430 <__assert_func>
10000dd0:	4b10      	ldr	r3, [pc, #64]	; (10000e14 <ph_add_child_node+0x94>)
10000dd2:	4a11      	ldr	r2, [pc, #68]	; (10000e18 <ph_add_child_node+0x98>)
10000dd4:	316f      	adds	r1, #111	; 0x6f
10000dd6:	480e      	ldr	r0, [pc, #56]	; (10000e10 <ph_add_child_node+0x90>)
10000dd8:	f001 fb2a 	bl	10002430 <__assert_func>
10000ddc:	4b0f      	ldr	r3, [pc, #60]	; (10000e1c <ph_add_child_node+0x9c>)
10000dde:	4a0e      	ldr	r2, [pc, #56]	; (10000e18 <ph_add_child_node+0x98>)
10000de0:	2170      	movs	r1, #112	; 0x70
10000de2:	480b      	ldr	r0, [pc, #44]	; (10000e10 <ph_add_child_node+0x90>)
10000de4:	f001 fb24 	bl	10002430 <__assert_func>
10000de8:	4b0d      	ldr	r3, [pc, #52]	; (10000e20 <ph_add_child_node+0xa0>)
10000dea:	4a0b      	ldr	r2, [pc, #44]	; (10000e18 <ph_add_child_node+0x98>)
10000dec:	2171      	movs	r1, #113	; 0x71
10000dee:	4808      	ldr	r0, [pc, #32]	; (10000e10 <ph_add_child_node+0x90>)
10000df0:	f001 fb1e 	bl	10002430 <__assert_func>
10000df4:	4b04      	ldr	r3, [pc, #16]	; (10000e08 <ph_add_child_node+0x88>)
10000df6:	4a05      	ldr	r2, [pc, #20]	; (10000e0c <ph_add_child_node+0x8c>)
10000df8:	2168      	movs	r1, #104	; 0x68
10000dfa:	4805      	ldr	r0, [pc, #20]	; (10000e10 <ph_add_child_node+0x90>)
10000dfc:	f001 fb18 	bl	10002430 <__assert_func>
10000e00:	7041      	strb	r1, [r0, #1]
10000e02:	701a      	strb	r2, [r3, #0]
10000e04:	e7dd      	b.n	10000dc2 <ph_add_child_node+0x42>
10000e06:	46c0      	nop			; (mov r8, r8)
10000e08:	1000533c 	.word	0x1000533c
10000e0c:	100055ec 	.word	0x100055ec
10000e10:	10005358 	.word	0x10005358
10000e14:	100053a8 	.word	0x100053a8
10000e18:	100055c8 	.word	0x100055c8
10000e1c:	100053b4 	.word	0x100053b4
10000e20:	100053c0 	.word	0x100053c0

10000e24 <ph_merge_nodes>:
10000e24:	b570      	push	{r4, r5, r6, lr}
10000e26:	0006      	movs	r6, r0
10000e28:	000d      	movs	r5, r1
10000e2a:	0014      	movs	r4, r2
10000e2c:	2900      	cmp	r1, #0
10000e2e:	d014      	beq.n	10000e5a <ph_merge_nodes+0x36>
10000e30:	2a00      	cmp	r2, #0
10000e32:	d014      	beq.n	10000e5e <ph_merge_nodes+0x3a>
10000e34:	6880      	ldr	r0, [r0, #8]
10000e36:	6873      	ldr	r3, [r6, #4]
10000e38:	4798      	blx	r3
10000e3a:	2800      	cmp	r0, #0
10000e3c:	d006      	beq.n	10000e4c <ph_merge_nodes+0x28>
10000e3e:	0022      	movs	r2, r4
10000e40:	0029      	movs	r1, r5
10000e42:	0030      	movs	r0, r6
10000e44:	f7ff ff9c 	bl	10000d80 <ph_add_child_node>
10000e48:	0028      	movs	r0, r5
10000e4a:	e007      	b.n	10000e5c <ph_merge_nodes+0x38>
10000e4c:	002a      	movs	r2, r5
10000e4e:	0021      	movs	r1, r4
10000e50:	0030      	movs	r0, r6
10000e52:	f7ff ff95 	bl	10000d80 <ph_add_child_node>
10000e56:	0020      	movs	r0, r4
10000e58:	e000      	b.n	10000e5c <ph_merge_nodes+0x38>
10000e5a:	0010      	movs	r0, r2
10000e5c:	bd70      	pop	{r4, r5, r6, pc}
10000e5e:	0008      	movs	r0, r1
10000e60:	e7fc      	b.n	10000e5c <ph_merge_nodes+0x38>
	...

10000e64 <add_alarm_under_lock>:
10000e64:	b5f0      	push	{r4, r5, r6, r7, lr}
10000e66:	b083      	sub	sp, #12
10000e68:	0005      	movs	r5, r0
10000e6a:	9200      	str	r2, [sp, #0]
10000e6c:	9301      	str	r3, [sp, #4]
10000e6e:	ab0a      	add	r3, sp, #40	; 0x28
10000e70:	781c      	ldrb	r4, [r3, #0]
10000e72:	ab0b      	add	r3, sp, #44	; 0x2c
10000e74:	781f      	ldrb	r7, [r3, #0]
10000e76:	2c00      	cmp	r4, #0
10000e78:	d026      	beq.n	10000ec8 <add_alarm_under_lock+0x64>
10000e7a:	6803      	ldr	r3, [r0, #0]
10000e7c:	7b5a      	ldrb	r2, [r3, #13]
10000e7e:	4294      	cmp	r4, r2
10000e80:	d107      	bne.n	10000e92 <add_alarm_under_lock+0x2e>
10000e82:	2301      	movs	r3, #1
10000e84:	2b00      	cmp	r3, #0
10000e86:	d119      	bne.n	10000ebc <add_alarm_under_lock+0x58>
10000e88:	2c00      	cmp	r4, #0
10000e8a:	d13b      	bne.n	10000f04 <add_alarm_under_lock+0xa0>
10000e8c:	0020      	movs	r0, r4
10000e8e:	b003      	add	sp, #12
10000e90:	bdf0      	pop	{r4, r5, r6, r7, pc}
10000e92:	2c00      	cmp	r4, #0
10000e94:	d00c      	beq.n	10000eb0 <add_alarm_under_lock+0x4c>
10000e96:	7b1a      	ldrb	r2, [r3, #12]
10000e98:	4294      	cmp	r4, r2
10000e9a:	d809      	bhi.n	10000eb0 <add_alarm_under_lock+0x4c>
10000e9c:	681a      	ldr	r2, [r3, #0]
10000e9e:	0063      	lsls	r3, r4, #1
10000ea0:	191b      	adds	r3, r3, r4
10000ea2:	3b03      	subs	r3, #3
10000ea4:	18d3      	adds	r3, r2, r3
10000ea6:	789b      	ldrb	r3, [r3, #2]
10000ea8:	2b00      	cmp	r3, #0
10000eaa:	d0eb      	beq.n	10000e84 <add_alarm_under_lock+0x20>
10000eac:	2301      	movs	r3, #1
10000eae:	e7e9      	b.n	10000e84 <add_alarm_under_lock+0x20>
10000eb0:	4b3e      	ldr	r3, [pc, #248]	; (10000fac <add_alarm_under_lock+0x148>)
10000eb2:	4a3f      	ldr	r2, [pc, #252]	; (10000fb0 <add_alarm_under_lock+0x14c>)
10000eb4:	2168      	movs	r1, #104	; 0x68
10000eb6:	483f      	ldr	r0, [pc, #252]	; (10000fb4 <add_alarm_under_lock+0x150>)
10000eb8:	f001 faba 	bl	10002430 <__assert_func>
10000ebc:	4b3e      	ldr	r3, [pc, #248]	; (10000fb8 <add_alarm_under_lock+0x154>)
10000ebe:	4a3f      	ldr	r2, [pc, #252]	; (10000fbc <add_alarm_under_lock+0x158>)
10000ec0:	2167      	movs	r1, #103	; 0x67
10000ec2:	483f      	ldr	r0, [pc, #252]	; (10000fc0 <add_alarm_under_lock+0x15c>)
10000ec4:	f001 fab4 	bl	10002430 <__assert_func>
10000ec8:	6803      	ldr	r3, [r0, #0]
10000eca:	7b9c      	ldrb	r4, [r3, #14]
10000ecc:	2c00      	cmp	r4, #0
10000ece:	d0db      	beq.n	10000e88 <add_alarm_under_lock+0x24>
10000ed0:	d012      	beq.n	10000ef8 <add_alarm_under_lock+0x94>
10000ed2:	7b1a      	ldrb	r2, [r3, #12]
10000ed4:	4294      	cmp	r4, r2
10000ed6:	d80f      	bhi.n	10000ef8 <add_alarm_under_lock+0x94>
10000ed8:	0062      	lsls	r2, r4, #1
10000eda:	1912      	adds	r2, r2, r4
10000edc:	3a03      	subs	r2, #3
10000ede:	6819      	ldr	r1, [r3, #0]
10000ee0:	468c      	mov	ip, r1
10000ee2:	4462      	add	r2, ip
10000ee4:	7851      	ldrb	r1, [r2, #1]
10000ee6:	7399      	strb	r1, [r3, #14]
10000ee8:	2900      	cmp	r1, #0
10000eea:	d100      	bne.n	10000eee <add_alarm_under_lock+0x8a>
10000eec:	73d9      	strb	r1, [r3, #15]
10000eee:	2300      	movs	r3, #0
10000ef0:	7093      	strb	r3, [r2, #2]
10000ef2:	7053      	strb	r3, [r2, #1]
10000ef4:	7013      	strb	r3, [r2, #0]
10000ef6:	e7c7      	b.n	10000e88 <add_alarm_under_lock+0x24>
10000ef8:	4b2c      	ldr	r3, [pc, #176]	; (10000fac <add_alarm_under_lock+0x148>)
10000efa:	4a2d      	ldr	r2, [pc, #180]	; (10000fb0 <add_alarm_under_lock+0x14c>)
10000efc:	2168      	movs	r1, #104	; 0x68
10000efe:	482d      	ldr	r0, [pc, #180]	; (10000fb4 <add_alarm_under_lock+0x150>)
10000f00:	f001 fa96 	bl	10002430 <__assert_func>
10000f04:	2c00      	cmp	r4, #0
10000f06:	d03a      	beq.n	10000f7e <add_alarm_under_lock+0x11a>
10000f08:	682b      	ldr	r3, [r5, #0]
10000f0a:	7b1b      	ldrb	r3, [r3, #12]
10000f0c:	429c      	cmp	r4, r3
10000f0e:	d836      	bhi.n	10000f7e <add_alarm_under_lock+0x11a>
10000f10:	4b2c      	ldr	r3, [pc, #176]	; (10000fc4 <add_alarm_under_lock+0x160>)
10000f12:	18e3      	adds	r3, r4, r3
10000f14:	011b      	lsls	r3, r3, #4
10000f16:	68aa      	ldr	r2, [r5, #8]
10000f18:	4694      	mov	ip, r2
10000f1a:	4463      	add	r3, ip
10000f1c:	9a00      	ldr	r2, [sp, #0]
10000f1e:	601a      	str	r2, [r3, #0]
10000f20:	9a01      	ldr	r2, [sp, #4]
10000f22:	605a      	str	r2, [r3, #4]
10000f24:	9a08      	ldr	r2, [sp, #32]
10000f26:	609a      	str	r2, [r3, #8]
10000f28:	9a09      	ldr	r2, [sp, #36]	; 0x24
10000f2a:	60da      	str	r2, [r3, #12]
10000f2c:	682e      	ldr	r6, [r5, #0]
10000f2e:	2c00      	cmp	r4, #0
10000f30:	d02b      	beq.n	10000f8a <add_alarm_under_lock+0x126>
10000f32:	d030      	beq.n	10000f96 <add_alarm_under_lock+0x132>
10000f34:	7b33      	ldrb	r3, [r6, #12]
10000f36:	429c      	cmp	r4, r3
10000f38:	d82d      	bhi.n	10000f96 <add_alarm_under_lock+0x132>
10000f3a:	0063      	lsls	r3, r4, #1
10000f3c:	191b      	adds	r3, r3, r4
10000f3e:	3b03      	subs	r3, #3
10000f40:	6832      	ldr	r2, [r6, #0]
10000f42:	4694      	mov	ip, r2
10000f44:	4463      	add	r3, ip
10000f46:	2200      	movs	r2, #0
10000f48:	709a      	strb	r2, [r3, #2]
10000f4a:	705a      	strb	r2, [r3, #1]
10000f4c:	701a      	strb	r2, [r3, #0]
10000f4e:	7b71      	ldrb	r1, [r6, #13]
10000f50:	0022      	movs	r2, r4
10000f52:	0030      	movs	r0, r6
10000f54:	f7ff ff66 	bl	10000e24 <ph_merge_nodes>
10000f58:	7370      	strb	r0, [r6, #13]
10000f5a:	4284      	cmp	r4, r0
10000f5c:	d000      	beq.n	10000f60 <add_alarm_under_lock+0xfc>
10000f5e:	e795      	b.n	10000e8c <add_alarm_under_lock+0x28>
10000f60:	7d28      	ldrb	r0, [r5, #20]
10000f62:	9a00      	ldr	r2, [sp, #0]
10000f64:	9b01      	ldr	r3, [sp, #4]
10000f66:	f000 fd25 	bl	100019b4 <hardware_alarm_set_target>
10000f6a:	1e06      	subs	r6, r0, #0
10000f6c:	d001      	beq.n	10000f72 <add_alarm_under_lock+0x10e>
10000f6e:	2f00      	cmp	r7, #0
10000f70:	d017      	beq.n	10000fa2 <add_alarm_under_lock+0x13e>
10000f72:	9b0c      	ldr	r3, [sp, #48]	; 0x30
10000f74:	2b00      	cmp	r3, #0
10000f76:	d100      	bne.n	10000f7a <add_alarm_under_lock+0x116>
10000f78:	e788      	b.n	10000e8c <add_alarm_under_lock+0x28>
10000f7a:	701e      	strb	r6, [r3, #0]
10000f7c:	e786      	b.n	10000e8c <add_alarm_under_lock+0x28>
10000f7e:	4b12      	ldr	r3, [pc, #72]	; (10000fc8 <add_alarm_under_lock+0x164>)
10000f80:	4a12      	ldr	r2, [pc, #72]	; (10000fcc <add_alarm_under_lock+0x168>)
10000f82:	213c      	movs	r1, #60	; 0x3c
10000f84:	480e      	ldr	r0, [pc, #56]	; (10000fc0 <add_alarm_under_lock+0x15c>)
10000f86:	f001 fa53 	bl	10002430 <__assert_func>
10000f8a:	4b11      	ldr	r3, [pc, #68]	; (10000fd0 <add_alarm_under_lock+0x16c>)
10000f8c:	4a11      	ldr	r2, [pc, #68]	; (10000fd4 <add_alarm_under_lock+0x170>)
10000f8e:	21a5      	movs	r1, #165	; 0xa5
10000f90:	4808      	ldr	r0, [pc, #32]	; (10000fb4 <add_alarm_under_lock+0x150>)
10000f92:	f001 fa4d 	bl	10002430 <__assert_func>
10000f96:	4b05      	ldr	r3, [pc, #20]	; (10000fac <add_alarm_under_lock+0x148>)
10000f98:	4a05      	ldr	r2, [pc, #20]	; (10000fb0 <add_alarm_under_lock+0x14c>)
10000f9a:	2168      	movs	r1, #104	; 0x68
10000f9c:	4805      	ldr	r0, [pc, #20]	; (10000fb4 <add_alarm_under_lock+0x150>)
10000f9e:	f001 fa47 	bl	10002430 <__assert_func>
10000fa2:	6828      	ldr	r0, [r5, #0]
10000fa4:	0021      	movs	r1, r4
10000fa6:	f000 ff3d 	bl	10001e24 <ph_remove_and_free_node>
10000faa:	e7e2      	b.n	10000f72 <add_alarm_under_lock+0x10e>
10000fac:	1000533c 	.word	0x1000533c
10000fb0:	100055ec 	.word	0x100055ec
10000fb4:	10005358 	.word	0x10005358
10000fb8:	100053d8 	.word	0x100053d8
10000fbc:	100055f8 	.word	0x100055f8
10000fc0:	100052dc 	.word	0x100052dc
10000fc4:	0fffffff 	.word	0x0fffffff
10000fc8:	10005318 	.word	0x10005318
10000fcc:	10005580 	.word	0x10005580
10000fd0:	100052d8 	.word	0x100052d8
10000fd4:	100055dc 	.word	0x100055dc

10000fd8 <alarm_pool_alarm_callback>:
10000fd8:	b5f0      	push	{r4, r5, r6, r7, lr}
10000fda:	46de      	mov	lr, fp
10000fdc:	4657      	mov	r7, sl
10000fde:	464e      	mov	r6, r9
10000fe0:	4645      	mov	r5, r8
10000fe2:	b5e0      	push	{r5, r6, r7, lr}
10000fe4:	b08b      	sub	sp, #44	; 0x2c
10000fe6:	9009      	str	r0, [sp, #36]	; 0x24
10000fe8:	2300      	movs	r3, #0
10000fea:	9308      	str	r3, [sp, #32]
10000fec:	0082      	lsls	r2, r0, #2
10000fee:	4bb5      	ldr	r3, [pc, #724]	; (100012c4 <alarm_pool_alarm_callback+0x2ec>)
10000ff0:	58d6      	ldr	r6, [r2, r3]
10000ff2:	0037      	movs	r7, r6
10000ff4:	e052      	b.n	1000109c <alarm_pool_alarm_callback+0xc4>
10000ff6:	4bb4      	ldr	r3, [pc, #720]	; (100012c8 <alarm_pool_alarm_callback+0x2f0>)
10000ff8:	4ab4      	ldr	r2, [pc, #720]	; (100012cc <alarm_pool_alarm_callback+0x2f4>)
10000ffa:	213f      	movs	r1, #63	; 0x3f
10000ffc:	48b4      	ldr	r0, [pc, #720]	; (100012d0 <alarm_pool_alarm_callback+0x2f8>)
10000ffe:	f001 fa17 	bl	10002430 <__assert_func>
10001002:	4bb4      	ldr	r3, [pc, #720]	; (100012d4 <alarm_pool_alarm_callback+0x2fc>)
10001004:	4ab4      	ldr	r2, [pc, #720]	; (100012d8 <alarm_pool_alarm_callback+0x300>)
10001006:	213c      	movs	r1, #60	; 0x3c
10001008:	48b4      	ldr	r0, [pc, #720]	; (100012dc <alarm_pool_alarm_callback+0x304>)
1000100a:	f001 fa11 	bl	10002430 <__assert_func>
1000100e:	2900      	cmp	r1, #0
10001010:	d101      	bne.n	10001016 <alarm_pool_alarm_callback+0x3e>
10001012:	2800      	cmp	r0, #0
10001014:	d169      	bne.n	100010ea <alarm_pool_alarm_callback+0x112>
10001016:	2100      	movs	r1, #0
10001018:	4640      	mov	r0, r8
1000101a:	f000 fef9 	bl	10001e10 <ph_remove_head>
1000101e:	42a0      	cmp	r0, r4
10001020:	d119      	bne.n	10001056 <alarm_pool_alarm_callback+0x7e>
10001022:	682a      	ldr	r2, [r5, #0]
10001024:	686b      	ldr	r3, [r5, #4]
10001026:	9206      	str	r2, [sp, #24]
10001028:	9307      	str	r3, [sp, #28]
1000102a:	68ab      	ldr	r3, [r5, #8]
1000102c:	4698      	mov	r8, r3
1000102e:	68eb      	ldr	r3, [r5, #12]
10001030:	469a      	mov	sl, r3
10001032:	4643      	mov	r3, r8
10001034:	2b00      	cmp	r3, #0
10001036:	d014      	beq.n	10001062 <alarm_pool_alarm_callback+0x8a>
10001038:	2c00      	cmp	r4, #0
1000103a:	d018      	beq.n	1000106e <alarm_pool_alarm_callback+0x96>
1000103c:	683b      	ldr	r3, [r7, #0]
1000103e:	7b1b      	ldrb	r3, [r3, #12]
10001040:	429c      	cmp	r4, r3
10001042:	d814      	bhi.n	1000106e <alarm_pool_alarm_callback+0x96>
10001044:	1e63      	subs	r3, r4, #1
10001046:	68fa      	ldr	r2, [r7, #12]
10001048:	5cd3      	ldrb	r3, [r2, r3]
1000104a:	9308      	str	r3, [sp, #32]
1000104c:	021b      	lsls	r3, r3, #8
1000104e:	4318      	orrs	r0, r3
10001050:	6138      	str	r0, [r7, #16]
10001052:	2000      	movs	r0, #0
10001054:	e015      	b.n	10001082 <alarm_pool_alarm_callback+0xaa>
10001056:	4ba2      	ldr	r3, [pc, #648]	; (100012e0 <alarm_pool_alarm_callback+0x308>)
10001058:	4aa2      	ldr	r2, [pc, #648]	; (100012e4 <alarm_pool_alarm_callback+0x30c>)
1000105a:	218e      	movs	r1, #142	; 0x8e
1000105c:	489f      	ldr	r0, [pc, #636]	; (100012dc <alarm_pool_alarm_callback+0x304>)
1000105e:	f001 f9e7 	bl	10002430 <__assert_func>
10001062:	4ba1      	ldr	r3, [pc, #644]	; (100012e8 <alarm_pool_alarm_callback+0x310>)
10001064:	4a9f      	ldr	r2, [pc, #636]	; (100012e4 <alarm_pool_alarm_callback+0x30c>)
10001066:	2192      	movs	r1, #146	; 0x92
10001068:	489c      	ldr	r0, [pc, #624]	; (100012dc <alarm_pool_alarm_callback+0x304>)
1000106a:	f001 f9e1 	bl	10002430 <__assert_func>
1000106e:	4b99      	ldr	r3, [pc, #612]	; (100012d4 <alarm_pool_alarm_callback+0x2fc>)
10001070:	4a9e      	ldr	r2, [pc, #632]	; (100012ec <alarm_pool_alarm_callback+0x314>)
10001072:	2141      	movs	r1, #65	; 0x41
10001074:	4899      	ldr	r0, [pc, #612]	; (100012dc <alarm_pool_alarm_callback+0x304>)
10001076:	f001 f9db 	bl	10002430 <__assert_func>
1000107a:	2300      	movs	r3, #0
1000107c:	469a      	mov	sl, r3
1000107e:	4698      	mov	r8, r3
10001080:	2000      	movs	r0, #0
10001082:	687b      	ldr	r3, [r7, #4]
10001084:	f3bf 8f5f 	dmb	sy
10001088:	2200      	movs	r2, #0
1000108a:	601a      	str	r2, [r3, #0]
1000108c:	f386 8810 	msr	PRIMASK, r6
10001090:	4643      	mov	r3, r8
10001092:	2b00      	cmp	r3, #0
10001094:	d132      	bne.n	100010fc <alarm_pool_alarm_callback+0x124>
10001096:	2800      	cmp	r0, #0
10001098:	d100      	bne.n	1000109c <alarm_pool_alarm_callback+0xc4>
1000109a:	e10c      	b.n	100012b6 <alarm_pool_alarm_callback+0x2de>
1000109c:	f000 fbfe 	bl	1000189c <time_us_64>
100010a0:	0002      	movs	r2, r0
100010a2:	1e0b      	subs	r3, r1, #0
100010a4:	dba7      	blt.n	10000ff6 <alarm_pool_alarm_callback+0x1e>
100010a6:	2000      	movs	r0, #0
100010a8:	2100      	movs	r1, #0
100010aa:	9006      	str	r0, [sp, #24]
100010ac:	9107      	str	r1, [sp, #28]
100010ae:	6878      	ldr	r0, [r7, #4]
100010b0:	f3ef 8610 	mrs	r6, PRIMASK
100010b4:	b672      	cpsid	i
100010b6:	6801      	ldr	r1, [r0, #0]
100010b8:	2900      	cmp	r1, #0
100010ba:	d0fc      	beq.n	100010b6 <alarm_pool_alarm_callback+0xde>
100010bc:	f3bf 8f5f 	dmb	sy
100010c0:	6839      	ldr	r1, [r7, #0]
100010c2:	4688      	mov	r8, r1
100010c4:	7b4c      	ldrb	r4, [r1, #13]
100010c6:	2c00      	cmp	r4, #0
100010c8:	d0d7      	beq.n	1000107a <alarm_pool_alarm_callback+0xa2>
100010ca:	d09a      	beq.n	10001002 <alarm_pool_alarm_callback+0x2a>
100010cc:	7b09      	ldrb	r1, [r1, #12]
100010ce:	428c      	cmp	r4, r1
100010d0:	d897      	bhi.n	10001002 <alarm_pool_alarm_callback+0x2a>
100010d2:	4987      	ldr	r1, [pc, #540]	; (100012f0 <alarm_pool_alarm_callback+0x318>)
100010d4:	1865      	adds	r5, r4, r1
100010d6:	012d      	lsls	r5, r5, #4
100010d8:	68b9      	ldr	r1, [r7, #8]
100010da:	468c      	mov	ip, r1
100010dc:	4465      	add	r5, ip
100010de:	6828      	ldr	r0, [r5, #0]
100010e0:	6869      	ldr	r1, [r5, #4]
100010e2:	1a80      	subs	r0, r0, r2
100010e4:	4199      	sbcs	r1, r3
100010e6:	2900      	cmp	r1, #0
100010e8:	dd91      	ble.n	1000100e <alarm_pool_alarm_callback+0x36>
100010ea:	682a      	ldr	r2, [r5, #0]
100010ec:	686b      	ldr	r3, [r5, #4]
100010ee:	9809      	ldr	r0, [sp, #36]	; 0x24
100010f0:	f000 fc60 	bl	100019b4 <hardware_alarm_set_target>
100010f4:	2300      	movs	r3, #0
100010f6:	469a      	mov	sl, r3
100010f8:	4698      	mov	r8, r3
100010fa:	e7c2      	b.n	10001082 <alarm_pool_alarm_callback+0xaa>
100010fc:	9b08      	ldr	r3, [sp, #32]
100010fe:	021b      	lsls	r3, r3, #8
10001100:	4323      	orrs	r3, r4
10001102:	4699      	mov	r9, r3
10001104:	4651      	mov	r1, sl
10001106:	0018      	movs	r0, r3
10001108:	47c0      	blx	r8
1000110a:	0005      	movs	r5, r0
1000110c:	000e      	movs	r6, r1
1000110e:	687a      	ldr	r2, [r7, #4]
10001110:	f3ef 8b10 	mrs	fp, PRIMASK
10001114:	b672      	cpsid	i
10001116:	6813      	ldr	r3, [r2, #0]
10001118:	4259      	negs	r1, r3
1000111a:	414b      	adcs	r3, r1
1000111c:	b2d9      	uxtb	r1, r3
1000111e:	2b00      	cmp	r3, #0
10001120:	d1f9      	bne.n	10001116 <alarm_pool_alarm_callback+0x13e>
10001122:	f3bf 8f5f 	dmb	sy
10001126:	2e00      	cmp	r6, #0
10001128:	db1e      	blt.n	10001168 <alarm_pool_alarm_callback+0x190>
1000112a:	2e00      	cmp	r6, #0
1000112c:	dd46      	ble.n	100011bc <alarm_pool_alarm_callback+0x1e4>
1000112e:	693b      	ldr	r3, [r7, #16]
10001130:	2b00      	cmp	r3, #0
10001132:	d047      	beq.n	100011c4 <alarm_pool_alarm_callback+0x1ec>
10001134:	454b      	cmp	r3, r9
10001136:	d16d      	bne.n	10001214 <alarm_pool_alarm_callback+0x23c>
10001138:	f000 fbb0 	bl	1000189c <time_us_64>
1000113c:	0002      	movs	r2, r0
1000113e:	1e0b      	subs	r3, r1, #0
10001140:	db6e      	blt.n	10001220 <alarm_pool_alarm_callback+0x248>
10001142:	1952      	adds	r2, r2, r5
10001144:	4173      	adcs	r3, r6
10001146:	2b00      	cmp	r3, #0
10001148:	db70      	blt.n	1000122c <alarm_pool_alarm_callback+0x254>
1000114a:	2b00      	cmp	r3, #0
1000114c:	db72      	blt.n	10001234 <alarm_pool_alarm_callback+0x25c>
1000114e:	2100      	movs	r1, #0
10001150:	9104      	str	r1, [sp, #16]
10001152:	3101      	adds	r1, #1
10001154:	9103      	str	r1, [sp, #12]
10001156:	9402      	str	r4, [sp, #8]
10001158:	4651      	mov	r1, sl
1000115a:	9101      	str	r1, [sp, #4]
1000115c:	4641      	mov	r1, r8
1000115e:	9100      	str	r1, [sp, #0]
10001160:	0038      	movs	r0, r7
10001162:	f7ff fe7f 	bl	10000e64 <add_alarm_under_lock>
10001166:	e04c      	b.n	10001202 <alarm_pool_alarm_callback+0x22a>
10001168:	693b      	ldr	r3, [r7, #16]
1000116a:	2b00      	cmp	r3, #0
1000116c:	d0dd      	beq.n	1000112a <alarm_pool_alarm_callback+0x152>
1000116e:	454b      	cmp	r3, r9
10001170:	d114      	bne.n	1000119c <alarm_pool_alarm_callback+0x1c4>
10001172:	9a06      	ldr	r2, [sp, #24]
10001174:	9b07      	ldr	r3, [sp, #28]
10001176:	1b52      	subs	r2, r2, r5
10001178:	41b3      	sbcs	r3, r6
1000117a:	2b00      	cmp	r3, #0
1000117c:	db14      	blt.n	100011a8 <alarm_pool_alarm_callback+0x1d0>
1000117e:	2b00      	cmp	r3, #0
10001180:	db16      	blt.n	100011b0 <alarm_pool_alarm_callback+0x1d8>
10001182:	2100      	movs	r1, #0
10001184:	9104      	str	r1, [sp, #16]
10001186:	3101      	adds	r1, #1
10001188:	9103      	str	r1, [sp, #12]
1000118a:	9402      	str	r4, [sp, #8]
1000118c:	4651      	mov	r1, sl
1000118e:	9101      	str	r1, [sp, #4]
10001190:	4641      	mov	r1, r8
10001192:	9100      	str	r1, [sp, #0]
10001194:	0038      	movs	r0, r7
10001196:	f7ff fe65 	bl	10000e64 <add_alarm_under_lock>
1000119a:	e032      	b.n	10001202 <alarm_pool_alarm_callback+0x22a>
1000119c:	4b55      	ldr	r3, [pc, #340]	; (100012f4 <alarm_pool_alarm_callback+0x31c>)
1000119e:	4a51      	ldr	r2, [pc, #324]	; (100012e4 <alarm_pool_alarm_callback+0x30c>)
100011a0:	21a1      	movs	r1, #161	; 0xa1
100011a2:	484e      	ldr	r0, [pc, #312]	; (100012dc <alarm_pool_alarm_callback+0x304>)
100011a4:	f001 f944 	bl	10002430 <__assert_func>
100011a8:	2201      	movs	r2, #1
100011aa:	4252      	negs	r2, r2
100011ac:	4b52      	ldr	r3, [pc, #328]	; (100012f8 <alarm_pool_alarm_callback+0x320>)
100011ae:	e7e6      	b.n	1000117e <alarm_pool_alarm_callback+0x1a6>
100011b0:	4b45      	ldr	r3, [pc, #276]	; (100012c8 <alarm_pool_alarm_callback+0x2f0>)
100011b2:	4a46      	ldr	r2, [pc, #280]	; (100012cc <alarm_pool_alarm_callback+0x2f4>)
100011b4:	213f      	movs	r1, #63	; 0x3f
100011b6:	4846      	ldr	r0, [pc, #280]	; (100012d0 <alarm_pool_alarm_callback+0x2f8>)
100011b8:	f001 f93a 	bl	10002430 <__assert_func>
100011bc:	2e00      	cmp	r6, #0
100011be:	d101      	bne.n	100011c4 <alarm_pool_alarm_callback+0x1ec>
100011c0:	2d00      	cmp	r5, #0
100011c2:	d1b4      	bne.n	1000112e <alarm_pool_alarm_callback+0x156>
100011c4:	683b      	ldr	r3, [r7, #0]
100011c6:	2c00      	cmp	r4, #0
100011c8:	d050      	beq.n	1000126c <alarm_pool_alarm_callback+0x294>
100011ca:	7b5a      	ldrb	r2, [r3, #13]
100011cc:	4294      	cmp	r4, r2
100011ce:	d137      	bne.n	10001240 <alarm_pool_alarm_callback+0x268>
100011d0:	2101      	movs	r1, #1
100011d2:	2900      	cmp	r1, #0
100011d4:	d14a      	bne.n	1000126c <alarm_pool_alarm_callback+0x294>
100011d6:	7bda      	ldrb	r2, [r3, #15]
100011d8:	2a00      	cmp	r2, #0
100011da:	d14d      	bne.n	10001278 <alarm_pool_alarm_callback+0x2a0>
100011dc:	7b9a      	ldrb	r2, [r3, #14]
100011de:	2a00      	cmp	r2, #0
100011e0:	d103      	bne.n	100011ea <alarm_pool_alarm_callback+0x212>
100011e2:	7bda      	ldrb	r2, [r3, #15]
100011e4:	2a00      	cmp	r2, #0
100011e6:	d15a      	bne.n	1000129e <alarm_pool_alarm_callback+0x2c6>
100011e8:	739c      	strb	r4, [r3, #14]
100011ea:	73dc      	strb	r4, [r3, #15]
100011ec:	2c00      	cmp	r4, #0
100011ee:	d05c      	beq.n	100012aa <alarm_pool_alarm_callback+0x2d2>
100011f0:	683b      	ldr	r3, [r7, #0]
100011f2:	7b1b      	ldrb	r3, [r3, #12]
100011f4:	429c      	cmp	r4, r3
100011f6:	d858      	bhi.n	100012aa <alarm_pool_alarm_callback+0x2d2>
100011f8:	68fa      	ldr	r2, [r7, #12]
100011fa:	3c01      	subs	r4, #1
100011fc:	5d13      	ldrb	r3, [r2, r4]
100011fe:	3301      	adds	r3, #1
10001200:	5513      	strb	r3, [r2, r4]
10001202:	2300      	movs	r3, #0
10001204:	613b      	str	r3, [r7, #16]
10001206:	687a      	ldr	r2, [r7, #4]
10001208:	f3bf 8f5f 	dmb	sy
1000120c:	6013      	str	r3, [r2, #0]
1000120e:	f38b 8810 	msr	PRIMASK, fp
10001212:	e743      	b.n	1000109c <alarm_pool_alarm_callback+0xc4>
10001214:	4b37      	ldr	r3, [pc, #220]	; (100012f4 <alarm_pool_alarm_callback+0x31c>)
10001216:	4a33      	ldr	r2, [pc, #204]	; (100012e4 <alarm_pool_alarm_callback+0x30c>)
10001218:	21a4      	movs	r1, #164	; 0xa4
1000121a:	4830      	ldr	r0, [pc, #192]	; (100012dc <alarm_pool_alarm_callback+0x304>)
1000121c:	f001 f908 	bl	10002430 <__assert_func>
10001220:	4b29      	ldr	r3, [pc, #164]	; (100012c8 <alarm_pool_alarm_callback+0x2f0>)
10001222:	4a2a      	ldr	r2, [pc, #168]	; (100012cc <alarm_pool_alarm_callback+0x2f4>)
10001224:	213f      	movs	r1, #63	; 0x3f
10001226:	482a      	ldr	r0, [pc, #168]	; (100012d0 <alarm_pool_alarm_callback+0x2f8>)
10001228:	f001 f902 	bl	10002430 <__assert_func>
1000122c:	2201      	movs	r2, #1
1000122e:	4252      	negs	r2, r2
10001230:	4b31      	ldr	r3, [pc, #196]	; (100012f8 <alarm_pool_alarm_callback+0x320>)
10001232:	e78a      	b.n	1000114a <alarm_pool_alarm_callback+0x172>
10001234:	4b24      	ldr	r3, [pc, #144]	; (100012c8 <alarm_pool_alarm_callback+0x2f0>)
10001236:	4a25      	ldr	r2, [pc, #148]	; (100012cc <alarm_pool_alarm_callback+0x2f4>)
10001238:	213f      	movs	r1, #63	; 0x3f
1000123a:	4825      	ldr	r0, [pc, #148]	; (100012d0 <alarm_pool_alarm_callback+0x2f8>)
1000123c:	f001 f8f8 	bl	10002430 <__assert_func>
10001240:	2c00      	cmp	r4, #0
10001242:	d00d      	beq.n	10001260 <alarm_pool_alarm_callback+0x288>
10001244:	7b1a      	ldrb	r2, [r3, #12]
10001246:	4294      	cmp	r4, r2
10001248:	d80a      	bhi.n	10001260 <alarm_pool_alarm_callback+0x288>
1000124a:	0062      	lsls	r2, r4, #1
1000124c:	1912      	adds	r2, r2, r4
1000124e:	3a03      	subs	r2, #3
10001250:	6818      	ldr	r0, [r3, #0]
10001252:	4684      	mov	ip, r0
10001254:	4462      	add	r2, ip
10001256:	7892      	ldrb	r2, [r2, #2]
10001258:	2a00      	cmp	r2, #0
1000125a:	d0ba      	beq.n	100011d2 <alarm_pool_alarm_callback+0x1fa>
1000125c:	2101      	movs	r1, #1
1000125e:	e7b8      	b.n	100011d2 <alarm_pool_alarm_callback+0x1fa>
10001260:	4b26      	ldr	r3, [pc, #152]	; (100012fc <alarm_pool_alarm_callback+0x324>)
10001262:	4a27      	ldr	r2, [pc, #156]	; (10001300 <alarm_pool_alarm_callback+0x328>)
10001264:	2168      	movs	r1, #104	; 0x68
10001266:	4827      	ldr	r0, [pc, #156]	; (10001304 <alarm_pool_alarm_callback+0x32c>)
10001268:	f001 f8e2 	bl	10002430 <__assert_func>
1000126c:	4b26      	ldr	r3, [pc, #152]	; (10001308 <alarm_pool_alarm_callback+0x330>)
1000126e:	4a27      	ldr	r2, [pc, #156]	; (1000130c <alarm_pool_alarm_callback+0x334>)
10001270:	21f6      	movs	r1, #246	; 0xf6
10001272:	4824      	ldr	r0, [pc, #144]	; (10001304 <alarm_pool_alarm_callback+0x32c>)
10001274:	f001 f8dc 	bl	10002430 <__assert_func>
10001278:	2a00      	cmp	r2, #0
1000127a:	d00a      	beq.n	10001292 <alarm_pool_alarm_callback+0x2ba>
1000127c:	7b19      	ldrb	r1, [r3, #12]
1000127e:	428a      	cmp	r2, r1
10001280:	d807      	bhi.n	10001292 <alarm_pool_alarm_callback+0x2ba>
10001282:	0051      	lsls	r1, r2, #1
10001284:	188a      	adds	r2, r1, r2
10001286:	3a03      	subs	r2, #3
10001288:	6819      	ldr	r1, [r3, #0]
1000128a:	468c      	mov	ip, r1
1000128c:	4462      	add	r2, ip
1000128e:	7054      	strb	r4, [r2, #1]
10001290:	e7a4      	b.n	100011dc <alarm_pool_alarm_callback+0x204>
10001292:	4b1a      	ldr	r3, [pc, #104]	; (100012fc <alarm_pool_alarm_callback+0x324>)
10001294:	4a1a      	ldr	r2, [pc, #104]	; (10001300 <alarm_pool_alarm_callback+0x328>)
10001296:	2168      	movs	r1, #104	; 0x68
10001298:	481a      	ldr	r0, [pc, #104]	; (10001304 <alarm_pool_alarm_callback+0x32c>)
1000129a:	f001 f8c9 	bl	10002430 <__assert_func>
1000129e:	4b1c      	ldr	r3, [pc, #112]	; (10001310 <alarm_pool_alarm_callback+0x338>)
100012a0:	4a1a      	ldr	r2, [pc, #104]	; (1000130c <alarm_pool_alarm_callback+0x334>)
100012a2:	21fb      	movs	r1, #251	; 0xfb
100012a4:	4817      	ldr	r0, [pc, #92]	; (10001304 <alarm_pool_alarm_callback+0x32c>)
100012a6:	f001 f8c3 	bl	10002430 <__assert_func>
100012aa:	4b0a      	ldr	r3, [pc, #40]	; (100012d4 <alarm_pool_alarm_callback+0x2fc>)
100012ac:	4a0f      	ldr	r2, [pc, #60]	; (100012ec <alarm_pool_alarm_callback+0x314>)
100012ae:	2141      	movs	r1, #65	; 0x41
100012b0:	480a      	ldr	r0, [pc, #40]	; (100012dc <alarm_pool_alarm_callback+0x304>)
100012b2:	f001 f8bd 	bl	10002430 <__assert_func>
100012b6:	b00b      	add	sp, #44	; 0x2c
100012b8:	bcf0      	pop	{r4, r5, r6, r7}
100012ba:	46bb      	mov	fp, r7
100012bc:	46b2      	mov	sl, r6
100012be:	46a9      	mov	r9, r5
100012c0:	46a0      	mov	r8, r4
100012c2:	bdf0      	pop	{r4, r5, r6, r7, pc}
100012c4:	200004b4 	.word	0x200004b4
100012c8:	10005204 	.word	0x10005204
100012cc:	1000554c 	.word	0x1000554c
100012d0:	10005220 	.word	0x10005220
100012d4:	10005318 	.word	0x10005318
100012d8:	10005580 	.word	0x10005580
100012dc:	100052dc 	.word	0x100052dc
100012e0:	10005400 	.word	0x10005400
100012e4:	10005564 	.word	0x10005564
100012e8:	10005418 	.word	0x10005418
100012ec:	100055a4 	.word	0x100055a4
100012f0:	0fffffff 	.word	0x0fffffff
100012f4:	10005424 	.word	0x10005424
100012f8:	7fffffff 	.word	0x7fffffff
100012fc:	1000533c 	.word	0x1000533c
10001300:	100055ec 	.word	0x100055ec
10001304:	10005358 	.word	0x10005358
10001308:	10005460 	.word	0x10005460
1000130c:	100055b8 	.word	0x100055b8
10001310:	10005484 	.word	0x10005484

10001314 <alarm_pool_init_default>:
10001314:	b510      	push	{r4, lr}
10001316:	4b0c      	ldr	r3, [pc, #48]	; (10001348 <alarm_pool_init_default+0x34>)
10001318:	685b      	ldr	r3, [r3, #4]
1000131a:	2b00      	cmp	r3, #0
1000131c:	d004      	beq.n	10001328 <alarm_pool_init_default+0x14>
1000131e:	210a      	movs	r1, #10
10001320:	480a      	ldr	r0, [pc, #40]	; (1000134c <alarm_pool_init_default+0x38>)
10001322:	f7ff fc93 	bl	10000c4c <lock_init>
10001326:	bd10      	pop	{r4, pc}
10001328:	4c07      	ldr	r4, [pc, #28]	; (10001348 <alarm_pool_init_default+0x34>)
1000132a:	0023      	movs	r3, r4
1000132c:	4a08      	ldr	r2, [pc, #32]	; (10001350 <alarm_pool_init_default+0x3c>)
1000132e:	2110      	movs	r1, #16
10001330:	6820      	ldr	r0, [r4, #0]
10001332:	f000 fc7d 	bl	10001c30 <ph_post_alloc_init>
10001336:	2003      	movs	r0, #3
10001338:	f000 faa4 	bl	10001884 <hardware_alarm_claim>
1000133c:	2103      	movs	r1, #3
1000133e:	0020      	movs	r0, r4
10001340:	f7ff fca8 	bl	10000c94 <alarm_pool_post_alloc_init>
10001344:	e7eb      	b.n	1000131e <alarm_pool_init_default+0xa>
10001346:	46c0      	nop			; (mov r8, r8)
10001348:	20000288 	.word	0x20000288
1000134c:	200006c8 	.word	0x200006c8
10001350:	10000d05 	.word	0x10000d05

10001354 <alarm_pool_get_default>:
10001354:	b510      	push	{r4, lr}
10001356:	4b06      	ldr	r3, [pc, #24]	; (10001370 <alarm_pool_get_default+0x1c>)
10001358:	685b      	ldr	r3, [r3, #4]
1000135a:	2b00      	cmp	r3, #0
1000135c:	d001      	beq.n	10001362 <alarm_pool_get_default+0xe>
1000135e:	4804      	ldr	r0, [pc, #16]	; (10001370 <alarm_pool_get_default+0x1c>)
10001360:	bd10      	pop	{r4, pc}
10001362:	4b04      	ldr	r3, [pc, #16]	; (10001374 <alarm_pool_get_default+0x20>)
10001364:	4a04      	ldr	r2, [pc, #16]	; (10001378 <alarm_pool_get_default+0x24>)
10001366:	215e      	movs	r1, #94	; 0x5e
10001368:	4804      	ldr	r0, [pc, #16]	; (1000137c <alarm_pool_get_default+0x28>)
1000136a:	f001 f861 	bl	10002430 <__assert_func>
1000136e:	46c0      	nop			; (mov r8, r8)
10001370:	20000288 	.word	0x20000288
10001374:	10005498 	.word	0x10005498
10001378:	1000558c 	.word	0x1000558c
1000137c:	100052dc 	.word	0x100052dc

10001380 <alarm_pool_add_alarm_at>:
10001380:	b5f0      	push	{r4, r5, r6, r7, lr}
10001382:	46de      	mov	lr, fp
10001384:	4657      	mov	r7, sl
10001386:	464e      	mov	r6, r9
10001388:	4645      	mov	r5, r8
1000138a:	b5e0      	push	{r5, r6, r7, lr}
1000138c:	b08b      	sub	sp, #44	; 0x2c
1000138e:	4680      	mov	r8, r0
10001390:	0016      	movs	r6, r2
10001392:	001f      	movs	r7, r3
10001394:	9b14      	ldr	r3, [sp, #80]	; 0x50
10001396:	469a      	mov	sl, r3
10001398:	9b15      	ldr	r3, [sp, #84]	; 0x54
1000139a:	4699      	mov	r9, r3
1000139c:	ab16      	add	r3, sp, #88	; 0x58
1000139e:	781b      	ldrb	r3, [r3, #0]
100013a0:	469b      	mov	fp, r3
100013a2:	231f      	movs	r3, #31
100013a4:	aa02      	add	r2, sp, #8
100013a6:	4694      	mov	ip, r2
100013a8:	4463      	add	r3, ip
100013aa:	2200      	movs	r2, #0
100013ac:	701a      	strb	r2, [r3, #0]
100013ae:	e02b      	b.n	10001408 <alarm_pool_add_alarm_at+0x88>
100013b0:	2800      	cmp	r0, #0
100013b2:	d009      	beq.n	100013c8 <alarm_pool_add_alarm_at+0x48>
100013b4:	4642      	mov	r2, r8
100013b6:	6812      	ldr	r2, [r2, #0]
100013b8:	7b12      	ldrb	r2, [r2, #12]
100013ba:	4290      	cmp	r0, r2
100013bc:	d804      	bhi.n	100013c8 <alarm_pool_add_alarm_at+0x48>
100013be:	1e42      	subs	r2, r0, #1
100013c0:	4641      	mov	r1, r8
100013c2:	68c9      	ldr	r1, [r1, #12]
100013c4:	5c8a      	ldrb	r2, [r1, r2]
100013c6:	e041      	b.n	1000144c <alarm_pool_add_alarm_at+0xcc>
100013c8:	4b40      	ldr	r3, [pc, #256]	; (100014cc <alarm_pool_add_alarm_at+0x14c>)
100013ca:	4a41      	ldr	r2, [pc, #260]	; (100014d0 <alarm_pool_add_alarm_at+0x150>)
100013cc:	2141      	movs	r1, #65	; 0x41
100013ce:	4841      	ldr	r0, [pc, #260]	; (100014d4 <alarm_pool_add_alarm_at+0x154>)
100013d0:	f001 f82e 	bl	10002430 <__assert_func>
100013d4:	9807      	ldr	r0, [sp, #28]
100013d6:	e04c      	b.n	10001472 <alarm_pool_add_alarm_at+0xf2>
100013d8:	1b36      	subs	r6, r6, r4
100013da:	41af      	sbcs	r7, r5
100013dc:	2f00      	cmp	r7, #0
100013de:	db07      	blt.n	100013f0 <alarm_pool_add_alarm_at+0x70>
100013e0:	2f00      	cmp	r7, #0
100013e2:	da11      	bge.n	10001408 <alarm_pool_add_alarm_at+0x88>
100013e4:	4b3c      	ldr	r3, [pc, #240]	; (100014d8 <alarm_pool_add_alarm_at+0x158>)
100013e6:	4a3d      	ldr	r2, [pc, #244]	; (100014dc <alarm_pool_add_alarm_at+0x15c>)
100013e8:	213f      	movs	r1, #63	; 0x3f
100013ea:	483d      	ldr	r0, [pc, #244]	; (100014e0 <alarm_pool_add_alarm_at+0x160>)
100013ec:	f001 f820 	bl	10002430 <__assert_func>
100013f0:	2601      	movs	r6, #1
100013f2:	4276      	negs	r6, r6
100013f4:	4f3b      	ldr	r7, [pc, #236]	; (100014e4 <alarm_pool_add_alarm_at+0x164>)
100013f6:	e7f3      	b.n	100013e0 <alarm_pool_add_alarm_at+0x60>
100013f8:	4b37      	ldr	r3, [pc, #220]	; (100014d8 <alarm_pool_add_alarm_at+0x158>)
100013fa:	4a38      	ldr	r2, [pc, #224]	; (100014dc <alarm_pool_add_alarm_at+0x15c>)
100013fc:	213f      	movs	r1, #63	; 0x3f
100013fe:	4838      	ldr	r0, [pc, #224]	; (100014e0 <alarm_pool_add_alarm_at+0x160>)
10001400:	f001 f816 	bl	10002430 <__assert_func>
10001404:	2f00      	cmp	r7, #0
10001406:	db4f      	blt.n	100014a8 <alarm_pool_add_alarm_at+0x128>
10001408:	4643      	mov	r3, r8
1000140a:	685a      	ldr	r2, [r3, #4]
1000140c:	f3ef 8410 	mrs	r4, PRIMASK
10001410:	b672      	cpsid	i
10001412:	6813      	ldr	r3, [r2, #0]
10001414:	4259      	negs	r1, r3
10001416:	414b      	adcs	r3, r1
10001418:	b2d9      	uxtb	r1, r3
1000141a:	9107      	str	r1, [sp, #28]
1000141c:	2b00      	cmp	r3, #0
1000141e:	d1f8      	bne.n	10001412 <alarm_pool_add_alarm_at+0x92>
10001420:	f3bf 8f5f 	dmb	sy
10001424:	331f      	adds	r3, #31
10001426:	aa02      	add	r2, sp, #8
10001428:	4694      	mov	ip, r2
1000142a:	4463      	add	r3, ip
1000142c:	9304      	str	r3, [sp, #16]
1000142e:	2300      	movs	r3, #0
10001430:	9303      	str	r3, [sp, #12]
10001432:	9302      	str	r3, [sp, #8]
10001434:	464b      	mov	r3, r9
10001436:	9301      	str	r3, [sp, #4]
10001438:	4653      	mov	r3, sl
1000143a:	9300      	str	r3, [sp, #0]
1000143c:	0032      	movs	r2, r6
1000143e:	003b      	movs	r3, r7
10001440:	4640      	mov	r0, r8
10001442:	f7ff fd0f 	bl	10000e64 <add_alarm_under_lock>
10001446:	1e03      	subs	r3, r0, #0
10001448:	d1b2      	bne.n	100013b0 <alarm_pool_add_alarm_at+0x30>
1000144a:	0002      	movs	r2, r0
1000144c:	4641      	mov	r1, r8
1000144e:	6849      	ldr	r1, [r1, #4]
10001450:	f3bf 8f5f 	dmb	sy
10001454:	2500      	movs	r5, #0
10001456:	600d      	str	r5, [r1, #0]
10001458:	f384 8810 	msr	PRIMASK, r4
1000145c:	2b00      	cmp	r3, #0
1000145e:	d029      	beq.n	100014b4 <alarm_pool_add_alarm_at+0x134>
10001460:	231f      	movs	r3, #31
10001462:	a902      	add	r1, sp, #8
10001464:	468c      	mov	ip, r1
10001466:	4463      	add	r3, ip
10001468:	781b      	ldrb	r3, [r3, #0]
1000146a:	2b00      	cmp	r3, #0
1000146c:	d1b2      	bne.n	100013d4 <alarm_pool_add_alarm_at+0x54>
1000146e:	0212      	lsls	r2, r2, #8
10001470:	4310      	orrs	r0, r2
10001472:	2b00      	cmp	r3, #0
10001474:	d020      	beq.n	100014b8 <alarm_pool_add_alarm_at+0x138>
10001476:	465b      	mov	r3, fp
10001478:	2b00      	cmp	r3, #0
1000147a:	d01d      	beq.n	100014b8 <alarm_pool_add_alarm_at+0x138>
1000147c:	4649      	mov	r1, r9
1000147e:	47d0      	blx	sl
10001480:	0004      	movs	r4, r0
10001482:	000d      	movs	r5, r1
10001484:	0003      	movs	r3, r0
10001486:	430b      	orrs	r3, r1
10001488:	d01d      	beq.n	100014c6 <alarm_pool_add_alarm_at+0x146>
1000148a:	2900      	cmp	r1, #0
1000148c:	dba4      	blt.n	100013d8 <alarm_pool_add_alarm_at+0x58>
1000148e:	f000 fa05 	bl	1000189c <time_us_64>
10001492:	0006      	movs	r6, r0
10001494:	1e0f      	subs	r7, r1, #0
10001496:	dbaf      	blt.n	100013f8 <alarm_pool_add_alarm_at+0x78>
10001498:	1936      	adds	r6, r6, r4
1000149a:	416f      	adcs	r7, r5
1000149c:	2f00      	cmp	r7, #0
1000149e:	dab1      	bge.n	10001404 <alarm_pool_add_alarm_at+0x84>
100014a0:	2601      	movs	r6, #1
100014a2:	4276      	negs	r6, r6
100014a4:	4f0f      	ldr	r7, [pc, #60]	; (100014e4 <alarm_pool_add_alarm_at+0x164>)
100014a6:	e7ad      	b.n	10001404 <alarm_pool_add_alarm_at+0x84>
100014a8:	4b0b      	ldr	r3, [pc, #44]	; (100014d8 <alarm_pool_add_alarm_at+0x158>)
100014aa:	4a0c      	ldr	r2, [pc, #48]	; (100014dc <alarm_pool_add_alarm_at+0x15c>)
100014ac:	213f      	movs	r1, #63	; 0x3f
100014ae:	480c      	ldr	r0, [pc, #48]	; (100014e0 <alarm_pool_add_alarm_at+0x160>)
100014b0:	f000 ffbe 	bl	10002430 <__assert_func>
100014b4:	2001      	movs	r0, #1
100014b6:	4240      	negs	r0, r0
100014b8:	b00b      	add	sp, #44	; 0x2c
100014ba:	bcf0      	pop	{r4, r5, r6, r7}
100014bc:	46bb      	mov	fp, r7
100014be:	46b2      	mov	sl, r6
100014c0:	46a9      	mov	r9, r5
100014c2:	46a0      	mov	r8, r4
100014c4:	bdf0      	pop	{r4, r5, r6, r7, pc}
100014c6:	9807      	ldr	r0, [sp, #28]
100014c8:	e7f6      	b.n	100014b8 <alarm_pool_add_alarm_at+0x138>
100014ca:	46c0      	nop			; (mov r8, r8)
100014cc:	10005318 	.word	0x10005318
100014d0:	100055a4 	.word	0x100055a4
100014d4:	100052dc 	.word	0x100052dc
100014d8:	10005204 	.word	0x10005204
100014dc:	1000554c 	.word	0x1000554c
100014e0:	10005220 	.word	0x10005220
100014e4:	7fffffff 	.word	0x7fffffff

100014e8 <alarm_pool_cancel_alarm>:
100014e8:	b5f8      	push	{r3, r4, r5, r6, r7, lr}
100014ea:	0004      	movs	r4, r0
100014ec:	2900      	cmp	r1, #0
100014ee:	d100      	bne.n	100014f2 <alarm_pool_cancel_alarm+0xa>
100014f0:	e062      	b.n	100015b8 <alarm_pool_cancel_alarm+0xd0>
100014f2:	6842      	ldr	r2, [r0, #4]
100014f4:	f3ef 8510 	mrs	r5, PRIMASK
100014f8:	b672      	cpsid	i
100014fa:	6813      	ldr	r3, [r2, #0]
100014fc:	4258      	negs	r0, r3
100014fe:	4143      	adcs	r3, r0
10001500:	b2d8      	uxtb	r0, r3
10001502:	2b00      	cmp	r3, #0
10001504:	d1f9      	bne.n	100014fa <alarm_pool_cancel_alarm+0x12>
10001506:	f3bf 8f5f 	dmb	sy
1000150a:	b2cb      	uxtb	r3, r1
1000150c:	6822      	ldr	r2, [r4, #0]
1000150e:	7b56      	ldrb	r6, [r2, #13]
10001510:	42b3      	cmp	r3, r6
10001512:	d11b      	bne.n	1000154c <alarm_pool_cancel_alarm+0x64>
10001514:	2001      	movs	r0, #1
10001516:	2800      	cmp	r0, #0
10001518:	d048      	beq.n	100015ac <alarm_pool_cancel_alarm+0xc4>
1000151a:	6920      	ldr	r0, [r4, #16]
1000151c:	4288      	cmp	r0, r1
1000151e:	d02b      	beq.n	10001578 <alarm_pool_cancel_alarm+0x90>
10001520:	0a09      	lsrs	r1, r1, #8
10001522:	b2c9      	uxtb	r1, r1
10001524:	2b00      	cmp	r3, #0
10001526:	d02e      	beq.n	10001586 <alarm_pool_cancel_alarm+0x9e>
10001528:	6820      	ldr	r0, [r4, #0]
1000152a:	7b00      	ldrb	r0, [r0, #12]
1000152c:	4283      	cmp	r3, r0
1000152e:	d82a      	bhi.n	10001586 <alarm_pool_cancel_alarm+0x9e>
10001530:	1e58      	subs	r0, r3, #1
10001532:	68e6      	ldr	r6, [r4, #12]
10001534:	5c30      	ldrb	r0, [r6, r0]
10001536:	4288      	cmp	r0, r1
10001538:	d02b      	beq.n	10001592 <alarm_pool_cancel_alarm+0xaa>
1000153a:	2000      	movs	r0, #0
1000153c:	6863      	ldr	r3, [r4, #4]
1000153e:	f3bf 8f5f 	dmb	sy
10001542:	2200      	movs	r2, #0
10001544:	601a      	str	r2, [r3, #0]
10001546:	f385 8810 	msr	PRIMASK, r5
1000154a:	bdf8      	pop	{r3, r4, r5, r6, r7, pc}
1000154c:	2b00      	cmp	r3, #0
1000154e:	d00d      	beq.n	1000156c <alarm_pool_cancel_alarm+0x84>
10001550:	7b16      	ldrb	r6, [r2, #12]
10001552:	42b3      	cmp	r3, r6
10001554:	d80a      	bhi.n	1000156c <alarm_pool_cancel_alarm+0x84>
10001556:	005e      	lsls	r6, r3, #1
10001558:	18f6      	adds	r6, r6, r3
1000155a:	3e03      	subs	r6, #3
1000155c:	6817      	ldr	r7, [r2, #0]
1000155e:	46bc      	mov	ip, r7
10001560:	4466      	add	r6, ip
10001562:	78b6      	ldrb	r6, [r6, #2]
10001564:	2e00      	cmp	r6, #0
10001566:	d0d6      	beq.n	10001516 <alarm_pool_cancel_alarm+0x2e>
10001568:	2001      	movs	r0, #1
1000156a:	e7d4      	b.n	10001516 <alarm_pool_cancel_alarm+0x2e>
1000156c:	4b13      	ldr	r3, [pc, #76]	; (100015bc <alarm_pool_cancel_alarm+0xd4>)
1000156e:	4a14      	ldr	r2, [pc, #80]	; (100015c0 <alarm_pool_cancel_alarm+0xd8>)
10001570:	2168      	movs	r1, #104	; 0x68
10001572:	4814      	ldr	r0, [pc, #80]	; (100015c4 <alarm_pool_cancel_alarm+0xdc>)
10001574:	f000 ff5c 	bl	10002430 <__assert_func>
10001578:	212c      	movs	r1, #44	; 0x2c
1000157a:	4b13      	ldr	r3, [pc, #76]	; (100015c8 <alarm_pool_cancel_alarm+0xe0>)
1000157c:	4a13      	ldr	r2, [pc, #76]	; (100015cc <alarm_pool_cancel_alarm+0xe4>)
1000157e:	31ff      	adds	r1, #255	; 0xff
10001580:	4813      	ldr	r0, [pc, #76]	; (100015d0 <alarm_pool_cancel_alarm+0xe8>)
10001582:	f000 ff55 	bl	10002430 <__assert_func>
10001586:	4b13      	ldr	r3, [pc, #76]	; (100015d4 <alarm_pool_cancel_alarm+0xec>)
10001588:	4a13      	ldr	r2, [pc, #76]	; (100015d8 <alarm_pool_cancel_alarm+0xf0>)
1000158a:	2141      	movs	r1, #65	; 0x41
1000158c:	4810      	ldr	r0, [pc, #64]	; (100015d0 <alarm_pool_cancel_alarm+0xe8>)
1000158e:	f000 ff4f 	bl	10002430 <__assert_func>
10001592:	0019      	movs	r1, r3
10001594:	0010      	movs	r0, r2
10001596:	f000 fc45 	bl	10001e24 <ph_remove_and_free_node>
1000159a:	2800      	cmp	r0, #0
1000159c:	d1ce      	bne.n	1000153c <alarm_pool_cancel_alarm+0x54>
1000159e:	2199      	movs	r1, #153	; 0x99
100015a0:	4b0e      	ldr	r3, [pc, #56]	; (100015dc <alarm_pool_cancel_alarm+0xf4>)
100015a2:	4a0a      	ldr	r2, [pc, #40]	; (100015cc <alarm_pool_cancel_alarm+0xe4>)
100015a4:	0049      	lsls	r1, r1, #1
100015a6:	480a      	ldr	r0, [pc, #40]	; (100015d0 <alarm_pool_cancel_alarm+0xe8>)
100015a8:	f000 ff42 	bl	10002430 <__assert_func>
100015ac:	6923      	ldr	r3, [r4, #16]
100015ae:	428b      	cmp	r3, r1
100015b0:	d1c4      	bne.n	1000153c <alarm_pool_cancel_alarm+0x54>
100015b2:	2300      	movs	r3, #0
100015b4:	6123      	str	r3, [r4, #16]
100015b6:	e7c1      	b.n	1000153c <alarm_pool_cancel_alarm+0x54>
100015b8:	2000      	movs	r0, #0
100015ba:	e7c6      	b.n	1000154a <alarm_pool_cancel_alarm+0x62>
100015bc:	1000533c 	.word	0x1000533c
100015c0:	100055ec 	.word	0x100055ec
100015c4:	10005358 	.word	0x10005358
100015c8:	100054bc 	.word	0x100054bc
100015cc:	10005534 	.word	0x10005534
100015d0:	100052dc 	.word	0x100052dc
100015d4:	10005318 	.word	0x10005318
100015d8:	100055a4 	.word	0x100055a4
100015dc:	100054e0 	.word	0x100054e0

100015e0 <sleep_until>:
100015e0:	b5f0      	push	{r4, r5, r6, r7, lr}
100015e2:	b087      	sub	sp, #28
100015e4:	0006      	movs	r6, r0
100015e6:	000f      	movs	r7, r1
100015e8:	f3ef 8305 	mrs	r3, IPSR
100015ec:	2b00      	cmp	r3, #0
100015ee:	d11f      	bne.n	10001630 <sleep_until+0x50>
100015f0:	2406      	movs	r4, #6
100015f2:	4264      	negs	r4, r4
100015f4:	17e5      	asrs	r5, r4, #31
100015f6:	19a4      	adds	r4, r4, r6
100015f8:	417d      	adcs	r5, r7
100015fa:	428d      	cmp	r5, r1
100015fc:	d802      	bhi.n	10001604 <sleep_until+0x24>
100015fe:	d103      	bne.n	10001608 <sleep_until+0x28>
10001600:	4284      	cmp	r4, r0
10001602:	d901      	bls.n	10001608 <sleep_until+0x28>
10001604:	2400      	movs	r4, #0
10001606:	2500      	movs	r5, #0
10001608:	2d00      	cmp	r5, #0
1000160a:	db14      	blt.n	10001636 <sleep_until+0x56>
1000160c:	9404      	str	r4, [sp, #16]
1000160e:	9505      	str	r5, [sp, #20]
10001610:	f000 f944 	bl	1000189c <time_us_64>
10001614:	0002      	movs	r2, r0
10001616:	1e0b      	subs	r3, r1, #0
10001618:	db13      	blt.n	10001642 <sleep_until+0x62>
1000161a:	1aa4      	subs	r4, r4, r2
1000161c:	419d      	sbcs	r5, r3
1000161e:	2d00      	cmp	r5, #0
10001620:	dc17      	bgt.n	10001652 <sleep_until+0x72>
10001622:	d014      	beq.n	1000164e <sleep_until+0x6e>
10001624:	0030      	movs	r0, r6
10001626:	0039      	movs	r1, r7
10001628:	f000 f944 	bl	100018b4 <busy_wait_until>
1000162c:	b007      	add	sp, #28
1000162e:	bdf0      	pop	{r4, r5, r6, r7, pc}
10001630:	4823      	ldr	r0, [pc, #140]	; (100016c0 <sleep_until+0xe0>)
10001632:	f000 ff97 	bl	10002564 <panic>
10001636:	4b23      	ldr	r3, [pc, #140]	; (100016c4 <sleep_until+0xe4>)
10001638:	4a23      	ldr	r2, [pc, #140]	; (100016c8 <sleep_until+0xe8>)
1000163a:	213f      	movs	r1, #63	; 0x3f
1000163c:	4823      	ldr	r0, [pc, #140]	; (100016cc <sleep_until+0xec>)
1000163e:	f000 fef7 	bl	10002430 <__assert_func>
10001642:	4b20      	ldr	r3, [pc, #128]	; (100016c4 <sleep_until+0xe4>)
10001644:	4a20      	ldr	r2, [pc, #128]	; (100016c8 <sleep_until+0xe8>)
10001646:	213f      	movs	r1, #63	; 0x3f
10001648:	4820      	ldr	r0, [pc, #128]	; (100016cc <sleep_until+0xec>)
1000164a:	f000 fef1 	bl	10002430 <__assert_func>
1000164e:	2c00      	cmp	r4, #0
10001650:	d0e8      	beq.n	10001624 <sleep_until+0x44>
10001652:	f7ff fe7f 	bl	10001354 <alarm_pool_get_default>
10001656:	2300      	movs	r3, #0
10001658:	9302      	str	r3, [sp, #8]
1000165a:	9301      	str	r3, [sp, #4]
1000165c:	4b1c      	ldr	r3, [pc, #112]	; (100016d0 <sleep_until+0xf0>)
1000165e:	9300      	str	r3, [sp, #0]
10001660:	9a04      	ldr	r2, [sp, #16]
10001662:	9b05      	ldr	r3, [sp, #20]
10001664:	f7ff fe8c 	bl	10001380 <alarm_pool_add_alarm_at>
10001668:	2800      	cmp	r0, #0
1000166a:	da18      	bge.n	1000169e <sleep_until+0xbe>
1000166c:	e7da      	b.n	10001624 <sleep_until+0x44>
1000166e:	2300      	movs	r3, #0
10001670:	e000      	b.n	10001674 <sleep_until+0x94>
10001672:	2300      	movs	r3, #0
10001674:	2b00      	cmp	r3, #0
10001676:	d1d5      	bne.n	10001624 <sleep_until+0x44>
10001678:	4b16      	ldr	r3, [pc, #88]	; (100016d4 <sleep_until+0xf4>)
1000167a:	681a      	ldr	r2, [r3, #0]
1000167c:	f3ef 8110 	mrs	r1, PRIMASK
10001680:	b672      	cpsid	i
10001682:	6813      	ldr	r3, [r2, #0]
10001684:	2b00      	cmp	r3, #0
10001686:	d0fc      	beq.n	10001682 <sleep_until+0xa2>
10001688:	f3bf 8f5f 	dmb	sy
1000168c:	4b11      	ldr	r3, [pc, #68]	; (100016d4 <sleep_until+0xf4>)
1000168e:	681b      	ldr	r3, [r3, #0]
10001690:	f3bf 8f5f 	dmb	sy
10001694:	2200      	movs	r2, #0
10001696:	601a      	str	r2, [r3, #0]
10001698:	f381 8810 	msr	PRIMASK, r1
1000169c:	bf20      	wfe
1000169e:	9904      	ldr	r1, [sp, #16]
100016a0:	9a05      	ldr	r2, [sp, #20]
100016a2:	4b0d      	ldr	r3, [pc, #52]	; (100016d8 <sleep_until+0xf8>)
100016a4:	6a5b      	ldr	r3, [r3, #36]	; 0x24
100016a6:	429a      	cmp	r2, r3
100016a8:	d8e3      	bhi.n	10001672 <sleep_until+0x92>
100016aa:	480b      	ldr	r0, [pc, #44]	; (100016d8 <sleep_until+0xf8>)
100016ac:	6a80      	ldr	r0, [r0, #40]	; 0x28
100016ae:	4288      	cmp	r0, r1
100016b0:	d203      	bcs.n	100016ba <sleep_until+0xda>
100016b2:	429a      	cmp	r2, r3
100016b4:	d0db      	beq.n	1000166e <sleep_until+0x8e>
100016b6:	2301      	movs	r3, #1
100016b8:	e7dc      	b.n	10001674 <sleep_until+0x94>
100016ba:	2301      	movs	r3, #1
100016bc:	e7da      	b.n	10001674 <sleep_until+0x94>
100016be:	46c0      	nop			; (mov r8, r8)
100016c0:	100054e4 	.word	0x100054e4
100016c4:	10005204 	.word	0x10005204
100016c8:	1000554c 	.word	0x1000554c
100016cc:	10005220 	.word	0x10005220
100016d0:	10000cd5 	.word	0x10000cd5
100016d4:	200006c8 	.word	0x200006c8
100016d8:	40054000 	.word	0x40054000

100016dc <sleep_us>:
100016dc:	b570      	push	{r4, r5, r6, lr}
100016de:	0004      	movs	r4, r0
100016e0:	000d      	movs	r5, r1
100016e2:	f000 f8db 	bl	1000189c <time_us_64>
100016e6:	0002      	movs	r2, r0
100016e8:	1e0b      	subs	r3, r1, #0
100016ea:	db0a      	blt.n	10001702 <sleep_us+0x26>
100016ec:	0020      	movs	r0, r4
100016ee:	0029      	movs	r1, r5
100016f0:	1880      	adds	r0, r0, r2
100016f2:	4159      	adcs	r1, r3
100016f4:	2900      	cmp	r1, #0
100016f6:	db0a      	blt.n	1000170e <sleep_us+0x32>
100016f8:	2900      	cmp	r1, #0
100016fa:	db0c      	blt.n	10001716 <sleep_us+0x3a>
100016fc:	f7ff ff70 	bl	100015e0 <sleep_until>
10001700:	bd70      	pop	{r4, r5, r6, pc}
10001702:	4b08      	ldr	r3, [pc, #32]	; (10001724 <sleep_us+0x48>)
10001704:	4a08      	ldr	r2, [pc, #32]	; (10001728 <sleep_us+0x4c>)
10001706:	213f      	movs	r1, #63	; 0x3f
10001708:	4808      	ldr	r0, [pc, #32]	; (1000172c <sleep_us+0x50>)
1000170a:	f000 fe91 	bl	10002430 <__assert_func>
1000170e:	2001      	movs	r0, #1
10001710:	4240      	negs	r0, r0
10001712:	4907      	ldr	r1, [pc, #28]	; (10001730 <sleep_us+0x54>)
10001714:	e7f0      	b.n	100016f8 <sleep_us+0x1c>
10001716:	4b03      	ldr	r3, [pc, #12]	; (10001724 <sleep_us+0x48>)
10001718:	4a03      	ldr	r2, [pc, #12]	; (10001728 <sleep_us+0x4c>)
1000171a:	213f      	movs	r1, #63	; 0x3f
1000171c:	4803      	ldr	r0, [pc, #12]	; (1000172c <sleep_us+0x50>)
1000171e:	f000 fe87 	bl	10002430 <__assert_func>
10001722:	46c0      	nop			; (mov r8, r8)
10001724:	10005204 	.word	0x10005204
10001728:	1000554c 	.word	0x1000554c
1000172c:	10005220 	.word	0x10005220
10001730:	7fffffff 	.word	0x7fffffff

10001734 <sleep_ms>:
10001734:	b510      	push	{r4, lr}
10001736:	22fa      	movs	r2, #250	; 0xfa
10001738:	0092      	lsls	r2, r2, #2
1000173a:	2300      	movs	r3, #0
1000173c:	2100      	movs	r1, #0
1000173e:	f002 fe61 	bl	10004404 <__wrap___aeabi_lmul>
10001742:	f7ff ffcb 	bl	100016dc <sleep_us>
10001746:	bd10      	pop	{r4, pc}

10001748 <best_effort_wfe_or_timeout>:
10001748:	b570      	push	{r4, r5, r6, lr}
1000174a:	b084      	sub	sp, #16
1000174c:	0005      	movs	r5, r0
1000174e:	000c      	movs	r4, r1
10001750:	f3ef 8305 	mrs	r3, IPSR
10001754:	2b00      	cmp	r3, #0
10001756:	d11e      	bne.n	10001796 <best_effort_wfe_or_timeout+0x4e>
10001758:	f7ff fdfc 	bl	10001354 <alarm_pool_get_default>
1000175c:	2300      	movs	r3, #0
1000175e:	9302      	str	r3, [sp, #8]
10001760:	9301      	str	r3, [sp, #4]
10001762:	4b22      	ldr	r3, [pc, #136]	; (100017ec <best_effort_wfe_or_timeout+0xa4>)
10001764:	9300      	str	r3, [sp, #0]
10001766:	002a      	movs	r2, r5
10001768:	0023      	movs	r3, r4
1000176a:	f7ff fe09 	bl	10001380 <alarm_pool_add_alarm_at>
1000176e:	1e06      	subs	r6, r0, #0
10001770:	dd23      	ble.n	100017ba <best_effort_wfe_or_timeout+0x72>
10001772:	bf20      	wfe
10001774:	f7ff fdee 	bl	10001354 <alarm_pool_get_default>
10001778:	0031      	movs	r1, r6
1000177a:	f7ff feb5 	bl	100014e8 <alarm_pool_cancel_alarm>
1000177e:	4b1c      	ldr	r3, [pc, #112]	; (100017f0 <best_effort_wfe_or_timeout+0xa8>)
10001780:	6a5b      	ldr	r3, [r3, #36]	; 0x24
10001782:	429c      	cmp	r4, r3
10001784:	d82d      	bhi.n	100017e2 <best_effort_wfe_or_timeout+0x9a>
10001786:	4a1a      	ldr	r2, [pc, #104]	; (100017f0 <best_effort_wfe_or_timeout+0xa8>)
10001788:	6a92      	ldr	r2, [r2, #40]	; 0x28
1000178a:	42aa      	cmp	r2, r5
1000178c:	d22c      	bcs.n	100017e8 <best_effort_wfe_or_timeout+0xa0>
1000178e:	429c      	cmp	r4, r3
10001790:	d025      	beq.n	100017de <best_effort_wfe_or_timeout+0x96>
10001792:	2001      	movs	r0, #1
10001794:	e026      	b.n	100017e4 <best_effort_wfe_or_timeout+0x9c>
10001796:	4b16      	ldr	r3, [pc, #88]	; (100017f0 <best_effort_wfe_or_timeout+0xa8>)
10001798:	6a5b      	ldr	r3, [r3, #36]	; 0x24
1000179a:	4299      	cmp	r1, r3
1000179c:	d809      	bhi.n	100017b2 <best_effort_wfe_or_timeout+0x6a>
1000179e:	4a14      	ldr	r2, [pc, #80]	; (100017f0 <best_effort_wfe_or_timeout+0xa8>)
100017a0:	6a92      	ldr	r2, [r2, #40]	; 0x28
100017a2:	4282      	cmp	r2, r0
100017a4:	d207      	bcs.n	100017b6 <best_effort_wfe_or_timeout+0x6e>
100017a6:	4299      	cmp	r1, r3
100017a8:	d001      	beq.n	100017ae <best_effort_wfe_or_timeout+0x66>
100017aa:	2001      	movs	r0, #1
100017ac:	e01a      	b.n	100017e4 <best_effort_wfe_or_timeout+0x9c>
100017ae:	2000      	movs	r0, #0
100017b0:	e018      	b.n	100017e4 <best_effort_wfe_or_timeout+0x9c>
100017b2:	2000      	movs	r0, #0
100017b4:	e016      	b.n	100017e4 <best_effort_wfe_or_timeout+0x9c>
100017b6:	2001      	movs	r0, #1
100017b8:	e014      	b.n	100017e4 <best_effort_wfe_or_timeout+0x9c>
100017ba:	4b0d      	ldr	r3, [pc, #52]	; (100017f0 <best_effort_wfe_or_timeout+0xa8>)
100017bc:	6a5b      	ldr	r3, [r3, #36]	; 0x24
100017be:	429c      	cmp	r4, r3
100017c0:	d809      	bhi.n	100017d6 <best_effort_wfe_or_timeout+0x8e>
100017c2:	4a0b      	ldr	r2, [pc, #44]	; (100017f0 <best_effort_wfe_or_timeout+0xa8>)
100017c4:	6a92      	ldr	r2, [r2, #40]	; 0x28
100017c6:	42aa      	cmp	r2, r5
100017c8:	d207      	bcs.n	100017da <best_effort_wfe_or_timeout+0x92>
100017ca:	429c      	cmp	r4, r3
100017cc:	d001      	beq.n	100017d2 <best_effort_wfe_or_timeout+0x8a>
100017ce:	2001      	movs	r0, #1
100017d0:	e008      	b.n	100017e4 <best_effort_wfe_or_timeout+0x9c>
100017d2:	2000      	movs	r0, #0
100017d4:	e006      	b.n	100017e4 <best_effort_wfe_or_timeout+0x9c>
100017d6:	2000      	movs	r0, #0
100017d8:	e004      	b.n	100017e4 <best_effort_wfe_or_timeout+0x9c>
100017da:	2001      	movs	r0, #1
100017dc:	e002      	b.n	100017e4 <best_effort_wfe_or_timeout+0x9c>
100017de:	2000      	movs	r0, #0
100017e0:	e000      	b.n	100017e4 <best_effort_wfe_or_timeout+0x9c>
100017e2:	2000      	movs	r0, #0
100017e4:	b004      	add	sp, #16
100017e6:	bd70      	pop	{r4, r5, r6, pc}
100017e8:	2001      	movs	r0, #1
100017ea:	e7fb      	b.n	100017e4 <best_effort_wfe_or_timeout+0x9c>
100017ec:	10000cd5 	.word	0x10000cd5
100017f0:	40054000 	.word	0x40054000

100017f4 <hardware_alarm_irq_handler>:
100017f4:	b570      	push	{r4, r5, r6, lr}
100017f6:	f3ef 8005 	mrs	r0, IPSR
100017fa:	3810      	subs	r0, #16
100017fc:	f3ef 8c10 	mrs	ip, PRIMASK
10001800:	b672      	cpsid	i
10001802:	4b1a      	ldr	r3, [pc, #104]	; (1000186c <hardware_alarm_irq_handler+0x78>)
10001804:	681b      	ldr	r3, [r3, #0]
10001806:	2b00      	cmp	r3, #0
10001808:	d0fb      	beq.n	10001802 <hardware_alarm_irq_handler+0xe>
1000180a:	f3bf 8f5f 	dmb	sy
1000180e:	2201      	movs	r2, #1
10001810:	0013      	movs	r3, r2
10001812:	4083      	lsls	r3, r0
10001814:	4916      	ldr	r1, [pc, #88]	; (10001870 <hardware_alarm_irq_handler+0x7c>)
10001816:	634b      	str	r3, [r1, #52]	; 0x34
10001818:	4916      	ldr	r1, [pc, #88]	; (10001874 <hardware_alarm_irq_handler+0x80>)
1000181a:	600b      	str	r3, [r1, #0]
1000181c:	4916      	ldr	r1, [pc, #88]	; (10001878 <hardware_alarm_irq_handler+0x84>)
1000181e:	7809      	ldrb	r1, [r1, #0]
10001820:	000c      	movs	r4, r1
10001822:	40c4      	lsrs	r4, r0
10001824:	4222      	tst	r2, r4
10001826:	d014      	beq.n	10001852 <hardware_alarm_irq_handler+0x5e>
10001828:	4a11      	ldr	r2, [pc, #68]	; (10001870 <hardware_alarm_irq_handler+0x7c>)
1000182a:	6a54      	ldr	r4, [r2, #36]	; 0x24
1000182c:	0082      	lsls	r2, r0, #2
1000182e:	4d13      	ldr	r5, [pc, #76]	; (1000187c <hardware_alarm_irq_handler+0x88>)
10001830:	5952      	ldr	r2, [r2, r5]
10001832:	4294      	cmp	r4, r2
10001834:	d306      	bcc.n	10001844 <hardware_alarm_irq_handler+0x50>
10001836:	0082      	lsls	r2, r0, #2
10001838:	4c11      	ldr	r4, [pc, #68]	; (10001880 <hardware_alarm_irq_handler+0x8c>)
1000183a:	5912      	ldr	r2, [r2, r4]
1000183c:	4399      	bics	r1, r3
1000183e:	4b0e      	ldr	r3, [pc, #56]	; (10001878 <hardware_alarm_irq_handler+0x84>)
10001840:	7019      	strb	r1, [r3, #0]
10001842:	e007      	b.n	10001854 <hardware_alarm_irq_handler+0x60>
10001844:	4a0a      	ldr	r2, [pc, #40]	; (10001870 <hardware_alarm_irq_handler+0x7c>)
10001846:	1d03      	adds	r3, r0, #4
10001848:	009b      	lsls	r3, r3, #2
1000184a:	5899      	ldr	r1, [r3, r2]
1000184c:	5099      	str	r1, [r3, r2]
1000184e:	2200      	movs	r2, #0
10001850:	e000      	b.n	10001854 <hardware_alarm_irq_handler+0x60>
10001852:	2200      	movs	r2, #0
10001854:	f3bf 8f5f 	dmb	sy
10001858:	4b04      	ldr	r3, [pc, #16]	; (1000186c <hardware_alarm_irq_handler+0x78>)
1000185a:	2100      	movs	r1, #0
1000185c:	6019      	str	r1, [r3, #0]
1000185e:	f38c 8810 	msr	PRIMASK, ip
10001862:	2a00      	cmp	r2, #0
10001864:	d000      	beq.n	10001868 <hardware_alarm_irq_handler+0x74>
10001866:	4790      	blx	r2
10001868:	bd70      	pop	{r4, r5, r6, pc}
1000186a:	46c0      	nop			; (mov r8, r8)
1000186c:	d0000128 	.word	0xd0000128
10001870:	40054000 	.word	0x40054000
10001874:	4005703c 	.word	0x4005703c
10001878:	20025ee6 	.word	0x20025ee6
1000187c:	200006cc 	.word	0x200006cc
10001880:	2000042c 	.word	0x2000042c

10001884 <hardware_alarm_claim>:
10001884:	b510      	push	{r4, lr}
10001886:	0001      	movs	r1, r0
10001888:	4a02      	ldr	r2, [pc, #8]	; (10001894 <hardware_alarm_claim+0x10>)
1000188a:	4803      	ldr	r0, [pc, #12]	; (10001898 <hardware_alarm_claim+0x14>)
1000188c:	f7fe ff9c 	bl	100007c8 <hw_claim_or_assert>
10001890:	bd10      	pop	{r4, pc}
10001892:	46c0      	nop			; (mov r8, r8)
10001894:	10005610 	.word	0x10005610
10001898:	20025ee4 	.word	0x20025ee4

1000189c <time_us_64>:
1000189c:	4b04      	ldr	r3, [pc, #16]	; (100018b0 <time_us_64+0x14>)
1000189e:	6a5b      	ldr	r3, [r3, #36]	; 0x24
100018a0:	4a03      	ldr	r2, [pc, #12]	; (100018b0 <time_us_64+0x14>)
100018a2:	6a90      	ldr	r0, [r2, #40]	; 0x28
100018a4:	0019      	movs	r1, r3
100018a6:	6a53      	ldr	r3, [r2, #36]	; 0x24
100018a8:	4299      	cmp	r1, r3
100018aa:	d1f9      	bne.n	100018a0 <time_us_64+0x4>
100018ac:	4770      	bx	lr
100018ae:	46c0      	nop			; (mov r8, r8)
100018b0:	40054000 	.word	0x40054000

100018b4 <busy_wait_until>:
100018b4:	4b08      	ldr	r3, [pc, #32]	; (100018d8 <busy_wait_until+0x24>)
100018b6:	6a5b      	ldr	r3, [r3, #36]	; 0x24
100018b8:	e001      	b.n	100018be <busy_wait_until+0xa>
100018ba:	4b07      	ldr	r3, [pc, #28]	; (100018d8 <busy_wait_until+0x24>)
100018bc:	6a5b      	ldr	r3, [r3, #36]	; 0x24
100018be:	428b      	cmp	r3, r1
100018c0:	d3fb      	bcc.n	100018ba <busy_wait_until+0x6>
100018c2:	e001      	b.n	100018c8 <busy_wait_until+0x14>
100018c4:	4b04      	ldr	r3, [pc, #16]	; (100018d8 <busy_wait_until+0x24>)
100018c6:	6a5b      	ldr	r3, [r3, #36]	; 0x24
100018c8:	428b      	cmp	r3, r1
100018ca:	d103      	bne.n	100018d4 <busy_wait_until+0x20>
100018cc:	4b02      	ldr	r3, [pc, #8]	; (100018d8 <busy_wait_until+0x24>)
100018ce:	6a9b      	ldr	r3, [r3, #40]	; 0x28
100018d0:	4283      	cmp	r3, r0
100018d2:	d3f7      	bcc.n	100018c4 <busy_wait_until+0x10>
100018d4:	4770      	bx	lr
100018d6:	46c0      	nop			; (mov r8, r8)
100018d8:	40054000 	.word	0x40054000

100018dc <busy_wait_us>:
100018dc:	b570      	push	{r4, r5, r6, lr}
100018de:	0004      	movs	r4, r0
100018e0:	000d      	movs	r5, r1
100018e2:	f7ff ffdb 	bl	1000189c <time_us_64>
100018e6:	0002      	movs	r2, r0
100018e8:	000b      	movs	r3, r1
100018ea:	0020      	movs	r0, r4
100018ec:	0029      	movs	r1, r5
100018ee:	1880      	adds	r0, r0, r2
100018f0:	4159      	adcs	r1, r3
100018f2:	428b      	cmp	r3, r1
100018f4:	d802      	bhi.n	100018fc <busy_wait_us+0x20>
100018f6:	d104      	bne.n	10001902 <busy_wait_us+0x26>
100018f8:	4282      	cmp	r2, r0
100018fa:	d902      	bls.n	10001902 <busy_wait_us+0x26>
100018fc:	2001      	movs	r0, #1
100018fe:	4240      	negs	r0, r0
10001900:	17c1      	asrs	r1, r0, #31
10001902:	2900      	cmp	r1, #0
10001904:	db02      	blt.n	1000190c <busy_wait_us+0x30>
10001906:	f7ff ffd5 	bl	100018b4 <busy_wait_until>
1000190a:	bd70      	pop	{r4, r5, r6, pc}
1000190c:	4b02      	ldr	r3, [pc, #8]	; (10001918 <busy_wait_us+0x3c>)
1000190e:	4a03      	ldr	r2, [pc, #12]	; (1000191c <busy_wait_us+0x40>)
10001910:	213f      	movs	r1, #63	; 0x3f
10001912:	4803      	ldr	r0, [pc, #12]	; (10001920 <busy_wait_us+0x44>)
10001914:	f000 fd8c 	bl	10002430 <__assert_func>
10001918:	10005204 	.word	0x10005204
1000191c:	100056bc 	.word	0x100056bc
10001920:	10005220 	.word	0x10005220

10001924 <hardware_alarm_set_callback>:
10001924:	b570      	push	{r4, r5, r6, lr}
10001926:	0004      	movs	r4, r0
10001928:	000d      	movs	r5, r1
1000192a:	f3ef 8610 	mrs	r6, PRIMASK
1000192e:	b672      	cpsid	i
10001930:	4b1b      	ldr	r3, [pc, #108]	; (100019a0 <hardware_alarm_set_callback+0x7c>)
10001932:	681b      	ldr	r3, [r3, #0]
10001934:	2b00      	cmp	r3, #0
10001936:	d0fb      	beq.n	10001930 <hardware_alarm_set_callback+0xc>
10001938:	f3bf 8f5f 	dmb	sy
1000193c:	2d00      	cmp	r5, #0
1000193e:	d01c      	beq.n	1000197a <hardware_alarm_set_callback+0x56>
10001940:	0020      	movs	r0, r4
10001942:	f7fe fff5 	bl	10000930 <irq_get_vtable_handler>
10001946:	4b17      	ldr	r3, [pc, #92]	; (100019a4 <hardware_alarm_set_callback+0x80>)
10001948:	4283      	cmp	r3, r0
1000194a:	d00b      	beq.n	10001964 <hardware_alarm_set_callback+0x40>
1000194c:	0019      	movs	r1, r3
1000194e:	0020      	movs	r0, r4
10001950:	f7fe fff6 	bl	10000940 <irq_set_exclusive_handler>
10001954:	2101      	movs	r1, #1
10001956:	0020      	movs	r0, r4
10001958:	f7fe ffe2 	bl	10000920 <irq_set_enabled>
1000195c:	2301      	movs	r3, #1
1000195e:	40a3      	lsls	r3, r4
10001960:	4a11      	ldr	r2, [pc, #68]	; (100019a8 <hardware_alarm_set_callback+0x84>)
10001962:	6013      	str	r3, [r2, #0]
10001964:	00a4      	lsls	r4, r4, #2
10001966:	4b11      	ldr	r3, [pc, #68]	; (100019ac <hardware_alarm_set_callback+0x88>)
10001968:	50e5      	str	r5, [r4, r3]
1000196a:	f3bf 8f5f 	dmb	sy
1000196e:	4b0c      	ldr	r3, [pc, #48]	; (100019a0 <hardware_alarm_set_callback+0x7c>)
10001970:	2200      	movs	r2, #0
10001972:	601a      	str	r2, [r3, #0]
10001974:	f386 8810 	msr	PRIMASK, r6
10001978:	bd70      	pop	{r4, r5, r6, pc}
1000197a:	00a2      	lsls	r2, r4, #2
1000197c:	4b0b      	ldr	r3, [pc, #44]	; (100019ac <hardware_alarm_set_callback+0x88>)
1000197e:	2100      	movs	r1, #0
10001980:	50d1      	str	r1, [r2, r3]
10001982:	2201      	movs	r2, #1
10001984:	40a2      	lsls	r2, r4
10001986:	490a      	ldr	r1, [pc, #40]	; (100019b0 <hardware_alarm_set_callback+0x8c>)
10001988:	780b      	ldrb	r3, [r1, #0]
1000198a:	4393      	bics	r3, r2
1000198c:	700b      	strb	r3, [r1, #0]
1000198e:	4905      	ldr	r1, [pc, #20]	; (100019a4 <hardware_alarm_set_callback+0x80>)
10001990:	0020      	movs	r0, r4
10001992:	f7fe ffff 	bl	10000994 <irq_remove_handler>
10001996:	2100      	movs	r1, #0
10001998:	0020      	movs	r0, r4
1000199a:	f7fe ffc1 	bl	10000920 <irq_set_enabled>
1000199e:	e7e4      	b.n	1000196a <hardware_alarm_set_callback+0x46>
100019a0:	d0000128 	.word	0xd0000128
100019a4:	100017f5 	.word	0x100017f5
100019a8:	40056038 	.word	0x40056038
100019ac:	2000042c 	.word	0x2000042c
100019b0:	20025ee6 	.word	0x20025ee6

100019b4 <hardware_alarm_set_target>:
100019b4:	b5f0      	push	{r4, r5, r6, r7, lr}
100019b6:	46de      	mov	lr, fp
100019b8:	b500      	push	{lr}
100019ba:	b084      	sub	sp, #16
100019bc:	0004      	movs	r4, r0
100019be:	0015      	movs	r5, r2
100019c0:	9201      	str	r2, [sp, #4]
100019c2:	001e      	movs	r6, r3
100019c4:	9302      	str	r3, [sp, #8]
100019c6:	f7ff ff69 	bl	1000189c <time_us_64>
100019ca:	9503      	str	r5, [sp, #12]
100019cc:	428e      	cmp	r6, r1
100019ce:	d802      	bhi.n	100019d6 <hardware_alarm_set_target+0x22>
100019d0:	d14e      	bne.n	10001a70 <hardware_alarm_set_target+0xbc>
100019d2:	4285      	cmp	r5, r0
100019d4:	d94c      	bls.n	10001a70 <hardware_alarm_set_target+0xbc>
100019d6:	f3ef 8b10 	mrs	fp, PRIMASK
100019da:	b672      	cpsid	i
100019dc:	4b27      	ldr	r3, [pc, #156]	; (10001a7c <hardware_alarm_set_target+0xc8>)
100019de:	681b      	ldr	r3, [r3, #0]
100019e0:	2b00      	cmp	r3, #0
100019e2:	d0fb      	beq.n	100019dc <hardware_alarm_set_target+0x28>
100019e4:	f3bf 8f5f 	dmb	sy
100019e8:	4a25      	ldr	r2, [pc, #148]	; (10001a80 <hardware_alarm_set_target+0xcc>)
100019ea:	7817      	ldrb	r7, [r2, #0]
100019ec:	2501      	movs	r5, #1
100019ee:	40a5      	lsls	r5, r4
100019f0:	b2eb      	uxtb	r3, r5
100019f2:	433b      	orrs	r3, r7
100019f4:	7013      	strb	r3, [r2, #0]
100019f6:	4b23      	ldr	r3, [pc, #140]	; (10001a84 <hardware_alarm_set_target+0xd0>)
100019f8:	635d      	str	r5, [r3, #52]	; 0x34
100019fa:	1d22      	adds	r2, r4, #4
100019fc:	0092      	lsls	r2, r2, #2
100019fe:	9901      	ldr	r1, [sp, #4]
10001a00:	50d1      	str	r1, [r2, r3]
10001a02:	00a2      	lsls	r2, r4, #2
10001a04:	4920      	ldr	r1, [pc, #128]	; (10001a88 <hardware_alarm_set_target+0xd4>)
10001a06:	9802      	ldr	r0, [sp, #8]
10001a08:	5050      	str	r0, [r2, r1]
10001a0a:	6a1b      	ldr	r3, [r3, #32]
10001a0c:	422b      	tst	r3, r5
10001a0e:	d112      	bne.n	10001a36 <hardware_alarm_set_target+0x82>
10001a10:	4b1c      	ldr	r3, [pc, #112]	; (10001a84 <hardware_alarm_set_target+0xd0>)
10001a12:	6c1b      	ldr	r3, [r3, #64]	; 0x40
10001a14:	422b      	tst	r3, r5
10001a16:	d008      	beq.n	10001a2a <hardware_alarm_set_target+0x76>
10001a18:	2000      	movs	r0, #0
10001a1a:	f3bf 8f5f 	dmb	sy
10001a1e:	4b17      	ldr	r3, [pc, #92]	; (10001a7c <hardware_alarm_set_target+0xc8>)
10001a20:	2200      	movs	r2, #0
10001a22:	601a      	str	r2, [r3, #0]
10001a24:	f38b 8810 	msr	PRIMASK, fp
10001a28:	e023      	b.n	10001a72 <hardware_alarm_set_target+0xbe>
10001a2a:	4b18      	ldr	r3, [pc, #96]	; (10001a8c <hardware_alarm_set_target+0xd8>)
10001a2c:	4a18      	ldr	r2, [pc, #96]	; (10001a90 <hardware_alarm_set_target+0xdc>)
10001a2e:	21c5      	movs	r1, #197	; 0xc5
10001a30:	4818      	ldr	r0, [pc, #96]	; (10001a94 <hardware_alarm_set_target+0xe0>)
10001a32:	f000 fcfd 	bl	10002430 <__assert_func>
10001a36:	f7ff ff31 	bl	1000189c <time_us_64>
10001a3a:	428e      	cmp	r6, r1
10001a3c:	d814      	bhi.n	10001a68 <hardware_alarm_set_target+0xb4>
10001a3e:	d102      	bne.n	10001a46 <hardware_alarm_set_target+0x92>
10001a40:	9b03      	ldr	r3, [sp, #12]
10001a42:	4283      	cmp	r3, r0
10001a44:	d810      	bhi.n	10001a68 <hardware_alarm_set_target+0xb4>
10001a46:	4b0e      	ldr	r3, [pc, #56]	; (10001a80 <hardware_alarm_set_target+0xcc>)
10001a48:	781b      	ldrb	r3, [r3, #0]
10001a4a:	42bb      	cmp	r3, r7
10001a4c:	d00e      	beq.n	10001a6c <hardware_alarm_set_target+0xb8>
10001a4e:	4b0d      	ldr	r3, [pc, #52]	; (10001a84 <hardware_alarm_set_target+0xd0>)
10001a50:	621d      	str	r5, [r3, #32]
10001a52:	635d      	str	r5, [r3, #52]	; 0x34
10001a54:	201f      	movs	r0, #31
10001a56:	4004      	ands	r4, r0
10001a58:	2301      	movs	r3, #1
10001a5a:	40a3      	lsls	r3, r4
10001a5c:	4a0e      	ldr	r2, [pc, #56]	; (10001a98 <hardware_alarm_set_target+0xe4>)
10001a5e:	6013      	str	r3, [r2, #0]
10001a60:	4b07      	ldr	r3, [pc, #28]	; (10001a80 <hardware_alarm_set_target+0xcc>)
10001a62:	701f      	strb	r7, [r3, #0]
10001a64:	381e      	subs	r0, #30
10001a66:	e7d8      	b.n	10001a1a <hardware_alarm_set_target+0x66>
10001a68:	2000      	movs	r0, #0
10001a6a:	e7d6      	b.n	10001a1a <hardware_alarm_set_target+0x66>
10001a6c:	2001      	movs	r0, #1
10001a6e:	e7d4      	b.n	10001a1a <hardware_alarm_set_target+0x66>
10001a70:	2001      	movs	r0, #1
10001a72:	b004      	add	sp, #16
10001a74:	bc80      	pop	{r7}
10001a76:	46bb      	mov	fp, r7
10001a78:	bdf0      	pop	{r4, r5, r6, r7, pc}
10001a7a:	46c0      	nop			; (mov r8, r8)
10001a7c:	d0000128 	.word	0xd0000128
10001a80:	20025ee6 	.word	0x20025ee6
10001a84:	40054000 	.word	0x40054000
10001a88:	200006cc 	.word	0x200006cc
10001a8c:	10005634 	.word	0x10005634
10001a90:	100056a0 	.word	0x100056a0
10001a94:	10005658 	.word	0x10005658
10001a98:	e000e280 	.word	0xe000e280

10001a9c <hardware_alarm_cancel>:
10001a9c:	f3ef 8c10 	mrs	ip, PRIMASK
10001aa0:	b672      	cpsid	i
10001aa2:	4b0b      	ldr	r3, [pc, #44]	; (10001ad0 <hardware_alarm_cancel+0x34>)
10001aa4:	681b      	ldr	r3, [r3, #0]
10001aa6:	2b00      	cmp	r3, #0
10001aa8:	d0fb      	beq.n	10001aa2 <hardware_alarm_cancel+0x6>
10001aaa:	f3bf 8f5f 	dmb	sy
10001aae:	2301      	movs	r3, #1
10001ab0:	4083      	lsls	r3, r0
10001ab2:	4a08      	ldr	r2, [pc, #32]	; (10001ad4 <hardware_alarm_cancel+0x38>)
10001ab4:	6213      	str	r3, [r2, #32]
10001ab6:	4908      	ldr	r1, [pc, #32]	; (10001ad8 <hardware_alarm_cancel+0x3c>)
10001ab8:	780a      	ldrb	r2, [r1, #0]
10001aba:	439a      	bics	r2, r3
10001abc:	700a      	strb	r2, [r1, #0]
10001abe:	f3bf 8f5f 	dmb	sy
10001ac2:	4b03      	ldr	r3, [pc, #12]	; (10001ad0 <hardware_alarm_cancel+0x34>)
10001ac4:	2200      	movs	r2, #0
10001ac6:	601a      	str	r2, [r3, #0]
10001ac8:	f38c 8810 	msr	PRIMASK, ip
10001acc:	4770      	bx	lr
10001ace:	46c0      	nop			; (mov r8, r8)
10001ad0:	d0000128 	.word	0xd0000128
10001ad4:	40054000 	.word	0x40054000
10001ad8:	20025ee6 	.word	0x20025ee6

10001adc <ph_add_child_node>:
10001adc:	b510      	push	{r4, lr}
10001ade:	2900      	cmp	r1, #0
10001ae0:	d01e      	beq.n	10001b20 <ph_add_child_node+0x44>
10001ae2:	7b03      	ldrb	r3, [r0, #12]
10001ae4:	4299      	cmp	r1, r3
10001ae6:	d81b      	bhi.n	10001b20 <ph_add_child_node+0x44>
10001ae8:	004b      	lsls	r3, r1, #1
10001aea:	185b      	adds	r3, r3, r1
10001aec:	3b03      	subs	r3, #3
10001aee:	6804      	ldr	r4, [r0, #0]
10001af0:	46a4      	mov	ip, r4
10001af2:	4463      	add	r3, ip
10001af4:	2900      	cmp	r1, #0
10001af6:	d019      	beq.n	10001b2c <ph_add_child_node+0x50>
10001af8:	2a00      	cmp	r2, #0
10001afa:	d01d      	beq.n	10001b38 <ph_add_child_node+0x5c>
10001afc:	4291      	cmp	r1, r2
10001afe:	d021      	beq.n	10001b44 <ph_add_child_node+0x68>
10001b00:	2a00      	cmp	r2, #0
10001b02:	d025      	beq.n	10001b50 <ph_add_child_node+0x74>
10001b04:	7b04      	ldrb	r4, [r0, #12]
10001b06:	42a2      	cmp	r2, r4
10001b08:	d822      	bhi.n	10001b50 <ph_add_child_node+0x74>
10001b0a:	6804      	ldr	r4, [r0, #0]
10001b0c:	0050      	lsls	r0, r2, #1
10001b0e:	1880      	adds	r0, r0, r2
10001b10:	3803      	subs	r0, #3
10001b12:	1820      	adds	r0, r4, r0
10001b14:	7081      	strb	r1, [r0, #2]
10001b16:	7819      	ldrb	r1, [r3, #0]
10001b18:	2900      	cmp	r1, #0
10001b1a:	d11f      	bne.n	10001b5c <ph_add_child_node+0x80>
10001b1c:	701a      	strb	r2, [r3, #0]
10001b1e:	bd10      	pop	{r4, pc}
10001b20:	4b10      	ldr	r3, [pc, #64]	; (10001b64 <ph_add_child_node+0x88>)
10001b22:	4a11      	ldr	r2, [pc, #68]	; (10001b68 <ph_add_child_node+0x8c>)
10001b24:	2168      	movs	r1, #104	; 0x68
10001b26:	4811      	ldr	r0, [pc, #68]	; (10001b6c <ph_add_child_node+0x90>)
10001b28:	f000 fc82 	bl	10002430 <__assert_func>
10001b2c:	4b10      	ldr	r3, [pc, #64]	; (10001b70 <ph_add_child_node+0x94>)
10001b2e:	4a11      	ldr	r2, [pc, #68]	; (10001b74 <ph_add_child_node+0x98>)
10001b30:	316f      	adds	r1, #111	; 0x6f
10001b32:	480e      	ldr	r0, [pc, #56]	; (10001b6c <ph_add_child_node+0x90>)
10001b34:	f000 fc7c 	bl	10002430 <__assert_func>
10001b38:	4b0f      	ldr	r3, [pc, #60]	; (10001b78 <ph_add_child_node+0x9c>)
10001b3a:	4a0e      	ldr	r2, [pc, #56]	; (10001b74 <ph_add_child_node+0x98>)
10001b3c:	2170      	movs	r1, #112	; 0x70
10001b3e:	480b      	ldr	r0, [pc, #44]	; (10001b6c <ph_add_child_node+0x90>)
10001b40:	f000 fc76 	bl	10002430 <__assert_func>
10001b44:	4b0d      	ldr	r3, [pc, #52]	; (10001b7c <ph_add_child_node+0xa0>)
10001b46:	4a0b      	ldr	r2, [pc, #44]	; (10001b74 <ph_add_child_node+0x98>)
10001b48:	2171      	movs	r1, #113	; 0x71
10001b4a:	4808      	ldr	r0, [pc, #32]	; (10001b6c <ph_add_child_node+0x90>)
10001b4c:	f000 fc70 	bl	10002430 <__assert_func>
10001b50:	4b04      	ldr	r3, [pc, #16]	; (10001b64 <ph_add_child_node+0x88>)
10001b52:	4a05      	ldr	r2, [pc, #20]	; (10001b68 <ph_add_child_node+0x8c>)
10001b54:	2168      	movs	r1, #104	; 0x68
10001b56:	4805      	ldr	r0, [pc, #20]	; (10001b6c <ph_add_child_node+0x90>)
10001b58:	f000 fc6a 	bl	10002430 <__assert_func>
10001b5c:	7041      	strb	r1, [r0, #1]
10001b5e:	701a      	strb	r2, [r3, #0]
10001b60:	e7dd      	b.n	10001b1e <ph_add_child_node+0x42>
10001b62:	46c0      	nop			; (mov r8, r8)
10001b64:	1000533c 	.word	0x1000533c
10001b68:	100057c4 	.word	0x100057c4
10001b6c:	10005358 	.word	0x10005358
10001b70:	100053a8 	.word	0x100053a8
10001b74:	100057b0 	.word	0x100057b0
10001b78:	100053b4 	.word	0x100053b4
10001b7c:	100053c0 	.word	0x100053c0

10001b80 <ph_merge_nodes>:
10001b80:	b570      	push	{r4, r5, r6, lr}
10001b82:	0006      	movs	r6, r0
10001b84:	000d      	movs	r5, r1
10001b86:	0014      	movs	r4, r2
10001b88:	2900      	cmp	r1, #0
10001b8a:	d014      	beq.n	10001bb6 <ph_merge_nodes+0x36>
10001b8c:	2a00      	cmp	r2, #0
10001b8e:	d014      	beq.n	10001bba <ph_merge_nodes+0x3a>
10001b90:	6880      	ldr	r0, [r0, #8]
10001b92:	6873      	ldr	r3, [r6, #4]
10001b94:	4798      	blx	r3
10001b96:	2800      	cmp	r0, #0
10001b98:	d006      	beq.n	10001ba8 <ph_merge_nodes+0x28>
10001b9a:	0022      	movs	r2, r4
10001b9c:	0029      	movs	r1, r5
10001b9e:	0030      	movs	r0, r6
10001ba0:	f7ff ff9c 	bl	10001adc <ph_add_child_node>
10001ba4:	0028      	movs	r0, r5
10001ba6:	e007      	b.n	10001bb8 <ph_merge_nodes+0x38>
10001ba8:	002a      	movs	r2, r5
10001baa:	0021      	movs	r1, r4
10001bac:	0030      	movs	r0, r6
10001bae:	f7ff ff95 	bl	10001adc <ph_add_child_node>
10001bb2:	0020      	movs	r0, r4
10001bb4:	e000      	b.n	10001bb8 <ph_merge_nodes+0x38>
10001bb6:	0010      	movs	r0, r2
10001bb8:	bd70      	pop	{r4, r5, r6, pc}
10001bba:	0008      	movs	r0, r1
10001bbc:	e7fc      	b.n	10001bb8 <ph_merge_nodes+0x38>
	...

10001bc0 <ph_clear>:
10001bc0:	b510      	push	{r4, lr}
10001bc2:	2300      	movs	r3, #0
10001bc4:	7343      	strb	r3, [r0, #13]
10001bc6:	3301      	adds	r3, #1
10001bc8:	7383      	strb	r3, [r0, #14]
10001bca:	7b03      	ldrb	r3, [r0, #12]
10001bcc:	73c3      	strb	r3, [r0, #15]
10001bce:	2301      	movs	r3, #1
10001bd0:	7b02      	ldrb	r2, [r0, #12]
10001bd2:	429a      	cmp	r2, r3
10001bd4:	d914      	bls.n	10001c00 <ph_clear+0x40>
10001bd6:	2b00      	cmp	r3, #0
10001bd8:	d00c      	beq.n	10001bf4 <ph_clear+0x34>
10001bda:	7b02      	ldrb	r2, [r0, #12]
10001bdc:	4293      	cmp	r3, r2
10001bde:	d809      	bhi.n	10001bf4 <ph_clear+0x34>
10001be0:	005a      	lsls	r2, r3, #1
10001be2:	18d2      	adds	r2, r2, r3
10001be4:	3a03      	subs	r2, #3
10001be6:	6801      	ldr	r1, [r0, #0]
10001be8:	468c      	mov	ip, r1
10001bea:	4462      	add	r2, ip
10001bec:	3301      	adds	r3, #1
10001bee:	b2db      	uxtb	r3, r3
10001bf0:	7053      	strb	r3, [r2, #1]
10001bf2:	e7ed      	b.n	10001bd0 <ph_clear+0x10>
10001bf4:	4b0b      	ldr	r3, [pc, #44]	; (10001c24 <ph_clear+0x64>)
10001bf6:	4a0c      	ldr	r2, [pc, #48]	; (10001c28 <ph_clear+0x68>)
10001bf8:	2168      	movs	r1, #104	; 0x68
10001bfa:	480c      	ldr	r0, [pc, #48]	; (10001c2c <ph_clear+0x6c>)
10001bfc:	f000 fc18 	bl	10002430 <__assert_func>
10001c00:	2a00      	cmp	r2, #0
10001c02:	d009      	beq.n	10001c18 <ph_clear+0x58>
10001c04:	4292      	cmp	r2, r2
10001c06:	d807      	bhi.n	10001c18 <ph_clear+0x58>
10001c08:	6801      	ldr	r1, [r0, #0]
10001c0a:	0053      	lsls	r3, r2, #1
10001c0c:	189a      	adds	r2, r3, r2
10001c0e:	3a03      	subs	r2, #3
10001c10:	188a      	adds	r2, r1, r2
10001c12:	2300      	movs	r3, #0
10001c14:	7053      	strb	r3, [r2, #1]
10001c16:	bd10      	pop	{r4, pc}
10001c18:	4b02      	ldr	r3, [pc, #8]	; (10001c24 <ph_clear+0x64>)
10001c1a:	4a03      	ldr	r2, [pc, #12]	; (10001c28 <ph_clear+0x68>)
10001c1c:	2168      	movs	r1, #104	; 0x68
10001c1e:	4803      	ldr	r0, [pc, #12]	; (10001c2c <ph_clear+0x6c>)
10001c20:	f000 fc06 	bl	10002430 <__assert_func>
10001c24:	1000533c 	.word	0x1000533c
10001c28:	100057c4 	.word	0x100057c4
10001c2c:	10005358 	.word	0x10005358

10001c30 <ph_post_alloc_init>:
10001c30:	b510      	push	{r4, lr}
10001c32:	7301      	strb	r1, [r0, #12]
10001c34:	6042      	str	r2, [r0, #4]
10001c36:	6083      	str	r3, [r0, #8]
10001c38:	f7ff ffc2 	bl	10001bc0 <ph_clear>
10001c3c:	bd10      	pop	{r4, pc}
	...

10001c40 <ph_merge_two_pass>:
10001c40:	b570      	push	{r4, r5, r6, lr}
10001c42:	0004      	movs	r4, r0
10001c44:	1e08      	subs	r0, r1, #0
10001c46:	d100      	bne.n	10001c4a <ph_merge_two_pass+0xa>
10001c48:	bd70      	pop	{r4, r5, r6, pc}
10001c4a:	2900      	cmp	r1, #0
10001c4c:	d034      	beq.n	10001cb8 <ph_merge_two_pass+0x78>
10001c4e:	7b23      	ldrb	r3, [r4, #12]
10001c50:	4299      	cmp	r1, r3
10001c52:	d831      	bhi.n	10001cb8 <ph_merge_two_pass+0x78>
10001c54:	004b      	lsls	r3, r1, #1
10001c56:	185b      	adds	r3, r3, r1
10001c58:	3b03      	subs	r3, #3
10001c5a:	6822      	ldr	r2, [r4, #0]
10001c5c:	4694      	mov	ip, r2
10001c5e:	4463      	add	r3, ip
10001c60:	785a      	ldrb	r2, [r3, #1]
10001c62:	2a00      	cmp	r2, #0
10001c64:	d0f0      	beq.n	10001c48 <ph_merge_two_pass+0x8>
10001c66:	d02d      	beq.n	10001cc4 <ph_merge_two_pass+0x84>
10001c68:	7b23      	ldrb	r3, [r4, #12]
10001c6a:	429a      	cmp	r2, r3
10001c6c:	d82a      	bhi.n	10001cc4 <ph_merge_two_pass+0x84>
10001c6e:	0053      	lsls	r3, r2, #1
10001c70:	189b      	adds	r3, r3, r2
10001c72:	3b03      	subs	r3, #3
10001c74:	6821      	ldr	r1, [r4, #0]
10001c76:	468c      	mov	ip, r1
10001c78:	4463      	add	r3, ip
10001c7a:	785d      	ldrb	r5, [r3, #1]
10001c7c:	2100      	movs	r1, #0
10001c7e:	7059      	strb	r1, [r3, #1]
10001c80:	2800      	cmp	r0, #0
10001c82:	d025      	beq.n	10001cd0 <ph_merge_two_pass+0x90>
10001c84:	7b23      	ldrb	r3, [r4, #12]
10001c86:	4298      	cmp	r0, r3
10001c88:	d822      	bhi.n	10001cd0 <ph_merge_two_pass+0x90>
10001c8a:	0043      	lsls	r3, r0, #1
10001c8c:	181b      	adds	r3, r3, r0
10001c8e:	3b03      	subs	r3, #3
10001c90:	6821      	ldr	r1, [r4, #0]
10001c92:	468c      	mov	ip, r1
10001c94:	4463      	add	r3, ip
10001c96:	2100      	movs	r1, #0
10001c98:	7059      	strb	r1, [r3, #1]
10001c9a:	0001      	movs	r1, r0
10001c9c:	0020      	movs	r0, r4
10001c9e:	f7ff ff6f 	bl	10001b80 <ph_merge_nodes>
10001ca2:	0006      	movs	r6, r0
10001ca4:	0029      	movs	r1, r5
10001ca6:	0020      	movs	r0, r4
10001ca8:	f7ff ffca 	bl	10001c40 <ph_merge_two_pass>
10001cac:	0002      	movs	r2, r0
10001cae:	0031      	movs	r1, r6
10001cb0:	0020      	movs	r0, r4
10001cb2:	f7ff ff65 	bl	10001b80 <ph_merge_nodes>
10001cb6:	e7c7      	b.n	10001c48 <ph_merge_two_pass+0x8>
10001cb8:	4b08      	ldr	r3, [pc, #32]	; (10001cdc <ph_merge_two_pass+0x9c>)
10001cba:	4a09      	ldr	r2, [pc, #36]	; (10001ce0 <ph_merge_two_pass+0xa0>)
10001cbc:	2168      	movs	r1, #104	; 0x68
10001cbe:	4809      	ldr	r0, [pc, #36]	; (10001ce4 <ph_merge_two_pass+0xa4>)
10001cc0:	f000 fbb6 	bl	10002430 <__assert_func>
10001cc4:	4b05      	ldr	r3, [pc, #20]	; (10001cdc <ph_merge_two_pass+0x9c>)
10001cc6:	4a06      	ldr	r2, [pc, #24]	; (10001ce0 <ph_merge_two_pass+0xa0>)
10001cc8:	2168      	movs	r1, #104	; 0x68
10001cca:	4806      	ldr	r0, [pc, #24]	; (10001ce4 <ph_merge_two_pass+0xa4>)
10001ccc:	f000 fbb0 	bl	10002430 <__assert_func>
10001cd0:	4b02      	ldr	r3, [pc, #8]	; (10001cdc <ph_merge_two_pass+0x9c>)
10001cd2:	4a03      	ldr	r2, [pc, #12]	; (10001ce0 <ph_merge_two_pass+0xa0>)
10001cd4:	2168      	movs	r1, #104	; 0x68
10001cd6:	4803      	ldr	r0, [pc, #12]	; (10001ce4 <ph_merge_two_pass+0xa4>)
10001cd8:	f000 fbaa 	bl	10002430 <__assert_func>
10001cdc:	1000533c 	.word	0x1000533c
10001ce0:	100057c4 	.word	0x100057c4
10001ce4:	10005358 	.word	0x10005358

10001ce8 <ph_remove_any_head>:
10001ce8:	b570      	push	{r4, r5, r6, lr}
10001cea:	0005      	movs	r5, r0
10001cec:	000c      	movs	r4, r1
10001cee:	0016      	movs	r6, r2
10001cf0:	2900      	cmp	r1, #0
10001cf2:	d02f      	beq.n	10001d54 <ph_remove_any_head+0x6c>
10001cf4:	d034      	beq.n	10001d60 <ph_remove_any_head+0x78>
10001cf6:	7b03      	ldrb	r3, [r0, #12]
10001cf8:	4299      	cmp	r1, r3
10001cfa:	d831      	bhi.n	10001d60 <ph_remove_any_head+0x78>
10001cfc:	004b      	lsls	r3, r1, #1
10001cfe:	185b      	adds	r3, r3, r1
10001d00:	3b03      	subs	r3, #3
10001d02:	6802      	ldr	r2, [r0, #0]
10001d04:	4694      	mov	ip, r2
10001d06:	4463      	add	r3, ip
10001d08:	785a      	ldrb	r2, [r3, #1]
10001d0a:	2a00      	cmp	r2, #0
10001d0c:	d12e      	bne.n	10001d6c <ph_remove_any_head+0x84>
10001d0e:	789a      	ldrb	r2, [r3, #2]
10001d10:	2a00      	cmp	r2, #0
10001d12:	d131      	bne.n	10001d78 <ph_remove_any_head+0x90>
10001d14:	7819      	ldrb	r1, [r3, #0]
10001d16:	f7ff ff93 	bl	10001c40 <ph_merge_two_pass>
10001d1a:	0003      	movs	r3, r0
10001d1c:	2e00      	cmp	r6, #0
10001d1e:	d00a      	beq.n	10001d36 <ph_remove_any_head+0x4e>
10001d20:	7bea      	ldrb	r2, [r5, #15]
10001d22:	2a00      	cmp	r2, #0
10001d24:	d12e      	bne.n	10001d84 <ph_remove_any_head+0x9c>
10001d26:	7baa      	ldrb	r2, [r5, #14]
10001d28:	2a00      	cmp	r2, #0
10001d2a:	d103      	bne.n	10001d34 <ph_remove_any_head+0x4c>
10001d2c:	7bea      	ldrb	r2, [r5, #15]
10001d2e:	2a00      	cmp	r2, #0
10001d30:	d13b      	bne.n	10001daa <ph_remove_any_head+0xc2>
10001d32:	73ac      	strb	r4, [r5, #14]
10001d34:	73ec      	strb	r4, [r5, #15]
10001d36:	2b00      	cmp	r3, #0
10001d38:	d13d      	bne.n	10001db6 <ph_remove_any_head+0xce>
10001d3a:	2c00      	cmp	r4, #0
10001d3c:	d04f      	beq.n	10001dde <ph_remove_any_head+0xf6>
10001d3e:	7b2b      	ldrb	r3, [r5, #12]
10001d40:	429c      	cmp	r4, r3
10001d42:	d84c      	bhi.n	10001dde <ph_remove_any_head+0xf6>
10001d44:	682b      	ldr	r3, [r5, #0]
10001d46:	0061      	lsls	r1, r4, #1
10001d48:	190c      	adds	r4, r1, r4
10001d4a:	3c03      	subs	r4, #3
10001d4c:	191c      	adds	r4, r3, r4
10001d4e:	2300      	movs	r3, #0
10001d50:	7063      	strb	r3, [r4, #1]
10001d52:	bd70      	pop	{r4, r5, r6, pc}
10001d54:	4b25      	ldr	r3, [pc, #148]	; (10001dec <ph_remove_any_head+0x104>)
10001d56:	4a26      	ldr	r2, [pc, #152]	; (10001df0 <ph_remove_any_head+0x108>)
10001d58:	2138      	movs	r1, #56	; 0x38
10001d5a:	4826      	ldr	r0, [pc, #152]	; (10001df4 <ph_remove_any_head+0x10c>)
10001d5c:	f000 fb68 	bl	10002430 <__assert_func>
10001d60:	4b25      	ldr	r3, [pc, #148]	; (10001df8 <ph_remove_any_head+0x110>)
10001d62:	4a26      	ldr	r2, [pc, #152]	; (10001dfc <ph_remove_any_head+0x114>)
10001d64:	2168      	movs	r1, #104	; 0x68
10001d66:	4826      	ldr	r0, [pc, #152]	; (10001e00 <ph_remove_any_head+0x118>)
10001d68:	f000 fb62 	bl	10002430 <__assert_func>
10001d6c:	4b25      	ldr	r3, [pc, #148]	; (10001e04 <ph_remove_any_head+0x11c>)
10001d6e:	4a20      	ldr	r2, [pc, #128]	; (10001df0 <ph_remove_any_head+0x108>)
10001d70:	213a      	movs	r1, #58	; 0x3a
10001d72:	4820      	ldr	r0, [pc, #128]	; (10001df4 <ph_remove_any_head+0x10c>)
10001d74:	f000 fb5c 	bl	10002430 <__assert_func>
10001d78:	4b23      	ldr	r3, [pc, #140]	; (10001e08 <ph_remove_any_head+0x120>)
10001d7a:	4a1d      	ldr	r2, [pc, #116]	; (10001df0 <ph_remove_any_head+0x108>)
10001d7c:	213b      	movs	r1, #59	; 0x3b
10001d7e:	481d      	ldr	r0, [pc, #116]	; (10001df4 <ph_remove_any_head+0x10c>)
10001d80:	f000 fb56 	bl	10002430 <__assert_func>
10001d84:	2a00      	cmp	r2, #0
10001d86:	d00a      	beq.n	10001d9e <ph_remove_any_head+0xb6>
10001d88:	7b29      	ldrb	r1, [r5, #12]
10001d8a:	428a      	cmp	r2, r1
10001d8c:	d807      	bhi.n	10001d9e <ph_remove_any_head+0xb6>
10001d8e:	0051      	lsls	r1, r2, #1
10001d90:	188a      	adds	r2, r1, r2
10001d92:	3a03      	subs	r2, #3
10001d94:	6829      	ldr	r1, [r5, #0]
10001d96:	468c      	mov	ip, r1
10001d98:	4462      	add	r2, ip
10001d9a:	7054      	strb	r4, [r2, #1]
10001d9c:	e7c3      	b.n	10001d26 <ph_remove_any_head+0x3e>
10001d9e:	4b16      	ldr	r3, [pc, #88]	; (10001df8 <ph_remove_any_head+0x110>)
10001da0:	4a16      	ldr	r2, [pc, #88]	; (10001dfc <ph_remove_any_head+0x114>)
10001da2:	2168      	movs	r1, #104	; 0x68
10001da4:	4816      	ldr	r0, [pc, #88]	; (10001e00 <ph_remove_any_head+0x118>)
10001da6:	f000 fb43 	bl	10002430 <__assert_func>
10001daa:	4b18      	ldr	r3, [pc, #96]	; (10001e0c <ph_remove_any_head+0x124>)
10001dac:	4a10      	ldr	r2, [pc, #64]	; (10001df0 <ph_remove_any_head+0x108>)
10001dae:	2142      	movs	r1, #66	; 0x42
10001db0:	4810      	ldr	r0, [pc, #64]	; (10001df4 <ph_remove_any_head+0x10c>)
10001db2:	f000 fb3d 	bl	10002430 <__assert_func>
10001db6:	2b00      	cmp	r3, #0
10001db8:	d00b      	beq.n	10001dd2 <ph_remove_any_head+0xea>
10001dba:	7b2a      	ldrb	r2, [r5, #12]
10001dbc:	4293      	cmp	r3, r2
10001dbe:	d808      	bhi.n	10001dd2 <ph_remove_any_head+0xea>
10001dc0:	0043      	lsls	r3, r0, #1
10001dc2:	181b      	adds	r3, r3, r0
10001dc4:	3b03      	subs	r3, #3
10001dc6:	682a      	ldr	r2, [r5, #0]
10001dc8:	4694      	mov	ip, r2
10001dca:	4463      	add	r3, ip
10001dcc:	2200      	movs	r2, #0
10001dce:	709a      	strb	r2, [r3, #2]
10001dd0:	e7b3      	b.n	10001d3a <ph_remove_any_head+0x52>
10001dd2:	4b09      	ldr	r3, [pc, #36]	; (10001df8 <ph_remove_any_head+0x110>)
10001dd4:	4a09      	ldr	r2, [pc, #36]	; (10001dfc <ph_remove_any_head+0x114>)
10001dd6:	2168      	movs	r1, #104	; 0x68
10001dd8:	4809      	ldr	r0, [pc, #36]	; (10001e00 <ph_remove_any_head+0x118>)
10001dda:	f000 fb29 	bl	10002430 <__assert_func>
10001dde:	4b06      	ldr	r3, [pc, #24]	; (10001df8 <ph_remove_any_head+0x110>)
10001de0:	4a06      	ldr	r2, [pc, #24]	; (10001dfc <ph_remove_any_head+0x114>)
10001de2:	2168      	movs	r1, #104	; 0x68
10001de4:	4806      	ldr	r0, [pc, #24]	; (10001e00 <ph_remove_any_head+0x118>)
10001de6:	f000 fb23 	bl	10002430 <__assert_func>
10001dea:	46c0      	nop			; (mov r8, r8)
10001dec:	100056d4 	.word	0x100056d4
10001df0:	1000579c 	.word	0x1000579c
10001df4:	100056dc 	.word	0x100056dc
10001df8:	1000533c 	.word	0x1000533c
10001dfc:	100057c4 	.word	0x100057c4
10001e00:	10005358 	.word	0x10005358
10001e04:	10005718 	.word	0x10005718
10001e08:	10005740 	.word	0x10005740
10001e0c:	10005484 	.word	0x10005484

10001e10 <ph_remove_head>:
10001e10:	b570      	push	{r4, r5, r6, lr}
10001e12:	0004      	movs	r4, r0
10001e14:	000a      	movs	r2, r1
10001e16:	7b45      	ldrb	r5, [r0, #13]
10001e18:	0029      	movs	r1, r5
10001e1a:	f7ff ff65 	bl	10001ce8 <ph_remove_any_head>
10001e1e:	7360      	strb	r0, [r4, #13]
10001e20:	0028      	movs	r0, r5
10001e22:	bd70      	pop	{r4, r5, r6, pc}

10001e24 <ph_remove_and_free_node>:
10001e24:	b570      	push	{r4, r5, r6, lr}
10001e26:	0004      	movs	r4, r0
10001e28:	2900      	cmp	r1, #0
10001e2a:	d067      	beq.n	10001efc <ph_remove_and_free_node+0xd8>
10001e2c:	7b43      	ldrb	r3, [r0, #13]
10001e2e:	428b      	cmp	r3, r1
10001e30:	d00e      	beq.n	10001e50 <ph_remove_and_free_node+0x2c>
10001e32:	2900      	cmp	r1, #0
10001e34:	d011      	beq.n	10001e5a <ph_remove_and_free_node+0x36>
10001e36:	7b03      	ldrb	r3, [r0, #12]
10001e38:	4299      	cmp	r1, r3
10001e3a:	d80e      	bhi.n	10001e5a <ph_remove_and_free_node+0x36>
10001e3c:	004b      	lsls	r3, r1, #1
10001e3e:	185b      	adds	r3, r3, r1
10001e40:	3b03      	subs	r3, #3
10001e42:	6802      	ldr	r2, [r0, #0]
10001e44:	18d0      	adds	r0, r2, r3
10001e46:	7883      	ldrb	r3, [r0, #2]
10001e48:	2b00      	cmp	r3, #0
10001e4a:	d10c      	bne.n	10001e66 <ph_remove_and_free_node+0x42>
10001e4c:	2000      	movs	r0, #0
10001e4e:	e056      	b.n	10001efe <ph_remove_and_free_node+0xda>
10001e50:	2101      	movs	r1, #1
10001e52:	f7ff ffdd 	bl	10001e10 <ph_remove_head>
10001e56:	2001      	movs	r0, #1
10001e58:	e051      	b.n	10001efe <ph_remove_and_free_node+0xda>
10001e5a:	4b29      	ldr	r3, [pc, #164]	; (10001f00 <ph_remove_and_free_node+0xdc>)
10001e5c:	4a29      	ldr	r2, [pc, #164]	; (10001f04 <ph_remove_and_free_node+0xe0>)
10001e5e:	2168      	movs	r1, #104	; 0x68
10001e60:	4829      	ldr	r0, [pc, #164]	; (10001f08 <ph_remove_and_free_node+0xe4>)
10001e62:	f000 fae5 	bl	10002430 <__assert_func>
10001e66:	2b00      	cmp	r3, #0
10001e68:	d020      	beq.n	10001eac <ph_remove_and_free_node+0x88>
10001e6a:	7b22      	ldrb	r2, [r4, #12]
10001e6c:	4293      	cmp	r3, r2
10001e6e:	d81d      	bhi.n	10001eac <ph_remove_and_free_node+0x88>
10001e70:	005a      	lsls	r2, r3, #1
10001e72:	18d3      	adds	r3, r2, r3
10001e74:	3b03      	subs	r3, #3
10001e76:	6822      	ldr	r2, [r4, #0]
10001e78:	18d2      	adds	r2, r2, r3
10001e7a:	6825      	ldr	r5, [r4, #0]
10001e7c:	5ceb      	ldrb	r3, [r5, r3]
10001e7e:	428b      	cmp	r3, r1
10001e80:	d01a      	beq.n	10001eb8 <ph_remove_and_free_node+0x94>
10001e82:	2b00      	cmp	r3, #0
10001e84:	d01b      	beq.n	10001ebe <ph_remove_and_free_node+0x9a>
10001e86:	7b22      	ldrb	r2, [r4, #12]
10001e88:	4293      	cmp	r3, r2
10001e8a:	d818      	bhi.n	10001ebe <ph_remove_and_free_node+0x9a>
10001e8c:	005a      	lsls	r2, r3, #1
10001e8e:	18d3      	adds	r3, r2, r3
10001e90:	3b03      	subs	r3, #3
10001e92:	6822      	ldr	r2, [r4, #0]
10001e94:	18d2      	adds	r2, r2, r3
10001e96:	7853      	ldrb	r3, [r2, #1]
10001e98:	428b      	cmp	r3, r1
10001e9a:	d016      	beq.n	10001eca <ph_remove_and_free_node+0xa6>
10001e9c:	2b00      	cmp	r3, #0
10001e9e:	d1f0      	bne.n	10001e82 <ph_remove_and_free_node+0x5e>
10001ea0:	4b1a      	ldr	r3, [pc, #104]	; (10001f0c <ph_remove_and_free_node+0xe8>)
10001ea2:	4a1b      	ldr	r2, [pc, #108]	; (10001f10 <ph_remove_and_free_node+0xec>)
10001ea4:	216b      	movs	r1, #107	; 0x6b
10001ea6:	481b      	ldr	r0, [pc, #108]	; (10001f14 <ph_remove_and_free_node+0xf0>)
10001ea8:	f000 fac2 	bl	10002430 <__assert_func>
10001eac:	4b14      	ldr	r3, [pc, #80]	; (10001f00 <ph_remove_and_free_node+0xdc>)
10001eae:	4a15      	ldr	r2, [pc, #84]	; (10001f04 <ph_remove_and_free_node+0xe0>)
10001eb0:	2168      	movs	r1, #104	; 0x68
10001eb2:	4815      	ldr	r0, [pc, #84]	; (10001f08 <ph_remove_and_free_node+0xe4>)
10001eb4:	f000 fabc 	bl	10002430 <__assert_func>
10001eb8:	7843      	ldrb	r3, [r0, #1]
10001eba:	7013      	strb	r3, [r2, #0]
10001ebc:	e007      	b.n	10001ece <ph_remove_and_free_node+0xaa>
10001ebe:	4b10      	ldr	r3, [pc, #64]	; (10001f00 <ph_remove_and_free_node+0xdc>)
10001ec0:	4a10      	ldr	r2, [pc, #64]	; (10001f04 <ph_remove_and_free_node+0xe0>)
10001ec2:	2168      	movs	r1, #104	; 0x68
10001ec4:	4810      	ldr	r0, [pc, #64]	; (10001f08 <ph_remove_and_free_node+0xe4>)
10001ec6:	f000 fab3 	bl	10002430 <__assert_func>
10001eca:	7843      	ldrb	r3, [r0, #1]
10001ecc:	7053      	strb	r3, [r2, #1]
10001ece:	2300      	movs	r3, #0
10001ed0:	7083      	strb	r3, [r0, #2]
10001ed2:	7043      	strb	r3, [r0, #1]
10001ed4:	2201      	movs	r2, #1
10001ed6:	0020      	movs	r0, r4
10001ed8:	f7ff ff06 	bl	10001ce8 <ph_remove_any_head>
10001edc:	0002      	movs	r2, r0
10001ede:	7b61      	ldrb	r1, [r4, #13]
10001ee0:	4281      	cmp	r1, r0
10001ee2:	d005      	beq.n	10001ef0 <ph_remove_and_free_node+0xcc>
10001ee4:	0020      	movs	r0, r4
10001ee6:	f7ff fe4b 	bl	10001b80 <ph_merge_nodes>
10001eea:	7360      	strb	r0, [r4, #13]
10001eec:	2001      	movs	r0, #1
10001eee:	e006      	b.n	10001efe <ph_remove_and_free_node+0xda>
10001ef0:	4b09      	ldr	r3, [pc, #36]	; (10001f18 <ph_remove_and_free_node+0xf4>)
10001ef2:	4a07      	ldr	r2, [pc, #28]	; (10001f10 <ph_remove_and_free_node+0xec>)
10001ef4:	2171      	movs	r1, #113	; 0x71
10001ef6:	4807      	ldr	r0, [pc, #28]	; (10001f14 <ph_remove_and_free_node+0xf0>)
10001ef8:	f000 fa9a 	bl	10002430 <__assert_func>
10001efc:	2000      	movs	r0, #0
10001efe:	bd70      	pop	{r4, r5, r6, pc}
10001f00:	1000533c 	.word	0x1000533c
10001f04:	100057c4 	.word	0x100057c4
10001f08:	10005358 	.word	0x10005358
10001f0c:	10005124 	.word	0x10005124
10001f10:	10005784 	.word	0x10005784
10001f14:	100056dc 	.word	0x100056dc
10001f18:	10005764 	.word	0x10005764

10001f1c <uart_disable_before_lcr_write>:
10001f1c:	b570      	push	{r4, r5, r6, lr}
10001f1e:	6b04      	ldr	r4, [r0, #48]	; 0x30
10001f20:	07e3      	lsls	r3, r4, #31
10001f22:	d401      	bmi.n	10001f28 <uart_disable_before_lcr_write+0xc>
10001f24:	0020      	movs	r0, r4
10001f26:	bd70      	pop	{r4, r5, r6, pc}
10001f28:	0002      	movs	r2, r0
10001f2a:	3230      	adds	r2, #48	; 0x30
10001f2c:	23c0      	movs	r3, #192	; 0xc0
10001f2e:	019b      	lsls	r3, r3, #6
10001f30:	4313      	orrs	r3, r2
10001f32:	4a0a      	ldr	r2, [pc, #40]	; (10001f5c <uart_disable_before_lcr_write+0x40>)
10001f34:	601a      	str	r2, [r3, #0]
10001f36:	6a45      	ldr	r5, [r0, #36]	; 0x24
10001f38:	6a82      	ldr	r2, [r0, #40]	; 0x28
10001f3a:	01ad      	lsls	r5, r5, #6
10001f3c:	18ad      	adds	r5, r5, r2
10001f3e:	02ad      	lsls	r5, r5, #10
10001f40:	2006      	movs	r0, #6
10001f42:	f000 f9bd 	bl	100022c0 <clock_get_hz>
10001f46:	4906      	ldr	r1, [pc, #24]	; (10001f60 <uart_disable_before_lcr_write+0x44>)
10001f48:	f001 fc20 	bl	1000378c <__wrap___aeabi_uidiv>
10001f4c:	0001      	movs	r1, r0
10001f4e:	0028      	movs	r0, r5
10001f50:	f001 fc1c 	bl	1000378c <__wrap___aeabi_uidiv>
10001f54:	2100      	movs	r1, #0
10001f56:	f7ff fcc1 	bl	100018dc <busy_wait_us>
10001f5a:	e7e3      	b.n	10001f24 <uart_disable_before_lcr_write+0x8>
10001f5c:	00000301 	.word	0x00000301
10001f60:	00000e4e 	.word	0x00000e4e

10001f64 <uart_write_lcr_bits_masked>:
10001f64:	b570      	push	{r4, r5, r6, lr}
10001f66:	0004      	movs	r4, r0
10001f68:	000e      	movs	r6, r1
10001f6a:	0015      	movs	r5, r2
10001f6c:	f7ff ffd6 	bl	10001f1c <uart_disable_before_lcr_write>
10001f70:	0022      	movs	r2, r4
10001f72:	322c      	adds	r2, #44	; 0x2c
10001f74:	6ae1      	ldr	r1, [r4, #44]	; 0x2c
10001f76:	404e      	eors	r6, r1
10001f78:	4035      	ands	r5, r6
10001f7a:	2380      	movs	r3, #128	; 0x80
10001f7c:	015b      	lsls	r3, r3, #5
10001f7e:	4313      	orrs	r3, r2
10001f80:	601d      	str	r5, [r3, #0]
10001f82:	6320      	str	r0, [r4, #48]	; 0x30
10001f84:	bd70      	pop	{r4, r5, r6, pc}
	...

10001f88 <uart_set_baudrate>:
10001f88:	b570      	push	{r4, r5, r6, lr}
10001f8a:	0005      	movs	r5, r0
10001f8c:	000c      	movs	r4, r1
10001f8e:	2006      	movs	r0, #6
10001f90:	f000 f996 	bl	100022c0 <clock_get_hz>
10001f94:	00c0      	lsls	r0, r0, #3
10001f96:	0021      	movs	r1, r4
10001f98:	f001 fbf8 	bl	1000378c <__wrap___aeabi_uidiv>
10001f9c:	09c6      	lsrs	r6, r0, #7
10001f9e:	d008      	beq.n	10001fb2 <uart_set_baudrate+0x2a>
10001fa0:	4b0e      	ldr	r3, [pc, #56]	; (10001fdc <uart_set_baudrate+0x54>)
10001fa2:	429e      	cmp	r6, r3
10001fa4:	d816      	bhi.n	10001fd4 <uart_set_baudrate+0x4c>
10001fa6:	237f      	movs	r3, #127	; 0x7f
10001fa8:	4018      	ands	r0, r3
10001faa:	3001      	adds	r0, #1
10001fac:	0034      	movs	r4, r6
10001fae:	0846      	lsrs	r6, r0, #1
10001fb0:	e000      	b.n	10001fb4 <uart_set_baudrate+0x2c>
10001fb2:	2401      	movs	r4, #1
10001fb4:	626c      	str	r4, [r5, #36]	; 0x24
10001fb6:	62ae      	str	r6, [r5, #40]	; 0x28
10001fb8:	2200      	movs	r2, #0
10001fba:	2100      	movs	r1, #0
10001fbc:	0028      	movs	r0, r5
10001fbe:	f7ff ffd1 	bl	10001f64 <uart_write_lcr_bits_masked>
10001fc2:	2006      	movs	r0, #6
10001fc4:	f000 f97c 	bl	100022c0 <clock_get_hz>
10001fc8:	0080      	lsls	r0, r0, #2
10001fca:	01a1      	lsls	r1, r4, #6
10001fcc:	1989      	adds	r1, r1, r6
10001fce:	f001 fbdd 	bl	1000378c <__wrap___aeabi_uidiv>
10001fd2:	bd70      	pop	{r4, r5, r6, pc}
10001fd4:	2600      	movs	r6, #0
10001fd6:	4c02      	ldr	r4, [pc, #8]	; (10001fe0 <uart_set_baudrate+0x58>)
10001fd8:	e7ec      	b.n	10001fb4 <uart_set_baudrate+0x2c>
10001fda:	46c0      	nop			; (mov r8, r8)
10001fdc:	0000fffe 	.word	0x0000fffe
10001fe0:	0000ffff 	.word	0x0000ffff

10001fe4 <uart_set_format>:
10001fe4:	b510      	push	{r4, lr}
10001fe6:	3905      	subs	r1, #5
10001fe8:	0149      	lsls	r1, r1, #5
10001fea:	3a01      	subs	r2, #1
10001fec:	00d2      	lsls	r2, r2, #3
10001fee:	4311      	orrs	r1, r2
10001ff0:	2b00      	cmp	r3, #0
10001ff2:	d009      	beq.n	10002008 <uart_set_format+0x24>
10001ff4:	2202      	movs	r2, #2
10001ff6:	430a      	orrs	r2, r1
10001ff8:	2b01      	cmp	r3, #1
10001ffa:	d007      	beq.n	1000200c <uart_set_format+0x28>
10001ffc:	2100      	movs	r1, #0
10001ffe:	4311      	orrs	r1, r2
10002000:	226e      	movs	r2, #110	; 0x6e
10002002:	f7ff ffaf 	bl	10001f64 <uart_write_lcr_bits_masked>
10002006:	bd10      	pop	{r4, pc}
10002008:	2200      	movs	r2, #0
1000200a:	e7f4      	b.n	10001ff6 <uart_set_format+0x12>
1000200c:	2104      	movs	r1, #4
1000200e:	e7f6      	b.n	10001ffe <uart_set_format+0x1a>

10002010 <uart_set_translate_crlf>:
10002010:	2900      	cmp	r1, #0
10002012:	d009      	beq.n	10002028 <uart_set_translate_crlf+0x18>
10002014:	220a      	movs	r2, #10
10002016:	4b06      	ldr	r3, [pc, #24]	; (10002030 <uart_set_translate_crlf+0x20>)
10002018:	469c      	mov	ip, r3
1000201a:	4460      	add	r0, ip
1000201c:	4243      	negs	r3, r0
1000201e:	4158      	adcs	r0, r3
10002020:	0040      	lsls	r0, r0, #1
10002022:	4b04      	ldr	r3, [pc, #16]	; (10002034 <uart_set_translate_crlf+0x24>)
10002024:	52c2      	strh	r2, [r0, r3]
10002026:	4770      	bx	lr
10002028:	2280      	movs	r2, #128	; 0x80
1000202a:	0052      	lsls	r2, r2, #1
1000202c:	e7f3      	b.n	10002016 <uart_set_translate_crlf+0x6>
1000202e:	46c0      	nop			; (mov r8, r8)
10002030:	bffc8000 	.word	0xbffc8000
10002034:	200006dc 	.word	0x200006dc

10002038 <uart_init>:
10002038:	b570      	push	{r4, r5, r6, lr}
1000203a:	0005      	movs	r5, r0
1000203c:	000c      	movs	r4, r1
1000203e:	2006      	movs	r0, #6
10002040:	f000 f93e 	bl	100022c0 <clock_get_hz>
10002044:	1e06      	subs	r6, r0, #0
10002046:	d027      	beq.n	10002098 <uart_init+0x60>
10002048:	4b16      	ldr	r3, [pc, #88]	; (100020a4 <uart_init+0x6c>)
1000204a:	429d      	cmp	r5, r3
1000204c:	d026      	beq.n	1000209c <uart_init+0x64>
1000204e:	2280      	movs	r2, #128	; 0x80
10002050:	03d2      	lsls	r2, r2, #15
10002052:	4b15      	ldr	r3, [pc, #84]	; (100020a8 <uart_init+0x70>)
10002054:	601a      	str	r2, [r3, #0]
10002056:	4b15      	ldr	r3, [pc, #84]	; (100020ac <uart_init+0x74>)
10002058:	601a      	str	r2, [r3, #0]
1000205a:	4b15      	ldr	r3, [pc, #84]	; (100020b0 <uart_init+0x78>)
1000205c:	689b      	ldr	r3, [r3, #8]
1000205e:	0011      	movs	r1, r2
10002060:	4399      	bics	r1, r3
10002062:	d1fa      	bne.n	1000205a <uart_init+0x22>
10002064:	2100      	movs	r1, #0
10002066:	0028      	movs	r0, r5
10002068:	f7ff ffd2 	bl	10002010 <uart_set_translate_crlf>
1000206c:	0021      	movs	r1, r4
1000206e:	0028      	movs	r0, r5
10002070:	f7ff ff8a 	bl	10001f88 <uart_set_baudrate>
10002074:	0006      	movs	r6, r0
10002076:	2300      	movs	r3, #0
10002078:	2201      	movs	r2, #1
1000207a:	2108      	movs	r1, #8
1000207c:	0028      	movs	r0, r5
1000207e:	f7ff ffb1 	bl	10001fe4 <uart_set_format>
10002082:	002a      	movs	r2, r5
10002084:	322c      	adds	r2, #44	; 0x2c
10002086:	2380      	movs	r3, #128	; 0x80
10002088:	019b      	lsls	r3, r3, #6
1000208a:	4313      	orrs	r3, r2
1000208c:	2210      	movs	r2, #16
1000208e:	601a      	str	r2, [r3, #0]
10002090:	4b08      	ldr	r3, [pc, #32]	; (100020b4 <uart_init+0x7c>)
10002092:	632b      	str	r3, [r5, #48]	; 0x30
10002094:	2303      	movs	r3, #3
10002096:	64ab      	str	r3, [r5, #72]	; 0x48
10002098:	0030      	movs	r0, r6
1000209a:	bd70      	pop	{r4, r5, r6, pc}
1000209c:	2280      	movs	r2, #128	; 0x80
1000209e:	0412      	lsls	r2, r2, #16
100020a0:	e7d7      	b.n	10002052 <uart_init+0x1a>
100020a2:	46c0      	nop			; (mov r8, r8)
100020a4:	40038000 	.word	0x40038000
100020a8:	4000e000 	.word	0x4000e000
100020ac:	4000f000 	.word	0x4000f000
100020b0:	4000c000 	.word	0x4000c000
100020b4:	00000301 	.word	0x00000301

100020b8 <clock_configure>:
100020b8:	b5f8      	push	{r3, r4, r5, r6, r7, lr}
100020ba:	46de      	mov	lr, fp
100020bc:	4657      	mov	r7, sl
100020be:	464e      	mov	r6, r9
100020c0:	4645      	mov	r5, r8
100020c2:	b5e0      	push	{r5, r6, r7, lr}
100020c4:	0005      	movs	r5, r0
100020c6:	000f      	movs	r7, r1
100020c8:	4692      	mov	sl, r2
100020ca:	9a0a      	ldr	r2, [sp, #40]	; 0x28
100020cc:	4293      	cmp	r3, r2
100020ce:	d350      	bcc.n	10002172 <clock_configure+0xba>
100020d0:	0e1a      	lsrs	r2, r3, #24
100020d2:	4691      	mov	r9, r2
100020d4:	021e      	lsls	r6, r3, #8
100020d6:	9a0a      	ldr	r2, [sp, #40]	; 0x28
100020d8:	2300      	movs	r3, #0
100020da:	0030      	movs	r0, r6
100020dc:	4649      	mov	r1, r9
100020de:	f001 fb93 	bl	10003808 <__wrap___aeabi_uldivmod>
100020e2:	4680      	mov	r8, r0
100020e4:	006c      	lsls	r4, r5, #1
100020e6:	1964      	adds	r4, r4, r5
100020e8:	00a4      	lsls	r4, r4, #2
100020ea:	4b30      	ldr	r3, [pc, #192]	; (100021ac <clock_configure+0xf4>)
100020ec:	469c      	mov	ip, r3
100020ee:	4464      	add	r4, ip
100020f0:	6863      	ldr	r3, [r4, #4]
100020f2:	4283      	cmp	r3, r0
100020f4:	d200      	bcs.n	100020f8 <clock_configure+0x40>
100020f6:	6060      	str	r0, [r4, #4]
100020f8:	1f2b      	subs	r3, r5, #4
100020fa:	b2db      	uxtb	r3, r3
100020fc:	469b      	mov	fp, r3
100020fe:	2b01      	cmp	r3, #1
10002100:	d93d      	bls.n	1000217e <clock_configure+0xc6>
10002102:	23c0      	movs	r3, #192	; 0xc0
10002104:	019b      	lsls	r3, r3, #6
10002106:	4323      	orrs	r3, r4
10002108:	2280      	movs	r2, #128	; 0x80
1000210a:	0112      	lsls	r2, r2, #4
1000210c:	601a      	str	r2, [r3, #0]
1000210e:	00ab      	lsls	r3, r5, #2
10002110:	4a27      	ldr	r2, [pc, #156]	; (100021b0 <clock_configure+0xf8>)
10002112:	5899      	ldr	r1, [r3, r2]
10002114:	2900      	cmp	r1, #0
10002116:	d007      	beq.n	10002128 <clock_configure+0x70>
10002118:	6950      	ldr	r0, [r2, #20]
1000211a:	f001 fb37 	bl	1000378c <__wrap___aeabi_uidiv>
1000211e:	1c43      	adds	r3, r0, #1
10002120:	0058      	lsls	r0, r3, #1
10002122:	18c0      	adds	r0, r0, r3
10002124:	3803      	subs	r0, #3
10002126:	d2fd      	bcs.n	10002124 <clock_configure+0x6c>
10002128:	4653      	mov	r3, sl
1000212a:	015a      	lsls	r2, r3, #5
1000212c:	6823      	ldr	r3, [r4, #0]
1000212e:	405a      	eors	r2, r3
10002130:	23e0      	movs	r3, #224	; 0xe0
10002132:	401a      	ands	r2, r3
10002134:	2380      	movs	r3, #128	; 0x80
10002136:	015b      	lsls	r3, r3, #5
10002138:	4323      	orrs	r3, r4
1000213a:	601a      	str	r2, [r3, #0]
1000213c:	465a      	mov	r2, fp
1000213e:	2a01      	cmp	r2, #1
10002140:	d928      	bls.n	10002194 <clock_configure+0xdc>
10002142:	2380      	movs	r3, #128	; 0x80
10002144:	019b      	lsls	r3, r3, #6
10002146:	4323      	orrs	r3, r4
10002148:	2280      	movs	r2, #128	; 0x80
1000214a:	0112      	lsls	r2, r2, #4
1000214c:	601a      	str	r2, [r3, #0]
1000214e:	4643      	mov	r3, r8
10002150:	6063      	str	r3, [r4, #4]
10002152:	4642      	mov	r2, r8
10002154:	2300      	movs	r3, #0
10002156:	0030      	movs	r0, r6
10002158:	4649      	mov	r1, r9
1000215a:	f001 fb55 	bl	10003808 <__wrap___aeabi_uldivmod>
1000215e:	00ad      	lsls	r5, r5, #2
10002160:	4b13      	ldr	r3, [pc, #76]	; (100021b0 <clock_configure+0xf8>)
10002162:	5158      	str	r0, [r3, r5]
10002164:	2001      	movs	r0, #1
10002166:	bcf0      	pop	{r4, r5, r6, r7}
10002168:	46bb      	mov	fp, r7
1000216a:	46b2      	mov	sl, r6
1000216c:	46a9      	mov	r9, r5
1000216e:	46a0      	mov	r8, r4
10002170:	bdf8      	pop	{r3, r4, r5, r6, r7, pc}
10002172:	4b10      	ldr	r3, [pc, #64]	; (100021b4 <clock_configure+0xfc>)
10002174:	4a10      	ldr	r2, [pc, #64]	; (100021b8 <clock_configure+0x100>)
10002176:	2133      	movs	r1, #51	; 0x33
10002178:	4810      	ldr	r0, [pc, #64]	; (100021bc <clock_configure+0x104>)
1000217a:	f000 f959 	bl	10002430 <__assert_func>
1000217e:	2f01      	cmp	r7, #1
10002180:	d1bf      	bne.n	10002102 <clock_configure+0x4a>
10002182:	23c0      	movs	r3, #192	; 0xc0
10002184:	019b      	lsls	r3, r3, #6
10002186:	4323      	orrs	r3, r4
10002188:	2203      	movs	r2, #3
1000218a:	601a      	str	r2, [r3, #0]
1000218c:	68a3      	ldr	r3, [r4, #8]
1000218e:	07db      	lsls	r3, r3, #31
10002190:	d5fc      	bpl.n	1000218c <clock_configure+0xd4>
10002192:	e7c9      	b.n	10002128 <clock_configure+0x70>
10002194:	6821      	ldr	r1, [r4, #0]
10002196:	4079      	eors	r1, r7
10002198:	2203      	movs	r2, #3
1000219a:	400a      	ands	r2, r1
1000219c:	601a      	str	r2, [r3, #0]
1000219e:	68a2      	ldr	r2, [r4, #8]
100021a0:	2301      	movs	r3, #1
100021a2:	40bb      	lsls	r3, r7
100021a4:	4213      	tst	r3, r2
100021a6:	d0fa      	beq.n	1000219e <clock_configure+0xe6>
100021a8:	e7cb      	b.n	10002142 <clock_configure+0x8a>
100021aa:	46c0      	nop			; (mov r8, r8)
100021ac:	40008000 	.word	0x40008000
100021b0:	20000444 	.word	0x20000444
100021b4:	100057d0 	.word	0x100057d0
100021b8:	1000582c 	.word	0x1000582c
100021bc:	100057e4 	.word	0x100057e4

100021c0 <clocks_init>:
100021c0:	b530      	push	{r4, r5, lr}
100021c2:	b083      	sub	sp, #12
100021c4:	200c      	movs	r0, #12
100021c6:	f000 f911 	bl	100023ec <watchdog_start_tick>
100021ca:	f7fe fadd 	bl	10000788 <running_on_fpga>
100021ce:	2800      	cmp	r0, #0
100021d0:	d00d      	beq.n	100021ee <clocks_init+0x2e>
100021d2:	2300      	movs	r3, #0
100021d4:	e004      	b.n	100021e0 <clocks_init+0x20>
100021d6:	0099      	lsls	r1, r3, #2
100021d8:	4a2d      	ldr	r2, [pc, #180]	; (10002290 <clocks_init+0xd0>)
100021da:	482e      	ldr	r0, [pc, #184]	; (10002294 <clocks_init+0xd4>)
100021dc:	5088      	str	r0, [r1, r2]
100021de:	3301      	adds	r3, #1
100021e0:	2b09      	cmp	r3, #9
100021e2:	d9f8      	bls.n	100021d6 <clocks_init+0x16>
100021e4:	4b2a      	ldr	r3, [pc, #168]	; (10002290 <clocks_init+0xd0>)
100021e6:	4a2c      	ldr	r2, [pc, #176]	; (10002298 <clocks_init+0xd8>)
100021e8:	625a      	str	r2, [r3, #36]	; 0x24
100021ea:	b003      	add	sp, #12
100021ec:	bd30      	pop	{r4, r5, pc}
100021ee:	4b2b      	ldr	r3, [pc, #172]	; (1000229c <clocks_init+0xdc>)
100021f0:	2200      	movs	r2, #0
100021f2:	679a      	str	r2, [r3, #120]	; 0x78
100021f4:	f000 f902 	bl	100023fc <xosc_init>
100021f8:	4b29      	ldr	r3, [pc, #164]	; (100022a0 <clocks_init+0xe0>)
100021fa:	2201      	movs	r2, #1
100021fc:	601a      	str	r2, [r3, #0]
100021fe:	4b27      	ldr	r3, [pc, #156]	; (1000229c <clocks_init+0xdc>)
10002200:	6c5b      	ldr	r3, [r3, #68]	; 0x44
10002202:	2b01      	cmp	r3, #1
10002204:	d1fb      	bne.n	100021fe <clocks_init+0x3e>
10002206:	4b27      	ldr	r3, [pc, #156]	; (100022a4 <clocks_init+0xe4>)
10002208:	2203      	movs	r2, #3
1000220a:	601a      	str	r2, [r3, #0]
1000220c:	4b23      	ldr	r3, [pc, #140]	; (1000229c <clocks_init+0xdc>)
1000220e:	6b9b      	ldr	r3, [r3, #56]	; 0x38
10002210:	2b01      	cmp	r3, #1
10002212:	d1fb      	bne.n	1000220c <clocks_init+0x4c>
10002214:	3301      	adds	r3, #1
10002216:	9300      	str	r3, [sp, #0]
10002218:	3304      	adds	r3, #4
1000221a:	4a23      	ldr	r2, [pc, #140]	; (100022a8 <clocks_init+0xe8>)
1000221c:	2101      	movs	r1, #1
1000221e:	4823      	ldr	r0, [pc, #140]	; (100022ac <clocks_init+0xec>)
10002220:	f000 f854 	bl	100022cc <pll_init>
10002224:	2305      	movs	r3, #5
10002226:	9300      	str	r3, [sp, #0]
10002228:	4a21      	ldr	r2, [pc, #132]	; (100022b0 <clocks_init+0xf0>)
1000222a:	2101      	movs	r1, #1
1000222c:	4821      	ldr	r0, [pc, #132]	; (100022b4 <clocks_init+0xf4>)
1000222e:	f000 f84d 	bl	100022cc <pll_init>
10002232:	4b21      	ldr	r3, [pc, #132]	; (100022b8 <clocks_init+0xf8>)
10002234:	9300      	str	r3, [sp, #0]
10002236:	2200      	movs	r2, #0
10002238:	2102      	movs	r1, #2
1000223a:	2004      	movs	r0, #4
1000223c:	f7ff ff3c 	bl	100020b8 <clock_configure>
10002240:	4d1e      	ldr	r5, [pc, #120]	; (100022bc <clocks_init+0xfc>)
10002242:	9500      	str	r5, [sp, #0]
10002244:	002b      	movs	r3, r5
10002246:	2200      	movs	r2, #0
10002248:	2101      	movs	r1, #1
1000224a:	2005      	movs	r0, #5
1000224c:	f7ff ff34 	bl	100020b8 <clock_configure>
10002250:	4c10      	ldr	r4, [pc, #64]	; (10002294 <clocks_init+0xd4>)
10002252:	9400      	str	r4, [sp, #0]
10002254:	0023      	movs	r3, r4
10002256:	2200      	movs	r2, #0
10002258:	2100      	movs	r1, #0
1000225a:	2007      	movs	r0, #7
1000225c:	f7ff ff2c 	bl	100020b8 <clock_configure>
10002260:	9400      	str	r4, [sp, #0]
10002262:	0023      	movs	r3, r4
10002264:	2200      	movs	r2, #0
10002266:	2100      	movs	r1, #0
10002268:	2008      	movs	r0, #8
1000226a:	f7ff ff25 	bl	100020b8 <clock_configure>
1000226e:	4b0a      	ldr	r3, [pc, #40]	; (10002298 <clocks_init+0xd8>)
10002270:	9300      	str	r3, [sp, #0]
10002272:	0023      	movs	r3, r4
10002274:	2200      	movs	r2, #0
10002276:	2100      	movs	r1, #0
10002278:	2009      	movs	r0, #9
1000227a:	f7ff ff1d 	bl	100020b8 <clock_configure>
1000227e:	9500      	str	r5, [sp, #0]
10002280:	002b      	movs	r3, r5
10002282:	2200      	movs	r2, #0
10002284:	2100      	movs	r1, #0
10002286:	2006      	movs	r0, #6
10002288:	f7ff ff16 	bl	100020b8 <clock_configure>
1000228c:	e7ad      	b.n	100021ea <clocks_init+0x2a>
1000228e:	46c0      	nop			; (mov r8, r8)
10002290:	20000444 	.word	0x20000444
10002294:	02dc6c00 	.word	0x02dc6c00
10002298:	0000b71b 	.word	0x0000b71b
1000229c:	40008000 	.word	0x40008000
100022a0:	4000b03c 	.word	0x4000b03c
100022a4:	4000b030 	.word	0x4000b030
100022a8:	59682f00 	.word	0x59682f00
100022ac:	40028000 	.word	0x40028000
100022b0:	47868c00 	.word	0x47868c00
100022b4:	4002c000 	.word	0x4002c000
100022b8:	00b71b00 	.word	0x00b71b00
100022bc:	07735940 	.word	0x07735940

100022c0 <clock_get_hz>:
100022c0:	0080      	lsls	r0, r0, #2
100022c2:	4b01      	ldr	r3, [pc, #4]	; (100022c8 <clock_get_hz+0x8>)
100022c4:	58c0      	ldr	r0, [r0, r3]
100022c6:	4770      	bx	lr
100022c8:	20000444 	.word	0x20000444

100022cc <pll_init>:
100022cc:	b5f0      	push	{r4, r5, r6, r7, lr}
100022ce:	46c6      	mov	lr, r8
100022d0:	b500      	push	{lr}
100022d2:	0004      	movs	r4, r0
100022d4:	000e      	movs	r6, r1
100022d6:	0017      	movs	r7, r2
100022d8:	001d      	movs	r5, r3
100022da:	4837      	ldr	r0, [pc, #220]	; (100023b8 <pll_init+0xec>)
100022dc:	f001 fa56 	bl	1000378c <__wrap___aeabi_uidiv>
100022e0:	4680      	mov	r8, r0
100022e2:	4b36      	ldr	r3, [pc, #216]	; (100023bc <pll_init+0xf0>)
100022e4:	18fa      	adds	r2, r7, r3
100022e6:	4b36      	ldr	r3, [pc, #216]	; (100023c0 <pll_init+0xf4>)
100022e8:	429a      	cmp	r2, r3
100022ea:	d839      	bhi.n	10002360 <pll_init+0x94>
100022ec:	0001      	movs	r1, r0
100022ee:	0038      	movs	r0, r7
100022f0:	f001 fa4c 	bl	1000378c <__wrap___aeabi_uidiv>
100022f4:	0002      	movs	r2, r0
100022f6:	3a10      	subs	r2, #16
100022f8:	2398      	movs	r3, #152	; 0x98
100022fa:	005b      	lsls	r3, r3, #1
100022fc:	429a      	cmp	r2, r3
100022fe:	d835      	bhi.n	1000236c <pll_init+0xa0>
10002300:	1e6b      	subs	r3, r5, #1
10002302:	2b06      	cmp	r3, #6
10002304:	d838      	bhi.n	10002378 <pll_init+0xac>
10002306:	9b06      	ldr	r3, [sp, #24]
10002308:	3b01      	subs	r3, #1
1000230a:	2b06      	cmp	r3, #6
1000230c:	d834      	bhi.n	10002378 <pll_init+0xac>
1000230e:	093f      	lsrs	r7, r7, #4
10002310:	4547      	cmp	r7, r8
10002312:	d337      	bcc.n	10002384 <pll_init+0xb8>
10002314:	042d      	lsls	r5, r5, #16
10002316:	9b06      	ldr	r3, [sp, #24]
10002318:	031a      	lsls	r2, r3, #12
1000231a:	4315      	orrs	r5, r2
1000231c:	6823      	ldr	r3, [r4, #0]
1000231e:	2b00      	cmp	r3, #0
10002320:	db36      	blt.n	10002390 <pll_init+0xc4>
10002322:	4b28      	ldr	r3, [pc, #160]	; (100023c4 <pll_init+0xf8>)
10002324:	429c      	cmp	r4, r3
10002326:	d044      	beq.n	100023b2 <pll_init+0xe6>
10002328:	2280      	movs	r2, #128	; 0x80
1000232a:	0152      	lsls	r2, r2, #5
1000232c:	4b26      	ldr	r3, [pc, #152]	; (100023c8 <pll_init+0xfc>)
1000232e:	601a      	str	r2, [r3, #0]
10002330:	4b26      	ldr	r3, [pc, #152]	; (100023cc <pll_init+0x100>)
10002332:	601a      	str	r2, [r3, #0]
10002334:	4b26      	ldr	r3, [pc, #152]	; (100023d0 <pll_init+0x104>)
10002336:	689b      	ldr	r3, [r3, #8]
10002338:	0011      	movs	r1, r2
1000233a:	4399      	bics	r1, r3
1000233c:	d1fa      	bne.n	10002334 <pll_init+0x68>
1000233e:	6026      	str	r6, [r4, #0]
10002340:	60a0      	str	r0, [r4, #8]
10002342:	1d23      	adds	r3, r4, #4
10002344:	22c0      	movs	r2, #192	; 0xc0
10002346:	0192      	lsls	r2, r2, #6
10002348:	431a      	orrs	r2, r3
1000234a:	2321      	movs	r3, #33	; 0x21
1000234c:	6013      	str	r3, [r2, #0]
1000234e:	6823      	ldr	r3, [r4, #0]
10002350:	2b00      	cmp	r3, #0
10002352:	dafc      	bge.n	1000234e <pll_init+0x82>
10002354:	60e5      	str	r5, [r4, #12]
10002356:	2308      	movs	r3, #8
10002358:	6013      	str	r3, [r2, #0]
1000235a:	bc80      	pop	{r7}
1000235c:	46b8      	mov	r8, r7
1000235e:	bdf0      	pop	{r4, r5, r6, r7, pc}
10002360:	4b1c      	ldr	r3, [pc, #112]	; (100023d4 <pll_init+0x108>)
10002362:	4a1d      	ldr	r2, [pc, #116]	; (100023d8 <pll_init+0x10c>)
10002364:	2111      	movs	r1, #17
10002366:	481d      	ldr	r0, [pc, #116]	; (100023dc <pll_init+0x110>)
10002368:	f000 f862 	bl	10002430 <__assert_func>
1000236c:	4b1c      	ldr	r3, [pc, #112]	; (100023e0 <pll_init+0x114>)
1000236e:	4a1a      	ldr	r2, [pc, #104]	; (100023d8 <pll_init+0x10c>)
10002370:	2119      	movs	r1, #25
10002372:	481a      	ldr	r0, [pc, #104]	; (100023dc <pll_init+0x110>)
10002374:	f000 f85c 	bl	10002430 <__assert_func>
10002378:	4b1a      	ldr	r3, [pc, #104]	; (100023e4 <pll_init+0x118>)
1000237a:	4a17      	ldr	r2, [pc, #92]	; (100023d8 <pll_init+0x10c>)
1000237c:	211c      	movs	r1, #28
1000237e:	4817      	ldr	r0, [pc, #92]	; (100023dc <pll_init+0x110>)
10002380:	f000 f856 	bl	10002430 <__assert_func>
10002384:	4b18      	ldr	r3, [pc, #96]	; (100023e8 <pll_init+0x11c>)
10002386:	4a14      	ldr	r2, [pc, #80]	; (100023d8 <pll_init+0x10c>)
10002388:	2123      	movs	r1, #35	; 0x23
1000238a:	4814      	ldr	r0, [pc, #80]	; (100023dc <pll_init+0x110>)
1000238c:	f000 f850 	bl	10002430 <__assert_func>
10002390:	6822      	ldr	r2, [r4, #0]
10002392:	233f      	movs	r3, #63	; 0x3f
10002394:	4013      	ands	r3, r2
10002396:	42b3      	cmp	r3, r6
10002398:	d1c3      	bne.n	10002322 <pll_init+0x56>
1000239a:	68a3      	ldr	r3, [r4, #8]
1000239c:	051b      	lsls	r3, r3, #20
1000239e:	0d1b      	lsrs	r3, r3, #20
100023a0:	4283      	cmp	r3, r0
100023a2:	d1be      	bne.n	10002322 <pll_init+0x56>
100023a4:	68e3      	ldr	r3, [r4, #12]
100023a6:	22ee      	movs	r2, #238	; 0xee
100023a8:	02d2      	lsls	r2, r2, #11
100023aa:	4013      	ands	r3, r2
100023ac:	42ab      	cmp	r3, r5
100023ae:	d1b8      	bne.n	10002322 <pll_init+0x56>
100023b0:	e7d3      	b.n	1000235a <pll_init+0x8e>
100023b2:	2280      	movs	r2, #128	; 0x80
100023b4:	0192      	lsls	r2, r2, #6
100023b6:	e7b9      	b.n	1000232c <pll_init+0x60>
100023b8:	00b71b00 	.word	0x00b71b00
100023bc:	d34be880 	.word	0xd34be880
100023c0:	32a9f880 	.word	0x32a9f880
100023c4:	4002c000 	.word	0x4002c000
100023c8:	4000e000 	.word	0x4000e000
100023cc:	4000f000 	.word	0x4000f000
100023d0:	4000c000 	.word	0x4000c000
100023d4:	1000583c 	.word	0x1000583c
100023d8:	10005964 	.word	0x10005964
100023dc:	1000589c 	.word	0x1000589c
100023e0:	100058e0 	.word	0x100058e0
100023e4:	100058fc 	.word	0x100058fc
100023e8:	10005948 	.word	0x10005948

100023ec <watchdog_start_tick>:
100023ec:	2380      	movs	r3, #128	; 0x80
100023ee:	009b      	lsls	r3, r3, #2
100023f0:	4303      	orrs	r3, r0
100023f2:	4a01      	ldr	r2, [pc, #4]	; (100023f8 <watchdog_start_tick+0xc>)
100023f4:	62d3      	str	r3, [r2, #44]	; 0x2c
100023f6:	4770      	bx	lr
100023f8:	40058000 	.word	0x40058000

100023fc <xosc_init>:
100023fc:	4b06      	ldr	r3, [pc, #24]	; (10002418 <xosc_init+0x1c>)
100023fe:	22aa      	movs	r2, #170	; 0xaa
10002400:	0112      	lsls	r2, r2, #4
10002402:	601a      	str	r2, [r3, #0]
10002404:	222f      	movs	r2, #47	; 0x2f
10002406:	60da      	str	r2, [r3, #12]
10002408:	4b04      	ldr	r3, [pc, #16]	; (1000241c <xosc_init+0x20>)
1000240a:	4a05      	ldr	r2, [pc, #20]	; (10002420 <xosc_init+0x24>)
1000240c:	601a      	str	r2, [r3, #0]
1000240e:	4b02      	ldr	r3, [pc, #8]	; (10002418 <xosc_init+0x1c>)
10002410:	685b      	ldr	r3, [r3, #4]
10002412:	2b00      	cmp	r3, #0
10002414:	dafb      	bge.n	1000240e <xosc_init+0x12>
10002416:	4770      	bx	lr
10002418:	40024000 	.word	0x40024000
1000241c:	40026000 	.word	0x40026000
10002420:	00fab000 	.word	0x00fab000

10002424 <_exit>:
10002424:	be00      	bkpt	0x0000
10002426:	e7fd      	b.n	10002424 <_exit>

10002428 <exit>:
10002428:	b510      	push	{r4, lr}
1000242a:	f7ff fffb 	bl	10002424 <_exit>
	...

10002430 <__assert_func>:
10002430:	b510      	push	{r4, lr}
10002432:	b082      	sub	sp, #8
10002434:	000c      	movs	r4, r1
10002436:	0019      	movs	r1, r3
10002438:	2a00      	cmp	r2, #0
1000243a:	d00c      	beq.n	10002456 <__assert_func+0x26>
1000243c:	4b08      	ldr	r3, [pc, #32]	; (10002460 <__assert_func+0x30>)
1000243e:	2a00      	cmp	r2, #0
10002440:	d00b      	beq.n	1000245a <__assert_func+0x2a>
10002442:	9201      	str	r2, [sp, #4]
10002444:	9300      	str	r3, [sp, #0]
10002446:	0023      	movs	r3, r4
10002448:	0002      	movs	r2, r0
1000244a:	4806      	ldr	r0, [pc, #24]	; (10002464 <__assert_func+0x34>)
1000244c:	f002 f9f2 	bl	10004834 <__wrap_printf>
10002450:	2001      	movs	r0, #1
10002452:	f7ff ffe7 	bl	10002424 <_exit>
10002456:	4b04      	ldr	r3, [pc, #16]	; (10002468 <__assert_func+0x38>)
10002458:	e7f1      	b.n	1000243e <__assert_func+0xe>
1000245a:	4a03      	ldr	r2, [pc, #12]	; (10002468 <__assert_func+0x38>)
1000245c:	e7f1      	b.n	10002442 <__assert_func+0x12>
1000245e:	46c0      	nop			; (mov r8, r8)
10002460:	10005970 	.word	0x10005970
10002464:	10005980 	.word	0x10005980
10002468:	1000597c 	.word	0x1000597c

1000246c <runtime_init>:
1000246c:	b570      	push	{r4, r5, r6, lr}
1000246e:	4b2b      	ldr	r3, [pc, #172]	; (1000251c <runtime_init+0xb0>)
10002470:	4a2b      	ldr	r2, [pc, #172]	; (10002520 <runtime_init+0xb4>)
10002472:	601a      	str	r2, [r3, #0]
10002474:	4b2b      	ldr	r3, [pc, #172]	; (10002524 <runtime_init+0xb8>)
10002476:	4a2c      	ldr	r2, [pc, #176]	; (10002528 <runtime_init+0xbc>)
10002478:	601a      	str	r2, [r3, #0]
1000247a:	4b2c      	ldr	r3, [pc, #176]	; (1000252c <runtime_init+0xc0>)
1000247c:	689a      	ldr	r2, [r3, #8]
1000247e:	4b2a      	ldr	r3, [pc, #168]	; (10002528 <runtime_init+0xbc>)
10002480:	4393      	bics	r3, r2
10002482:	d1fa      	bne.n	1000247a <runtime_init+0xe>
10002484:	4c2a      	ldr	r4, [pc, #168]	; (10002530 <runtime_init+0xc4>)
10002486:	e001      	b.n	1000248c <runtime_init+0x20>
10002488:	cc08      	ldmia	r4!, {r3}
1000248a:	4798      	blx	r3
1000248c:	4b29      	ldr	r3, [pc, #164]	; (10002534 <runtime_init+0xc8>)
1000248e:	429c      	cmp	r4, r3
10002490:	d3fa      	bcc.n	10002488 <runtime_init+0x1c>
10002492:	f7ff fe95 	bl	100021c0 <clocks_init>
10002496:	4b23      	ldr	r3, [pc, #140]	; (10002524 <runtime_init+0xb8>)
10002498:	4a27      	ldr	r2, [pc, #156]	; (10002538 <runtime_init+0xcc>)
1000249a:	601a      	str	r2, [r3, #0]
1000249c:	4b23      	ldr	r3, [pc, #140]	; (1000252c <runtime_init+0xc0>)
1000249e:	689b      	ldr	r3, [r3, #8]
100024a0:	43db      	mvns	r3, r3
100024a2:	01db      	lsls	r3, r3, #7
100024a4:	d1fa      	bne.n	1000249c <runtime_init+0x30>
100024a6:	4b25      	ldr	r3, [pc, #148]	; (1000253c <runtime_init+0xd0>)
100024a8:	2240      	movs	r2, #64	; 0x40
100024aa:	679a      	str	r2, [r3, #120]	; 0x78
100024ac:	675a      	str	r2, [r3, #116]	; 0x74
100024ae:	671a      	str	r2, [r3, #112]	; 0x70
100024b0:	66da      	str	r2, [r3, #108]	; 0x6c
100024b2:	4c23      	ldr	r4, [pc, #140]	; (10002540 <runtime_init+0xd4>)
100024b4:	e009      	b.n	100024ca <runtime_init+0x5e>
100024b6:	4b23      	ldr	r3, [pc, #140]	; (10002544 <runtime_init+0xd8>)
100024b8:	4a23      	ldr	r2, [pc, #140]	; (10002548 <runtime_init+0xdc>)
100024ba:	2187      	movs	r1, #135	; 0x87
100024bc:	4823      	ldr	r0, [pc, #140]	; (1000254c <runtime_init+0xe0>)
100024be:	f7ff ffb7 	bl	10002430 <__assert_func>
100024c2:	0020      	movs	r0, r4
100024c4:	f7fe fbca 	bl	10000c5c <mutex_init>
100024c8:	3408      	adds	r4, #8
100024ca:	4b21      	ldr	r3, [pc, #132]	; (10002550 <runtime_init+0xe4>)
100024cc:	429c      	cmp	r4, r3
100024ce:	d209      	bcs.n	100024e4 <runtime_init+0x78>
100024d0:	6823      	ldr	r3, [r4, #0]
100024d2:	2b00      	cmp	r3, #0
100024d4:	d0f5      	beq.n	100024c2 <runtime_init+0x56>
100024d6:	2b01      	cmp	r3, #1
100024d8:	d1ed      	bne.n	100024b6 <runtime_init+0x4a>
100024da:	0020      	movs	r0, r4
100024dc:	f7fe fbcb 	bl	10000c76 <recursive_mutex_init>
100024e0:	3408      	adds	r4, #8
100024e2:	e7f2      	b.n	100024ca <runtime_init+0x5e>
100024e4:	4c1b      	ldr	r4, [pc, #108]	; (10002554 <runtime_init+0xe8>)
100024e6:	68a1      	ldr	r1, [r4, #8]
100024e8:	4d1b      	ldr	r5, [pc, #108]	; (10002558 <runtime_init+0xec>)
100024ea:	22c0      	movs	r2, #192	; 0xc0
100024ec:	0028      	movs	r0, r5
100024ee:	f002 f849 	bl	10004584 <__wrap___aeabi_memcpy>
100024f2:	60a5      	str	r5, [r4, #8]
100024f4:	f3ef 8305 	mrs	r3, IPSR
100024f8:	2b00      	cmp	r3, #0
100024fa:	d000      	beq.n	100024fe <runtime_init+0x92>
100024fc:	be00      	bkpt	0x0000
100024fe:	f7fe f97d 	bl	100007fc <spin_locks_reset>
10002502:	f7fe fb95 	bl	10000c30 <irq_init_priorities>
10002506:	f7fe ff05 	bl	10001314 <alarm_pool_init_default>
1000250a:	4c14      	ldr	r4, [pc, #80]	; (1000255c <runtime_init+0xf0>)
1000250c:	e001      	b.n	10002512 <runtime_init+0xa6>
1000250e:	cc08      	ldmia	r4!, {r3}
10002510:	4798      	blx	r3
10002512:	4b13      	ldr	r3, [pc, #76]	; (10002560 <runtime_init+0xf4>)
10002514:	429c      	cmp	r4, r3
10002516:	d3fa      	bcc.n	1000250e <runtime_init+0xa2>
10002518:	bd70      	pop	{r4, r5, r6, pc}
1000251a:	46c0      	nop			; (mov r8, r8)
1000251c:	4000e000 	.word	0x4000e000
10002520:	fefbcdbf 	.word	0xfefbcdbf
10002524:	4000f000 	.word	0x4000f000
10002528:	003c7ffe 	.word	0x003c7ffe
1000252c:	4000c000 	.word	0x4000c000
10002530:	200002f0 	.word	0x200002f0
10002534:	20000300 	.word	0x20000300
10002538:	01ffffff 	.word	0x01ffffff
1000253c:	4001f000 	.word	0x4001f000
10002540:	200002e8 	.word	0x200002e8
10002544:	100059b0 	.word	0x100059b0
10002548:	10005a2c 	.word	0x10005a2c
1000254c:	100059d0 	.word	0x100059d0
10002550:	200002f0 	.word	0x200002f0
10002554:	e000ed00 	.word	0xe000ed00
10002558:	20000000 	.word	0x20000000
1000255c:	20000300 	.word	0x20000300
10002560:	20000304 	.word	0x20000304

10002564 <panic>:
10002564:	b40f      	push	{r0, r1, r2, r3}
10002566:	b500      	push	{lr}
10002568:	b083      	sub	sp, #12
1000256a:	4808      	ldr	r0, [pc, #32]	; (1000258c <panic+0x28>)
1000256c:	f002 f932 	bl	100047d4 <__wrap_puts>
10002570:	9b04      	ldr	r3, [sp, #16]
10002572:	2b00      	cmp	r3, #0
10002574:	d007      	beq.n	10002586 <panic+0x22>
10002576:	a905      	add	r1, sp, #20
10002578:	9101      	str	r1, [sp, #4]
1000257a:	0018      	movs	r0, r3
1000257c:	f002 f93a 	bl	100047f4 <__wrap_vprintf>
10002580:	4803      	ldr	r0, [pc, #12]	; (10002590 <panic+0x2c>)
10002582:	f002 f927 	bl	100047d4 <__wrap_puts>
10002586:	2001      	movs	r0, #1
10002588:	f7ff ff4c 	bl	10002424 <_exit>
1000258c:	10005a18 	.word	0x10005a18
10002590:	10005a28 	.word	0x10005a28

10002594 <_out_null>:
10002594:	4770      	bx	lr

10002596 <_out_fct>:
10002596:	b510      	push	{r4, lr}
10002598:	2800      	cmp	r0, #0
1000259a:	d002      	beq.n	100025a2 <_out_fct+0xc>
1000259c:	680b      	ldr	r3, [r1, #0]
1000259e:	6849      	ldr	r1, [r1, #4]
100025a0:	4798      	blx	r3
100025a2:	bd10      	pop	{r4, pc}

100025a4 <_atoi>:
100025a4:	0001      	movs	r1, r0
100025a6:	2000      	movs	r0, #0
100025a8:	e007      	b.n	100025ba <_atoi+0x16>
100025aa:	0083      	lsls	r3, r0, #2
100025ac:	181b      	adds	r3, r3, r0
100025ae:	005b      	lsls	r3, r3, #1
100025b0:	1c50      	adds	r0, r2, #1
100025b2:	6008      	str	r0, [r1, #0]
100025b4:	7810      	ldrb	r0, [r2, #0]
100025b6:	18c0      	adds	r0, r0, r3
100025b8:	3830      	subs	r0, #48	; 0x30
100025ba:	680a      	ldr	r2, [r1, #0]
100025bc:	7813      	ldrb	r3, [r2, #0]
100025be:	3b30      	subs	r3, #48	; 0x30
100025c0:	b2db      	uxtb	r3, r3
100025c2:	2b09      	cmp	r3, #9
100025c4:	d9f1      	bls.n	100025aa <_atoi+0x6>
100025c6:	4770      	bx	lr

100025c8 <_out_rev>:
100025c8:	b5f0      	push	{r4, r5, r6, r7, lr}
100025ca:	46de      	mov	lr, fp
100025cc:	4657      	mov	r7, sl
100025ce:	464e      	mov	r6, r9
100025d0:	4645      	mov	r5, r8
100025d2:	b5e0      	push	{r5, r6, r7, lr}
100025d4:	b083      	sub	sp, #12
100025d6:	4693      	mov	fp, r2
100025d8:	001f      	movs	r7, r3
100025da:	9b0c      	ldr	r3, [sp, #48]	; 0x30
100025dc:	469a      	mov	sl, r3
100025de:	9c0d      	ldr	r4, [sp, #52]	; 0x34
100025e0:	9b0e      	ldr	r3, [sp, #56]	; 0x38
100025e2:	4699      	mov	r9, r3
100025e4:	9b0f      	ldr	r3, [sp, #60]	; 0x3c
100025e6:	079b      	lsls	r3, r3, #30
100025e8:	d003      	beq.n	100025f2 <_out_rev+0x2a>
100025ea:	46b8      	mov	r8, r7
100025ec:	000f      	movs	r7, r1
100025ee:	0006      	movs	r6, r0
100025f0:	e022      	b.n	10002638 <_out_rev+0x70>
100025f2:	9201      	str	r2, [sp, #4]
100025f4:	46a3      	mov	fp, r4
100025f6:	4688      	mov	r8, r1
100025f8:	464e      	mov	r6, r9
100025fa:	46b9      	mov	r9, r7
100025fc:	0007      	movs	r7, r0
100025fe:	42b4      	cmp	r4, r6
10002600:	d207      	bcs.n	10002612 <_out_rev+0x4a>
10002602:	1c55      	adds	r5, r2, #1
10002604:	464b      	mov	r3, r9
10002606:	4641      	mov	r1, r8
10002608:	2020      	movs	r0, #32
1000260a:	47b8      	blx	r7
1000260c:	3401      	adds	r4, #1
1000260e:	002a      	movs	r2, r5
10002610:	e7f5      	b.n	100025fe <_out_rev+0x36>
10002612:	003d      	movs	r5, r7
10002614:	464f      	mov	r7, r9
10002616:	465c      	mov	r4, fp
10002618:	9b01      	ldr	r3, [sp, #4]
1000261a:	469b      	mov	fp, r3
1000261c:	46b1      	mov	r9, r6
1000261e:	4646      	mov	r6, r8
10002620:	46b8      	mov	r8, r7
10002622:	0037      	movs	r7, r6
10002624:	002e      	movs	r6, r5
10002626:	e007      	b.n	10002638 <_out_rev+0x70>
10002628:	3c01      	subs	r4, #1
1000262a:	1c55      	adds	r5, r2, #1
1000262c:	4653      	mov	r3, sl
1000262e:	5d18      	ldrb	r0, [r3, r4]
10002630:	4643      	mov	r3, r8
10002632:	0039      	movs	r1, r7
10002634:	47b0      	blx	r6
10002636:	002a      	movs	r2, r5
10002638:	2c00      	cmp	r4, #0
1000263a:	d1f5      	bne.n	10002628 <_out_rev+0x60>
1000263c:	0035      	movs	r5, r6
1000263e:	003e      	movs	r6, r7
10002640:	4647      	mov	r7, r8
10002642:	9b0f      	ldr	r3, [sp, #60]	; 0x3c
10002644:	079b      	lsls	r3, r3, #30
10002646:	d407      	bmi.n	10002658 <_out_rev+0x90>
10002648:	0010      	movs	r0, r2
1000264a:	b003      	add	sp, #12
1000264c:	bcf0      	pop	{r4, r5, r6, r7}
1000264e:	46bb      	mov	fp, r7
10002650:	46b2      	mov	sl, r6
10002652:	46a9      	mov	r9, r5
10002654:	46a0      	mov	r8, r4
10002656:	bdf0      	pop	{r4, r5, r6, r7, pc}
10002658:	46b0      	mov	r8, r6
1000265a:	464e      	mov	r6, r9
1000265c:	46b9      	mov	r9, r7
1000265e:	002f      	movs	r7, r5
10002660:	465d      	mov	r5, fp
10002662:	1b53      	subs	r3, r2, r5
10002664:	42b3      	cmp	r3, r6
10002666:	d2ef      	bcs.n	10002648 <_out_rev+0x80>
10002668:	1c54      	adds	r4, r2, #1
1000266a:	464b      	mov	r3, r9
1000266c:	4641      	mov	r1, r8
1000266e:	2020      	movs	r0, #32
10002670:	47b8      	blx	r7
10002672:	0022      	movs	r2, r4
10002674:	e7f5      	b.n	10002662 <_out_rev+0x9a>

10002676 <_ntoa_format>:
10002676:	b5f0      	push	{r4, r5, r6, r7, lr}
10002678:	46ce      	mov	lr, r9
1000267a:	4647      	mov	r7, r8
1000267c:	b580      	push	{r7, lr}
1000267e:	b085      	sub	sp, #20
10002680:	4694      	mov	ip, r2
10002682:	4698      	mov	r8, r3
10002684:	9d0c      	ldr	r5, [sp, #48]	; 0x30
10002686:	9c0d      	ldr	r4, [sp, #52]	; 0x34
10002688:	ab0e      	add	r3, sp, #56	; 0x38
1000268a:	781b      	ldrb	r3, [r3, #0]
1000268c:	4699      	mov	r9, r3
1000268e:	9a10      	ldr	r2, [sp, #64]	; 0x40
10002690:	9b11      	ldr	r3, [sp, #68]	; 0x44
10002692:	9e12      	ldr	r6, [sp, #72]	; 0x48
10002694:	07b7      	lsls	r7, r6, #30
10002696:	d41c      	bmi.n	100026d2 <_ntoa_format+0x5c>
10002698:	2b00      	cmp	r3, #0
1000269a:	d00c      	beq.n	100026b6 <_ntoa_format+0x40>
1000269c:	07f7      	lsls	r7, r6, #31
1000269e:	d50a      	bpl.n	100026b6 <_ntoa_format+0x40>
100026a0:	464f      	mov	r7, r9
100026a2:	2f00      	cmp	r7, #0
100026a4:	d102      	bne.n	100026ac <_ntoa_format+0x36>
100026a6:	370c      	adds	r7, #12
100026a8:	4237      	tst	r7, r6
100026aa:	d004      	beq.n	100026b6 <_ntoa_format+0x40>
100026ac:	3b01      	subs	r3, #1
100026ae:	e002      	b.n	100026b6 <_ntoa_format+0x40>
100026b0:	2730      	movs	r7, #48	; 0x30
100026b2:	552f      	strb	r7, [r5, r4]
100026b4:	3401      	adds	r4, #1
100026b6:	4294      	cmp	r4, r2
100026b8:	d201      	bcs.n	100026be <_ntoa_format+0x48>
100026ba:	2c1f      	cmp	r4, #31
100026bc:	d9f8      	bls.n	100026b0 <_ntoa_format+0x3a>
100026be:	07f7      	lsls	r7, r6, #31
100026c0:	d507      	bpl.n	100026d2 <_ntoa_format+0x5c>
100026c2:	429c      	cmp	r4, r3
100026c4:	d205      	bcs.n	100026d2 <_ntoa_format+0x5c>
100026c6:	2c1f      	cmp	r4, #31
100026c8:	d803      	bhi.n	100026d2 <_ntoa_format+0x5c>
100026ca:	2730      	movs	r7, #48	; 0x30
100026cc:	552f      	strb	r7, [r5, r4]
100026ce:	3401      	adds	r4, #1
100026d0:	e7f5      	b.n	100026be <_ntoa_format+0x48>
100026d2:	06f7      	lsls	r7, r6, #27
100026d4:	d515      	bpl.n	10002702 <_ntoa_format+0x8c>
100026d6:	0577      	lsls	r7, r6, #21
100026d8:	d405      	bmi.n	100026e6 <_ntoa_format+0x70>
100026da:	2c00      	cmp	r4, #0
100026dc:	d003      	beq.n	100026e6 <_ntoa_format+0x70>
100026de:	4294      	cmp	r4, r2
100026e0:	d024      	beq.n	1000272c <_ntoa_format+0xb6>
100026e2:	429c      	cmp	r4, r3
100026e4:	d022      	beq.n	1000272c <_ntoa_format+0xb6>
100026e6:	9a0f      	ldr	r2, [sp, #60]	; 0x3c
100026e8:	2a10      	cmp	r2, #16
100026ea:	d02b      	beq.n	10002744 <_ntoa_format+0xce>
100026ec:	9a0f      	ldr	r2, [sp, #60]	; 0x3c
100026ee:	2a10      	cmp	r2, #16
100026f0:	d030      	beq.n	10002754 <_ntoa_format+0xde>
100026f2:	9a0f      	ldr	r2, [sp, #60]	; 0x3c
100026f4:	2a02      	cmp	r2, #2
100026f6:	d035      	beq.n	10002764 <_ntoa_format+0xee>
100026f8:	2c1f      	cmp	r4, #31
100026fa:	d802      	bhi.n	10002702 <_ntoa_format+0x8c>
100026fc:	2230      	movs	r2, #48	; 0x30
100026fe:	552a      	strb	r2, [r5, r4]
10002700:	3401      	adds	r4, #1
10002702:	2c1f      	cmp	r4, #31
10002704:	d805      	bhi.n	10002712 <_ntoa_format+0x9c>
10002706:	464a      	mov	r2, r9
10002708:	2a00      	cmp	r2, #0
1000270a:	d031      	beq.n	10002770 <_ntoa_format+0xfa>
1000270c:	222d      	movs	r2, #45	; 0x2d
1000270e:	552a      	strb	r2, [r5, r4]
10002710:	3401      	adds	r4, #1
10002712:	9603      	str	r6, [sp, #12]
10002714:	9302      	str	r3, [sp, #8]
10002716:	9401      	str	r4, [sp, #4]
10002718:	9500      	str	r5, [sp, #0]
1000271a:	4643      	mov	r3, r8
1000271c:	4662      	mov	r2, ip
1000271e:	f7ff ff53 	bl	100025c8 <_out_rev>
10002722:	b005      	add	sp, #20
10002724:	bcc0      	pop	{r6, r7}
10002726:	46b9      	mov	r9, r7
10002728:	46b0      	mov	r8, r6
1000272a:	bdf0      	pop	{r4, r5, r6, r7, pc}
1000272c:	1e62      	subs	r2, r4, #1
1000272e:	2c01      	cmp	r4, #1
10002730:	d006      	beq.n	10002740 <_ntoa_format+0xca>
10002732:	9f0f      	ldr	r7, [sp, #60]	; 0x3c
10002734:	2f10      	cmp	r7, #16
10002736:	d001      	beq.n	1000273c <_ntoa_format+0xc6>
10002738:	0014      	movs	r4, r2
1000273a:	e7d4      	b.n	100026e6 <_ntoa_format+0x70>
1000273c:	3c02      	subs	r4, #2
1000273e:	e7d2      	b.n	100026e6 <_ntoa_format+0x70>
10002740:	0014      	movs	r4, r2
10002742:	e7d0      	b.n	100026e6 <_ntoa_format+0x70>
10002744:	06b2      	lsls	r2, r6, #26
10002746:	d4d1      	bmi.n	100026ec <_ntoa_format+0x76>
10002748:	2c1f      	cmp	r4, #31
1000274a:	d8cf      	bhi.n	100026ec <_ntoa_format+0x76>
1000274c:	2278      	movs	r2, #120	; 0x78
1000274e:	552a      	strb	r2, [r5, r4]
10002750:	3401      	adds	r4, #1
10002752:	e7d1      	b.n	100026f8 <_ntoa_format+0x82>
10002754:	06b2      	lsls	r2, r6, #26
10002756:	d5cc      	bpl.n	100026f2 <_ntoa_format+0x7c>
10002758:	2c1f      	cmp	r4, #31
1000275a:	d8ca      	bhi.n	100026f2 <_ntoa_format+0x7c>
1000275c:	2258      	movs	r2, #88	; 0x58
1000275e:	552a      	strb	r2, [r5, r4]
10002760:	3401      	adds	r4, #1
10002762:	e7c9      	b.n	100026f8 <_ntoa_format+0x82>
10002764:	2c1f      	cmp	r4, #31
10002766:	d8c7      	bhi.n	100026f8 <_ntoa_format+0x82>
10002768:	3260      	adds	r2, #96	; 0x60
1000276a:	552a      	strb	r2, [r5, r4]
1000276c:	3401      	adds	r4, #1
1000276e:	e7c3      	b.n	100026f8 <_ntoa_format+0x82>
10002770:	0772      	lsls	r2, r6, #29
10002772:	d503      	bpl.n	1000277c <_ntoa_format+0x106>
10002774:	222b      	movs	r2, #43	; 0x2b
10002776:	552a      	strb	r2, [r5, r4]
10002778:	3401      	adds	r4, #1
1000277a:	e7ca      	b.n	10002712 <_ntoa_format+0x9c>
1000277c:	0732      	lsls	r2, r6, #28
1000277e:	d5c8      	bpl.n	10002712 <_ntoa_format+0x9c>
10002780:	2220      	movs	r2, #32
10002782:	552a      	strb	r2, [r5, r4]
10002784:	3401      	adds	r4, #1
10002786:	e7c4      	b.n	10002712 <_ntoa_format+0x9c>

10002788 <_ntoa_long>:
10002788:	b5f0      	push	{r4, r5, r6, r7, lr}
1000278a:	46de      	mov	lr, fp
1000278c:	4657      	mov	r7, sl
1000278e:	464e      	mov	r6, r9
10002790:	4645      	mov	r5, r8
10002792:	b5e0      	push	{r5, r6, r7, lr}
10002794:	b093      	sub	sp, #76	; 0x4c
10002796:	4681      	mov	r9, r0
10002798:	468a      	mov	sl, r1
1000279a:	9208      	str	r2, [sp, #32]
1000279c:	9309      	str	r3, [sp, #36]	; 0x24
1000279e:	ab1c      	add	r3, sp, #112	; 0x70
100027a0:	cb10      	ldmia	r3!, {r4}
100027a2:	781b      	ldrb	r3, [r3, #0]
100027a4:	469b      	mov	fp, r3
100027a6:	9d1e      	ldr	r5, [sp, #120]	; 0x78
100027a8:	9b21      	ldr	r3, [sp, #132]	; 0x84
100027aa:	4698      	mov	r8, r3
100027ac:	2c00      	cmp	r4, #0
100027ae:	d103      	bne.n	100027b8 <_ntoa_long+0x30>
100027b0:	2310      	movs	r3, #16
100027b2:	4642      	mov	r2, r8
100027b4:	439a      	bics	r2, r3
100027b6:	4690      	mov	r8, r2
100027b8:	2380      	movs	r3, #128	; 0x80
100027ba:	00db      	lsls	r3, r3, #3
100027bc:	4646      	mov	r6, r8
100027be:	401e      	ands	r6, r3
100027c0:	4642      	mov	r2, r8
100027c2:	421a      	tst	r2, r3
100027c4:	d012      	beq.n	100027ec <_ntoa_long+0x64>
100027c6:	2c00      	cmp	r4, #0
100027c8:	d022      	beq.n	10002810 <_ntoa_long+0x88>
100027ca:	2600      	movs	r6, #0
100027cc:	e00e      	b.n	100027ec <_ntoa_long+0x64>
100027ce:	3330      	adds	r3, #48	; 0x30
100027d0:	b2d9      	uxtb	r1, r3
100027d2:	1c77      	adds	r7, r6, #1
100027d4:	ab0a      	add	r3, sp, #40	; 0x28
100027d6:	5599      	strb	r1, [r3, r6]
100027d8:	0029      	movs	r1, r5
100027da:	0020      	movs	r0, r4
100027dc:	f000 ffd6 	bl	1000378c <__wrap___aeabi_uidiv>
100027e0:	42ac      	cmp	r4, r5
100027e2:	d316      	bcc.n	10002812 <_ntoa_long+0x8a>
100027e4:	2f1f      	cmp	r7, #31
100027e6:	d814      	bhi.n	10002812 <_ntoa_long+0x8a>
100027e8:	003e      	movs	r6, r7
100027ea:	0004      	movs	r4, r0
100027ec:	0029      	movs	r1, r5
100027ee:	0020      	movs	r0, r4
100027f0:	f000 ffcc 	bl	1000378c <__wrap___aeabi_uidiv>
100027f4:	b2cb      	uxtb	r3, r1
100027f6:	2b09      	cmp	r3, #9
100027f8:	d9e9      	bls.n	100027ce <_ntoa_long+0x46>
100027fa:	4642      	mov	r2, r8
100027fc:	0692      	lsls	r2, r2, #26
100027fe:	d505      	bpl.n	1000280c <_ntoa_long+0x84>
10002800:	2141      	movs	r1, #65	; 0x41
10002802:	18c9      	adds	r1, r1, r3
10002804:	b2c9      	uxtb	r1, r1
10002806:	390a      	subs	r1, #10
10002808:	b2c9      	uxtb	r1, r1
1000280a:	e7e2      	b.n	100027d2 <_ntoa_long+0x4a>
1000280c:	2161      	movs	r1, #97	; 0x61
1000280e:	e7f8      	b.n	10002802 <_ntoa_long+0x7a>
10002810:	0027      	movs	r7, r4
10002812:	4643      	mov	r3, r8
10002814:	9306      	str	r3, [sp, #24]
10002816:	9b20      	ldr	r3, [sp, #128]	; 0x80
10002818:	9305      	str	r3, [sp, #20]
